:020000040800F2
:10800000A8C20020A1810008A9810008DD9F000806
:10801000AD810008AF810008B181000800000000B8
:10802000000000000000000000000000B381000814
:10803000B581000800000000B7810008B981000880
:10804000BB810008BB810008BB810008BB81000820
:10805000BB810008BB810008BB810008BB81000810
:10806000BB810008BB810008BB810008BB81000800
:10807000BB810008BB810008979200089B92000812
:10808000BB8100089F920008BB810008BB810008EB
:10809000BB810008BB810008BB810008BB810008D0
:1080A000BB810008BB810008BB810008BB810008C0
:1080B000399D0108BB810008BB810008BB81000815
:1080C000BB810008BB810008BB810008BB810008A0
:1080D000BB810008BDA60108C1A60108C5A601080C
:1080E00053960008BB810008BB810008BB810008D3
:1080F000BB810008BB810008BB810008A392000877
:10810000BB810008BB810008BB810008BB8100085F
:10811000B5A60108B9A60108BB810008BB8100080B
:10812000BB810008BB810008BB810008BB8100083F
:10813000BB810008BB810008BB810008BB8100082F
:10814000BB810008BB810008BB810008BB8100081F
:10815000BB810008A7920008AB920008C9A60108DD
:10816000BB810008BB810008BB810008BB810008FF
:10817000BB810008BB810008BB810008BB810008EF
:10818000BB810008BB810008DFF810D000F0BEFB07
:10819000004800478DC30108AFF30080A8C200204B
:1081A0000648804706480047FEE7FEE7FEE7FEE791
:1081B000FEE7FEE7FEE7FEE7FEE7FEE7DD9C0108DF
:1081C000898100082DE9F0410024061B254671F144
:1081D000000605DA01240027D0EB070067EB010158
:1081E000161E73F1000605DA0027D2EB07020125FF
:1081F00067EB030300F077FA86460E4617469C4667
:10820000AC4204D00025D0EB050E65EB010624B18D
:108210000020D2EB000760EB030C704631463A4673
:108220006346BDE8F081202A06DBCB17203A41FAED
:1082300002F043EAE07306E041FA02F3D040C2F1F3
:108240002002914008431946704740EA01039B070A
:1082500003D009E008C9121F08C0042AFAD203E0BB
:1082600011F8013B00F8013B521EF9D27047421E43
:1082700012F8013F002BFBD111F8013B02F8013B42
:10828000002BF9D17047421C10F8011B0029FBD1CB
:10829000801A704730B505460020034600E05B1C9D
:1082A000934205D2EC5CC85C201A01D1002CF6D1B7
:1082B00030BD2DE9FE4F804681EA0300C00F0C4619
:1082C000009021F0004123F00045B8EB0200A941E5
:1082D00005D24046214690461C460B46024623F0F6
:1082E0000040104347D0270DC7F30A00C3F30A51DB
:1082F0000290401A019040286BDAC3F3130040F457
:10830000801B0098924620B10023D2EB030A63EB56
:108310000B0B01985946C0F14002504600F014FA88
:1083200006460D4650465946019AFFF77CFF10EB72
:1083300008006141002487EA115284EAE7731A4376
:1083400040D0009A62B3019A012A4FEA075215DC25
:10835000001B61EB02014FF0004202EA0752CDE937
:108360000042001C41F5801132462B4600F051FAC4
:1083700003B0BDE8F08F40462146F9E7001B61EBF2
:108380000201001C41F5801300185B412018A2F582
:10839000001747EB030140EAD570B6196D4111E0B3
:1083A0006D084FEA360645EAC0754FEA0752001BD2
:1083B00061EB0201001C41F5801149084FEA3000D1
:1083C0000019514132462B4603B0BDE8F04F00F092
:1083D00011BA0098012240000023D0EB020263EBA7
:1083E000E073009821464FEAE074B8EB000061EBBF
:1083F0000401E9E783F000435BE781F0004158E7BF
:108400002DE9FE4F81EA030404F0004421F000410D
:1084100000944FF0000B23F0004350EA01045ED0BB
:1084200052EA03045BD0C3F30A54C1F30A552C4447
:10843000A4F2F3340194A0FB0254C1F3130141F4FC
:108440008011C3F3130343F4801301FB024400FBC8
:10845000034E840A970A44EA815447EA8357A4FBEF
:10846000076802958D0A05FB07854FEA932C04FBEC
:108470000C542705029D4FEA065847EA1637B5EB1C
:1084800008056EEB070C870E920E47EA811742EA49
:108490008312A7FB0201B6EB0B0164EB00042B0D6A
:1084A00043EA0C335E1844EB1C50DA465146E7FBB6
:1084B0000201C5F313044FEA0B3343EA14534FEAA6
:1084C0000432019C43EA0603A4F10C040294009CCC
:1084D000CDE900B400F09DF903B0BDE8F08F0020B5
:1084E0000146F9E72DE9F04D81EA030404F0004B61
:1084F00021F0004514464FF0000A23F0004150EAF5
:10850000050220D054EA01021DD0C5F30A570246E5
:10851000C5F31303C1F31300C1F30A5640F48015E9
:1085200043F48013A7EB0608101BD64608F2FD386B
:1085300073EB050002D308F1010801E092185B41DA
:10854000B8F1000F03DA00200146BDE8F08D0020ED
:108550004FF48011064684460EE0171B73EB0507A7
:1085600005D3121B63EB050306434CEA010C4908D3
:108570004FEA300092185B4150EA0107EDD152EA10
:10858000030012D082EA040083EA0501084305D003
:10859000101BAB4106D20122002306E000224FF05F
:1085A000004302E06FF0010253101AEB06004CEB9F
:1085B000085110EB0A0041EB0B01BDE8F04D00F053
:1085C00019B90EB5C10F80EAE0700844CA0700214E
:1085D00040F233438DE80E000A460B4600F019F9CD
:1085E00003B000BD0EB540F2334102910021CDE948
:1085F00000110A460B4600F00CF903B000BD3EB571
:10860000CA17CB0F002450405140C0186141DA070F
:1086100040F233430094CDE901232246234600F083
:10862000F8F803B030BD70B5C1F30A5201F000454F
:108630000024C1F3130140F2FF3341F480119A4248
:1086400001DA002070BD40F233439A42A2F2334275
:1086500003DC524200F087F800E090402C43F1D058
:10866000404270BD70B5C1F30A5201F000450024CC
:10867000C1F3130140F2FF3341F480119A4202DA50
:108680000020014670BD40F233439A42A2F23342C9
:1086900003DC524200F067F801E000F055F82C438B
:1086A000F0D00023D0EB030063EB010170BD01F0BB
:1086B000004330B421F0004150EA010206D00A0D17
:1086C000A2F56072C1F31301002A02DC30BC002065
:1086D0007047440F44EAC104C100E01830BC00EB0D
:1086E000C25000F050B82DE9F05F054600209246D8
:1086F0009B4688460646814640241BE02846414664
:108700004746224600F02FF853465A46C01A914178
:1087100010D311461846224600F016F82D1A67EBC2
:1087200001084F4622460120002100F00DF817EB0A
:1087300000094E41201EA4F10104DFDC4846314609
:108740002A464346BDE8F09F202A04DB203A00FA7F
:1087500002F1002070479140C2F1200320FA03F398
:10876000194390407047202A04DB203A21FA02F096
:108770000021704721FA02F3D040C2F1200291405B
:108780000843194670470029A8BF7047401C49009C
:1087900008BF20F00100704710B4B0FA80FC00FA66
:1087A0000CF050EA010404BF10BC704749B1CCF191
:1087B000200421FA04F411FA0CF118BF012121431D
:1087C0000843A3EB0C01CB1D4FEA00614FEA1020D8
:1087D00042BF002010BC704700EBC350104400297A
:1087E000A4BF10BC7047401C490008BF20F0010026
:1087F00010BC704710B5141E73F1000408DA401C59
:1088000041F1000192185B411A4301D120F00100AF
:1088100010BD2DE9F04D92469B4611B1B1FA81F29F
:1088200002E0B0FA80F220329046FFF78DFF044656
:108830000F4640EA0A0041EA0B0153465A460843F4
:1088400013D0114653EA010019D0C8F14002504636
:10885000FFF789FF05460E46504659464246FFF748
:1088600073FF084305D0012004E020463946BDE8E7
:10887000F08D0020054346EAE0762C4337430A9802
:108880006305E40AA0EB08000022FD0A44EA47540D
:108890000A3002D500200146E9E7010510196941B7
:1088A000DDE9084500196941BDE8F04DA2E770B562
:1088B00021F0004303430CD0C1F30A550024D5EB4B
:1088C000040564EB0403D617AD1AB34102DB0020A4
:1088D000014670BD201841EB025170BD30B5041E39
:1088E00071F1000404DB4FF00044404264EB0101ED
:1088F000141E73F1000405DB1C464FF00043524286
:1089000063EB0403994208BF904230BD064C074D0B
:1089100006E0E06840F0010394E80700984710344F
:10892000AC42F6D3FFF734FC68F2010888F2010884
:108930002DE9F04D00231A461B1A8A4103DB002063
:108940000146BDE8F08DC1F30A52C1F3130141F4B1
:1089500080154FF0000BD10702D100186D41521E57
:108960000027044640F2FF11384601EB620A3E46FA
:108970008046024600204FF48011FFF7F4FEC21932
:108980007141BB1846EB0100B4EB030C75EB000C16
:1089900004D3E41A65EB000517460E46241908F1C6
:1089A00001006D4180463428E3DDF91946EB0600ED
:1089B000091BA84103D24FF0FF32134601E0002209
:1089C00013461BEB070046EB0A51BDE8F04DFFF7DD
:1089D00011BF000030B5041E71F1000404DB4FF03C
:1089E0000044404264EB0101141E73F1000405DBF6
:1089F0001C464FF00043524263EB04038B4208BF16
:108A0000824230BD70B58C1810F8015B15F0070379
:108A100001D110F8013B2A1106D110F8012B03E017
:108A200010F8016B01F8016B5B1EF9D12B0705D41F
:108A30000023521E0DD401F8013BFAE710F8013B68
:108A4000CB1A921C03E013F8015B01F8015B521E84
:108A5000F9D5A142D8D3002070BD027803E010F808
:108A6000013B1A44D2B2491E89B2F8D2104670476F
:108A700070B5ADF5287D00260D46ADF89462ADF8D1
:108A8000986200EB40012D4800EBC104608AA842C7
:108A900051D9ADF898624AE0A089228A284481B26F
:108AA000274800F0B1F8ADF894626A46208A0BE0DE
:108AB000BDF894326168C95CBDF89432D154BDF8F8
:108AC0009412491CADF89412BDF894128842EFD864
:108AD000401E81B21046FFF7C0FF1A498870228AF3
:108AE0000DF1FF31515C814219D1ADF894620CE077
:108AF000BDF894126068BDF89422405CA168885467
:108B0000BDF89402401CADF89402208ABDF894127E
:108B1000401E8842ECDC01200DF5287D70BD6420EC
:108B200013F0C4FABDF89802401CADF89802BDF8E5
:108B300098020628B0D30020EEE700005CD00108C0
:108B4000107C0020220A0020F0B50D46064600EBFE
:108B500046011C48002200EBC104ADF5257D608A6A
:108B6000A8422BD9694606E0A0686368805C9854E7
:108B70008854521C92B2208A401E9042F4DC208A13
:108B8000401E81B26846FFF768FF228A0DF1FF316F
:108B900000275054A089228A284481B2684600F0F8
:108BA0002FF929463046FFF763FF012807D06420DC
:108BB00013F07CFA7F1CBFB2062FEBD300200DF51B
:108BC000257DF0BD5CD0010838B50025ADF800501A
:108BD0000FF036F90A4C207000F088F82178094827
:108BE000242907D0272908D0282902D1022180F87A
:108BF000E51138BD80F8E55138BD0121F7E70000E7
:108C0000220A0020A42200202DE9F0410646154644
:108C10000C46012080F31088254F0020B8800FF00B
:108C2000EFF8000609D4012013F040FAB888401C80
:108C300080B2B880C828F2D335E0B888C82832D2CC
:108C40001C4F1021384601F0BCF90821384601F0CC
:108C5000BAF9E82000F030F8C4F3871000F02CF8DF
:108C6000A006000E00F028F8002000F025F80024EF
:108C7000002000F021F8641CA4B2042CF8D30024D6
:108C800005E0FF2000F018F83055641CA4B2AC4297
:108C9000F7D31021384601F096F9002080F31088B0
:108CA0000120BDE8F081002080F31088F9E7000082
:108CB000220A00200000024070B50B4C054602213C
:108CC00020460FF0B7F90028F9D0294620460FF0CA
:108CD000BAF9012120460FF0ADF90028F9D020465D
:108CE0000FF0AFF9C0B270BD0030014010B50120E7
:108CF00080F310881A4C0020A0800FF081F8000645
:108D000009D4012013F0D2F9A088401C80B2A080C1
:108D1000C828F2D320E0A088C8281DD2114C102109
:108D2000204601F04EF90821204601F04CF93D2083
:108D3000FFF7C2FF2A20FFF7BFFF8020FFF7BCFF2D
:108D4000A720FFF7B9FF1021204601F03CF90020D1
:108D500080F31088012010BD002080F3108810BD22
:108D6000220A0020000002402DE9F04106460D468F
:108D7000012080F31088204C0020A0800FF040F8E4
:108D8000000609D4012013F091F9A088401C82B29A
:108D9000A280C82AF2D32AE0A088C82827D2174F79
:108DA0001021384601F00DF90821384601F00BF981
:108DB0008420FFF781FF0020FFF77EFF0020FFF7F0
:108DC0007BFF0020FFF778FF002404E0305DFFF711
:108DD00073FF641CA4B2AC42F8D31021384601F0F2
:108DE000F2F8002080F310880120BDE8F081002017
:108DF00080F31088F9E70000220A002000000240FA
:108E000070B50D46012181F310881146FFF7ACFFC4
:108E1000002832D01B4C0020A0800EF0F1FF00068D
:108E200009D4012013F042F9A088401C80B2A08030
:108E3000C828F2D322E0A088C8281FD2124C1021E3
:108E4000204601F0BEF80821204601F0BCF883203E
:108E5000FFF732FFC5F38710FFF72EFFA806000EBD
:108E6000FFF72AFF0020FFF727FF1021204601F01F
:108E7000AAF8002080F31088012070BD002080F344
:108E8000108870BD220A00200000024010B50023A7
:108E90001A4604E010F8014B6340521CD2B28A42D9
:108EA000F8D3184610BD000010B50446392013F061
:108EB000FDFAE0B213F01AFBC4F3072013F016FB1F
:108EC000C4F3074013F012FB200E13F00FFB4FF416
:108ED0008051034801F077F8BDE8104011F0E6BC7E
:108EE000000402402DE9F041054614460E463A20A2
:108EF00013F0DCFAF0B213F0F9FA300A13F0F6FAD4
:108F0000104F4FF480563146384601F05CF8B046B9
:108F10003E4611F0CBFC1D2811D1284600F0A4F8E4
:108F200007463B2013F0C2FA4146304601F04BF8A9
:108F30003D44002CEDD0208838442080E9E7BDE88E
:108F4000F0810000000402402DE9F041054614467E
:108F50000E463C2013F0AAFAF0B213F0C7FA300A1A
:108F600013F0C4FA114F4FF480563146384601F0E1
:108F70002AF80CB100202080B0463E4611F096FC45
:108F80001E2811D1284600F017F907463D2013F09E
:108F90008DFA4146304601F016F83D44002CEDD0E4
:108FA000208838442080E9E7BDE8F08100040240D1
:108FB00010B50EF06DFE08B100F028F8BDE81040C5
:108FC000302000F09FB80146362000F089B810B577
:108FD00008B100F0A5F8BDE81040342000F092B8C8
:108FE00010B5044600F09CF820785C2801D02F28AA
:108FF00003D10021642000F0FBF8BDE810403220CE
:1090000000F080B8682000F04BB8000010B52220B6
:1090100013F04CFA13F040FA04464FF48051024822
:1090200000F0D1FF204610BD000402402DE9F041C0
:1090300013F032FA064613F02FFA054613F02CFA15
:10904000044613F029FA07464FF48051054800F012
:10905000BAFF46EA052040EA044040EA0760BDE85E
:10906000F08100000004024070B50546272013F08F
:109070001DFA13F011FA0446260007D013F00CFA7B
:10908000641E05F8010B14F0FF04F7D14FF4805172
:10909000024800F098FF304670BD00000004024016
:1090A00010B504460C2013F001FA204613F01EFA06
:1090B000BDE81040FFF7BABF10B504460A2013F010
:1090C000F5F9204613F012FA13F0E6F904464FF4CE
:1090D0008051024800F077FF204610BD0004024096
:1090E00010B50C4613F0E2F9204613F0FFF94FF4E7
:1090F0008051034800F067FFBDE8104011F0D6BB77
:109100000004024010B513F0D1F94FF48051034828
:1091100000F059FFBDE8104011F0C8BB0004024048
:1091200070B50546012013F0C1F913F0B5F94328D5
:1091300028D22B20FFF7C0FF102823D22F2013F0B6
:10914000B5F9002013F0D2F93220FFF7DBFF142825
:1091500018D1CF20FFF7B0FF040013D04C20FFF749
:109160009FFF00EB04214C2000F042F85020FFF755
:1091700097FF00EB0421502000F03AF80021702006
:1091800000F036F82F2013F091F92C7806E015F84E
:10919000014F5C2C01D02F2C00D10024204613F06D
:1091A000A5F9002CF3D1BDE870404FF4805101487F
:1091B00000F009BF0004024070B505462D2013F0F1
:1091C00075F913F069F90446260007D0287813F0E2
:1091D0008DF9641E6D1C14F0FF04F7D14FF480511B
:1091E000024800F0F0FE304670BD0000000402406E
:1091F00070B505460C460D2013F058F9284613F0BB
:1092000075F9E0B213F072F9C4F3072013F06EF9A8
:10921000C4F3074013F06AF9200E13F067F9BDE8B4
:1092200070404FF48051014800F0CDBE0004024070
:1092300070B5094DFF22134605F5807605E010F85C
:10924000014B54402A5D5A40335D491E89B2F6D223
:1092500042EA032070BD0000E9CD010870B500228C
:109260001346154605E010F8014BA2186B41491E44
:1092700089B20029F7D1100C40EA034092B280185D
:1092800045EB13414FEA014242EA104108186FEAE8
:10929000000080B270BD08F001BE08F09FBD08F06C
:1092A0006DBD08F0CBBD0AF053B80EF063B90000F5
:1092B000074A904201D2074801E005481038064AA3
:1092C0008B0001EA020101D5C160704781607047DF
:1092D00010640240006002407D0F7D0F002901688C
:1092E00002D041F0010101E021F00101016070476D
:1092F0002DE9F043016821F00101016000210160C6
:1093000041608160C1600161212141613C493C4A69
:109310003D251039904202D18D60BDE8F083384A76
:109320004FF474661832904201D18E60F5E7344AEA
:109330004FF474173032904201D18F60EDE7304A1C
:109340004FF0746C4832904202D1C1F808C0E4E793
:109350002B4B2C4A6033984201D1CA60DDE7284C80
:10936000294B7834A04201D1CB60D6E7DFF890805A
:10937000264C08F19008404501D1CC60CDE7DFF8DC
:1093800080804FF03D5908F1A808404502D1C1F84E
:109390000C90C2E71E49DFF878800839404501D1BA
:1093A0000D60BAE71A4D1835A84201D10E60B4E736
:1093B000174D3035A84201D10F60AEE7144D483546
:1093C000A84202D1C1F800C0A7E7114D104960358D
:1093D000091FA84201D10A609FE70D4A78329042E6
:1093E00001D10B6099E70A4A9032904201D10C609A
:1093F00093E7074AA83290428FD1C1F800908CE7DA
:10940000106002403D000020400F002000003D2081
:10941000106402400B0607D5436912B143F0800384
:1094200001E023F080034361802908D0002A02680C
:1094300001F01E0101D00A4300E08A430260704738
:1094400030B50368124ACC6813400A682243D1E958
:1094500005452C432243CC6922430C6A22434C6AC3
:1094600022438C6A22434C6B22438C6B22431A4367
:109470000260426922F00703D1E90B2422431A4318
:1094800042610A6942604A6882608968C16030BD91
:109490003F801CF02DE9FC41012120200EF000FC52
:1094A00001268DF8046000258DF8065003208DF804
:1094B00005001B4C302700978DF807506946204661
:1094C00000F02CFD3021204600F07DFD154C84F885
:1094D000705684F8725684F8716684F873664FF497
:1094E000FA70C4F8780600F01FF894F8E8038028B2
:1094F00014D1A4F580508565232084F8ED03052060
:1095000084F8EC0384F8EB73142084F8EA03202039
:1095100084F8E90384F8E85300F042F8BDE8FC81E0
:1095200000140240A42200207CB512F093FED0204B
:1095300012F060FE12F0C2FE002012F05BFE12F08C
:10954000BDFE12F087FED12012F054FE12F0B6FEDE
:1095500000246D4601E0062C01D2012000E000202D
:1095600012F018FE2855641CE4B2072CF3D312F055
:109570008BFE0A489DF8061041719DF80510017197
:109580009DF80410C1709DF8021081709DF80110C3
:1095900041709DF8001001707CBD00008C260020F9
:1095A0007CB51848002401788DF8001041788DF8BA
:1095B000011081788DF8021001218DF80310C17817
:1095C0008DF8041001798DF8051040798DF80600AA
:1095D00012F040FED02012F00DFE12F06FFE0020BF
:1095E00012F008FE12F06AFE6D46285D12F002FECF
:1095F00012F064FE641CE4B2072CF6D312F044FEB1
:109600007CBD00008C26002070B5094D0022134659
:1096100005F5807605E010F8014B54402A5D5A406C
:10962000335D491E89B2F6D242EA032070BD0000C4
:10963000E9CD0108072A00D9072240EA002021B11C
:10964000012901D1D040C0B270479040C0F307203B
:1096500070477047072A00D9072240EA002029B145
:10966000012902D19040C0F307207047D040C0B21A
:109670007047000070B5ADF5327D00260D46ADF89F
:10968000BC62ADF8C06200EB4001324800EBC1049F
:10969000608AA8425CD9ADF8C06255E0012264211D
:1096A0002D4800F0BFF92C4800788DF800003828CC
:1096B00042D1228AE06802FB0501274800F0B2F996
:1096C000ADF8BC626A46208A0BE0BDF8BC32616826
:1096D000C95CBDF8BC32D154BDF8BC12491CADF810
:1096E000BC12BDF8BC128842EFD8401E81B21046B1
:1096F00000F05AFA228A0DF1FF31515C81421BD1F0
:10970000ADF8BC620EE0BDF8BC226168895CA2685D
:1097100000FB0520BDF8BC221154BDF8BC02401C62
:10972000ADF8BC02208ABDF8BC12401E8842EADCBB
:1097300001200DF5327D70BD642012F0B7FCBDF83C
:10974000C002401CADF8C002BDF8C0020628A5D377
:109750000020EEE7B0C9010834570020F0B50E46EE
:10976000074600EB47012648ADF5317D002500EBAB
:10977000C1048DF8BC52608AB0423DD90021084630
:10978000FFF778FF012837D1694609E0A268401E3B
:1097900000FB06206268285C505548556D1CADB230
:1097A000208AA842F2D80025208AE16800FB061131
:1097B000401E82B2134800F0B3F9208A401E81B2E5
:1097C000684600F0F1F98DF8BC02208AE1680122B8
:1097D00001447043401E0144AFA800F0A1F9314696
:1097E0003846FFF747FF012807D0642012F05EFCDF
:1097F0006D1CADB2062DD7D300200DF5317DF0BD27
:10980000B0C90108345700202DE9F041ADF5307D95
:10981000354D4FF000088DF8BC82344EA5F800801D
:1098200000243FE000206F4607E056F832204968E8
:10983000125C0A543A54401C80B2298801EB410260
:1098400006EBC2010B8A5B1E8342EEDC288800EB2C
:10985000400006EBC000008A401E81B2384600F08E
:10986000A3F98DF8BC02288800EB400006EBC0008D
:10987000C168008A00FB0411401E82B21C4800F03F
:109880004FF92888012200EB400006EBC000C168B8
:10989000008A01446043401E0144AFA800F040F933
:1098A000641CA4B2288800EB400006EBC000408A8C
:1098B000A042B7D82888401C80B228800B28AFD39C
:1098C0000C48017821F001010170017841F0060196
:1098D0000170A0F8028000210120FFF73FFF0DF585
:1098E000307DBDE8F081000010000020B0C9010803
:1098F00034570020802400207CB5012108460EF05A
:10990000CFF901208DF8040002258DF805500024C0
:109910008DF806408DF807001820154E0090694616
:10992000304600F0FBFA05221146304600F032FBCB
:1099300005220621304600F02DFB05220721304686
:1099400000F028FBA02000908DF8045003208DF833
:1099500005008DF806408DF807406946304600F056
:10996000DDFA402000906946304600F0D7FA7CBD11
:1099700000000240F8B5002634460096FFF7BCFF11
:1099800000F0A0F82248641C8442FCD3214C08213A
:10999000204600F016FB1021204600F014FB0620A4
:1099A00000F076F80821204600F00DFB0821204643
:1099B00000F007FB1021204600F005FB012000F01D
:1099C00067F8002000F064F80821204600F0FBFA58
:1099D0001148D0F81C0208B9FFF716FF0F4D2E8072
:1099E0000F4E002405E0C0B22146FFF743FE641C81
:1099F000A4B2288800EB400106EBC101498AA142CC
:109A0000F1D880B2401C80B228800B28E9D3F8BD81
:109A1000FFFF0F0000000240000043421000002042
:109A2000B0C901082DE9F0410546002416460F464D
:109A3000012080F31088DFF854800821404600F0B0
:109A4000C0FA1021404600F0BEFA032000F020F8D2
:109A5000C7F3074000F01CF8C7F3072000F018F820
:109A6000F8B200F015F806E0002000F011F8641CD0
:109A700005F8010BA4B2B442F6D30821404600F029
:109A8000A2FA002080F31088BDE8F08100000240B7
:109A900070B50B4C0546022120460EF0CBFA00288B
:109AA000F9D0294620460EF0CEFA012120460EF0CC
:109AB000C1FA0028F9D020460EF0C3FAC0B270BD3A
:109AC0000030014010B5012186B008030EF024F9E2
:109AD000124C20460EF084FA0021ADF808106015F3
:109AE000ADF80A003820ADF80C000720ADF80010E2
:109AF000ADF81000ADF804104FF48270ADF8061008
:109B0000ADF80E10ADF80200694620460EF09DFA41
:109B1000012120460EF05AFA06B010BD0030014077
:109B20002DE9F0410546002416460F46012080F33A
:109B30001088DFF870800821404600F042FA1021BA
:109B4000404600F040FA0620FFF7A2FF08214046F9
:109B500000F039FA0821404600F033FA102140465F
:109B600000F031FA0220FFF793FFC7F30740FFF739
:109B70008FFFC7F30720FFF78BFFF8B2FFF788FFCF
:109B800005E02878FFF784FF641CA4B26D1CB44282
:109B9000F7D30821404600F016FA002080F3108821
:109BA000BDE8F08100000240027803E010F8013BBC
:109BB0001A44D2B2491E89B2F8D21046704700004A
:109BC00070B51E4A907B012825D1002595731C494C
:109BD0001C480F244E780123F6B14D70D0F828525E
:109BE000D0F8346245EAC605D0F83062D0F82C02CD
:109BF000B60046EA40000543AC43CC708878CC7888
:109C0000A04208D108710C78A04204D010720870EC
:109C1000002800D0D37170BD4B70D0F82852D0F816
:109C2000346245EAC605D0F83062D0F82C02B6009E
:109C300046EA40000543AC438C70DFE7A4120020E5
:109C4000C90A0020000042422DE9F041ADF57C7DBB
:109C500000273D46ADF8E873FFF7AAF9142808D0AD
:109C6000664880F8E75312F05DFB0DF57C7DBDE89A
:109C7000F0816348FFF7B4F9614C103C1428207060
:109C800006D0422879D00120FFF79DF92570ECE736
:109C9000FFF7B8F9C4E90205A046BDF8E803FFF7ED
:109CA00003F9FAAA4FF4FA716846FFF71BF955A1B8
:109CB000684612F09BFBA080544C6E46F0B1E1194F
:109CC00001F5805181F83F577F1CBFB2282FF6D392
:109CD000474630444EA112F089FB78800021001FD6
:109CE0000AE0BA880A443244D378621802F58052F6
:109CF00082F83F37491C89B28142F2DB45A16846B0
:109D000012F074FB4746A8F80400F0B10021621875
:109D100002F5805282F86757491C89B22829F6D388
:109D200030443BA112F062FB7880002109380AE040
:109D3000BA880A443244137A621802F5805282F8D3
:109D40006737491C89B28142F2DB35A1684612F0BF
:109D50004DFBB880F8B10021621802F5805282F8FC
:109D60008F57491C89B21429F6D3304428A112F028
:109D70003DFB788000210D380BE03AE0BA880A44B8
:109D80003244137B621802F5805282F88F37491CE7
:109D900089B28142F2DB26A1684612F027FBB88027
:109DA000F0B10021621802F5805282F8F956491C80
:109DB00089B23229F6D3304415A112F017FB78800E
:109DC0000021C01F0AE0BA880A443244937962181D
:109DD00002F5805282F8F936491C89B28142F2DBE1
:109DE00000210320FFF7BAFC0120FFF7ECF8012067
:109DF0003BE70348FFF7EBF837E70000A422002019
:109E0000380A002041504E3D00000000A4120020FE
:109E10003B000000574946494E414D453D0000007A
:109E20005749464950415353574F52443D00000053
:109E30005345525645523D002F4910B5884206D130
:109E4000012108460DF038FF002101204FE02B4989
:109E5000884206D1012102200DF02EFF00210220B0
:109E600045E02749884206D1012104200DF024FF56
:109E7000002104203BE02349884206D1012108202B
:109E80000DF01AFF0021082031E01F49884206D159
:109E9000012110200DF010FF0021102027E01B49A8
:109EA000884206D1012120200DF006FF002120204C
:109EB0001DE01749884206D1012140200DF0FCFE2B
:109EC0000021402013E01349884206D1012180205F
:109ED0000DF0F2FE0021802009E00F4988420AD1EE
:109EE0008415012120460DF0E7FE00212046BDE843
:109EF00010400DF0E1BE10BD000002400004024021
:109F000000080240000C0240001002400014024011
:109F100000180240001C024000200240F0B5002260
:109F200001274FF0030C0B6807FA02F52B40AB42F8
:109F30002CD1066853000CFA03F4A64306600E7990
:109F4000D0F800E09E4046EA0E0606600E79012E2B
:109F500001D0022E12D18668A64386604E79D0F8D1
:109F600008E09E4046EA0E0686604668AE434660BC
:109F700045688E799640B6B235434560C568A543BD
:109F8000C560CC799C40C3681C43C460521C102A35
:109F9000C9D3F0BD4B07DB0E9A40C90810B500EBE2
:109FA0008100016A0F249C40A1430162016A1143B0
:109FB000016210BD0246002012690A4200D0012051
:109FC0007047418370470183704700000249087A57
:109FD00000220A7270470000A412002002480068A4
:109FE000C00700D000BEFEE7F0ED00E002494AF6EF
:109FF000AA200860704700000030004010B512F041
:10A0000091F9BDE81040642012F050B82DE9F04FEE
:10A0100083466AA0ADF57D7D002500689A460F460F
:10A02000A946FB90ADF8E853042A25D8644C94F86F
:10A03000EC03302101EB101302EBC20000EB021223
:10A0400060481618337194F8EC0300F00F003030BC
:10A05000707194F8EB0301EB1010B07194F8EB03FE
:10A0600000F00F003030F071FEF7A2FF142807D087
:10A0700084F8E79312F056F90DF57D7DBDE8F08F79
:10A08000DFF84081A8F1240898F8000014280ED0C9
:10A090003046FEF7A5FF88F80000142807D04228B4
:10A0A0007ED00120FEF78FFF88F80090E4E74FF4A0
:10A0B0007A70874200D90746FEF7A4FFC8E9020973
:10A0C0004E46FEF7F1FE94F8EB13302000EB111131
:10A0D0008DF8001094F8EB1301F00F0130318DF87A
:10A0E000011094F8EA1300EB11118DF8021094F8A6
:10A0F000EA1301F00F0130318DF8031094F8E913E1
:10A1000000EB11118DF8041094F8E91301F00F0120
:10A1100030318DF8051094F8E81300EB11108DF82C
:10A12000060094F8E80300F00F0030308DF80700C7
:10A13000BAF1000F03D0BAF1010F02D004E05420AD
:10A1400000E052208DF808003A208DF809000A231B
:10A150006C4617E00BEB550108780009B0FBF3F2F1
:10A16000C2EBC2021044621930309072087800F0DD
:10A170000F00B0FBF3F1C1EBC10108443030AD1C5E
:10A18000D072ADB2B5EB470FE4D303EB470081B219
:10A19000FAAA2046FEF7D8FEFAAA0221FBA800E0A0
:10A1A00007E0FEF7D1FE0120FEF70DFF88F8006002
:10A1B00062E73046FEF70BFF5EE700000D0A000085
:10A1C000A42200204C0A00202DE9F04F00272DED9D
:10A1D000028B9FB08DF824708DF804708DF800709C
:10A1E000CDE91077CDE90A778DF808708DF80C70FD
:10A1F0008DF820708DF81470ADF818709FEDFE0A80
:10A20000DFF8F8938DED010AFD4C41F6865504F117
:10A210002900079004F59C5004F5804A01264FF070
:10A22000D50BDFF8E08304F580540490A0E094F8A7
:10A230002A0B28B384F82A7BBAF83C14D9F88C206E
:10A240004846C2F57A7291421AD1D0F88C00C0F516
:10A250007A70AAF83404E94800218830FFF73EF804
:10A26000E648E9498830FFF723F888F800604FF4A2
:10A270007A70C9F88C00E14801218830FFF72EF888
:10A2800094F8360B20B384F8367BBAF83E14D9F82C
:10A2900044204846C2F57A72914219D1406CC0F50B
:10A2A0007A70AAF83604D54800214030FFF716F836
:10A2B000D248D6494030FEF7FBFF88F801604FF4E2
:10A2C0007A70C9F84400CD4801214030FFF706F804
:10A2D00094F8420B20B384F8427BBAF84014D9F8C2
:10A2E00014204846C2F57A72914219D14069C0F5EE
:10A2F0007A70AAF83804C14800211030FEF7EEFF4A
:10A30000BE48C3491030FEF7D3FF88F802604FF40F
:10A310007A70C9F81400B94801211030FEF7DEFF49
:10A3200094F84E0B20B384F84E7BBAF84214D9F857
:10A330002C204846C2F57A72914219D1C06AC0F504
:10A340007A70AAF83A04AD4800212830FEF7C6FF1B
:10A35000AA48B0492830FEF7ABFF88F803604FF4F5
:10A360007A70C9F82C00A54801212830FEF7B6FF05
:10A3700094F82A0B94F8361B084494F8421B94F87E
:10A380004E2B1144C8427FF452AF06F07DB80178DD
:10A3900019B107708DF8087010E0417819B1477055
:10A3A0008DF808600AE0817811B18770022003E01F
:10A3B000C17819B1C77003208DF808009DF8080016
:10A3C00000EB400101EB00118D4800EB011000F59E
:10A3D000805090F85A1D9DF8080000EB4002C2EB37
:10A3E000C0128D4810F83200C1280BD19DF808002A
:10A3F00000EB4002C2EBC012874800EBC20080783D
:10A4000008280CD0082986F00980DFE811F0D71F52
:10A410002700ED0AF414BB1D811F082303278AF8C7
:10A420008C649DF8080030B1012807D002280FD0B5
:10A43000032808D10FE04FF4804101E04FF40051B0
:10A440007648FFF7BEFD7648C0F8887205F0E6BF93
:10A450004FF48051F4E74FF40061F1E79DF80800F4
:10A46000DFF8B48100EB4001C1EBC01108EBC10083
:10A470004078002107F0B4FB8DF820008DF80070C3
:10A48000DFF87C911BE09DF808009DF8001000EBC0
:10A49000400202EB001009EB001000EB011000F588
:10A4A000805090F8850D9DF8201088429DF800009E
:10A4B00002D18DF8200012E0401C8DF800009DF8BC
:10A4C000080000EB400101EB001009EB001000F563
:10A4D000805090F85B0D9DF800209042D3D89DF8F5
:10A4E000080000EB4001C1EBC01008EBC000807811
:10A4F0000A22B2EB101F9DF8080000EB4002C2EBED
:10A50000C01008EBC000807801D100F00F008DF87A
:10A510000C009DF80C0010B910208DF80C009DF86F
:10A5200008009DF80C1000EB4002C2EBC01208EBD3
:10A53000C20008444078ADF818009DF8080000EB10
:10A540004001C1EBC01108EBC1009DF80C10491C83
:10A5500007F027FF8DF804009DF8080000EB40018C
:10A56000C1EBC01108EBC1009DF80C1008448078C5
:10A570009DF80410884245F051879DF80800424636
:10A5800000EB4001C1EBC01008EBC0004078002890
:10A5900005F044879DF8080000EB4001C1EBC010B6
:10A5A0009DF80C1002EBC0000844C3789DF8080029
:10A5B00000EB001101EB002109EBC10C9DF820100C
:10A5C000484601EB01110CEBC10101F5005181F886
:10A5D00058329DF8081009EB01139DF8201019441A
:10A5E00001F5805181F8887B99F81810012938D13C
:10A5F0009DF8081016E00000000000000060024016
:10A60000A4120020120000200088002000802010EA
:10A610002080001000880010806400200018024094
:10A620000000424201EB410303EB01119DF8203091
:10A6300000EB011101EB031129440B7843F0800377
:10A640000B70BDF81810B62905D0C52903D0D5293F
:10A6500001D0D92903D19DF80C10032901D2ADF8FE
:10A660001870BDF81810CE2913D013DCB9297DD08D
:10A6700009DC5A298CD0B22979D0B529F7D0B6296E
:10A6800045F0CC86FDE3C32972D0C52971D0CA2913
:10A69000F6D1F7E3E129FCD006DCD52909D0D7298A
:10A6A000E8D0D929ECD1D8E2E5297CD0E729E7D157
:10A6B000E9E39DF8081001EB4103C3EBC11108EB7E
:10A6C000C101C97884F8E2119DF8081001EB01126C
:10A6D00002EB012100EBC1029DF8201001EB0111FA
:10A6E00002EBC10101F5005191F81C1201299DF8FE
:10A6F000081001EB41027DD002EB0112014600EB94
:10A7000002109DF82020C84600EB021094F8E221C8
:10A710002844A6EBD213027863F3000202709DF87E
:10A72000080000EB400202EB00109DF8202001EB36
:10A73000001000EB021094F8E2212844530902783B
:10A7400063F3410202709DF8080000EB400202EB47
:10A75000001001EB00129DF8200002EB001000F544
:10A76000805090F8860DC0F3400203E0FEE3FEE364
:10A77000FEE3FEE39DF8080000EB001303EB00206E
:10A7800008EBC0019DF8200000EB001001EBC000B9
:10A7900000F5005090F83402C0F34000824254D0DB
:10A7A0009DF8080000E0E5E300EB001101EB00205C
:10A7B0009DF82020414608EBC00002EB021200EB9E
:10A7C000C20042F2342210449DF8082002EB4203FA
:10A7D00003EB02129DF8203008EB021202EB031289
:10A7E00002F5805292F8862D5308027863F34102F5
:10A7F000027000E02AE09DF8080000EB400202EB46
:10A8000000109DF8202001EB001000EB021000F575
:10A81000805090F8860D80074AD59DF80800D9220F
:10A8200000EB001303EB002008EBC0019DF82000B3
:10A8300000EB001001EBC00000F5005080F8212271
:10A840009DF808100220FEF789FF79E002EB011164
:10A850009DF8202000EB011101EB021194F8E22198
:10A860002944A6EBD2130A7863F300020A709DF81C
:10A87000081001EB011202EB012100EBC10101F50F
:10A88000005181F817729DF80810022201EB0113A4
:10A8900003EB012100EBC1039DF8201001EB011136
:10A8A00003EBC10101F5005181F81C22B622FCE343
:10A8B0009DF8080000EB001202EB002001EBC00243
:10A8C0009DF8200000EB001002EBC00000F50050E6
:10A8D00080F829629DF80800D92200EB001303EBF1
:10A8E000002001EBC0039DF8200000EB001003EBFB
:10A8F000C00000F5005080F821229DF8080000EB10
:10A90000400202EB001001EB00129DF8200002EB68
:10A9100000104219107820F0200313709DF80800F1
:10A9200000EB001202EB002008EBC0019DF82000B4
:10A9300000EB001001EBC00000F5005080F85A62F7
:10A940009DF80800434600EB400101EB001008EBC6
:10A9500000119DF8200001EB001000F5805090F8E8
:10A96000860D00F001019DF8080000EB001202EBDB
:10A97000002008EBC0029DF8200000EB001002EB65
:10A98000C00000F5005090F8340200F00100814250
:10A9900071D09DF808009DF8202000EB001101EB1C
:10A9A0000020194603EBC00002EB021200EBC200CC
:10A9B00042F2342210449DF8082002EB420303EBDC
:10A9C00002129DF8203001EB021202EB031202F595
:10A9D000805292F8862D037862F3000303709DF88D
:10A9E000080000EB400202EB00109DF8202001EB74
:10A9F000001000EB021000F5805090F8860DC007A3
:10AA00009DF8080038D000EB001202EB002001EBAB
:10AA1000C0029DF8200000EB001002EBC00000F522
:10AA2000005090F85A0200289DF8080000EB001230
:10AA300002EB002001EBC0029DF8200000EB0010AB
:10AA400002EBC00000F5005038D080F859729DF834
:10AA5000080000EB400202EB001001EB00129DF831
:10AA6000200002EB00104219107820F0010313704F
:10AA700094F8A40728B3DBE000EB400202EB0010DF
:10AA80009DF8202001EB001000EB02102844027812
:10AA900022F0200303709DF8080000EB001202EB87
:10AAA000002001EBC0019DF8200000EB001001EB3D
:10AAB000C00000F5005080F85972B9E080F8596282
:10AAC000D6E7487E012868D1886D4A8B904264D2CF
:10AAD0009DF8080000EB001202EB002001EBC00221
:10AAE0009DF8200000EB001002EBC00000F50050C4
:10AAF00090F85902012850D19DF8080000EB00128F
:10AB000002EB002001EBC0029DF8200000EB0010DA
:10AB100002EBC00000F5005090F89302E8BB9DF8EE
:10AB2000080000EB400202EB001001EB00129DF860
:10AB3000200002EB001000F5805090F8842D9DF865
:10AB4000080000EB001303EB002001EBC00000F550
:10AB5000005080F815229DF80800C32200EB001376
:10AB600003EB002001EBC0039DF8200000EB001078
:10AB700003EBC00000F5005080F821229DF808008A
:10AB800000EB400202EB001008EB00119DF82000E2
:10AB900001EB001000F5805000E049E0C0F8887D2E
:10ABA0009DF808100220FEF7D9FD8DF8247041466B
:10ABB00019E09DF8080000EB001202EB002001EB09
:10ABC000C0039DF820009DF8242000EB001003EB4B
:10ABD000C000104400F5005080F85B729DF824001E
:10ABE000401C8DF824009DF824001428E1D38DF832
:10ABF000247019E09DF8080000EB001202EB002021
:10AC000001EBC0029DF8200000EB001002EBC00039
:10AC10009DF82420104400F5005080F877729DF8CC
:10AC20002400401C8DF824009DF824000A28E1D35C
:10AC30009DF808009DF8202000EB400101EB00107A
:10AC400008EB001000EB021000F5805090F8860D24
:10AC5000800745F1E383D9229EE19DF80810C8469C
:10AC600001EB410303EB011109EB011000F58050EA
:10AC700090F8600D00289DF80C0003D00A2845F0DC
:10AC8000CD8396E00828FAD18DF8247024E09DF851
:10AC9000080000EB4001C1EBC01002EBC0019DF8C1
:10ACA00024000844C07800F00F00092818D89DF847
:10ACB000080000EB4001C1EBC0109DF8241002EB2E
:10ACC000C0000844C07800F0F000902808D89DF833
:10ACD0002400401C8DF824009DF824000628D6D3BB
:10ACE0009DF824000628C5F099839DF8080000EB24
:10ACF0004001C1EBC01002EBC000C07801049DF818
:10AD0000080000EB4003C3EBC01002EBC000007969
:10AD100041EA00239DF8080000EB4001C1EBC010A0
:10AD200002EBC000407903439DF8080000EB0011DE
:10AD300001EB002008EBC00C9DF82000414600EB21
:10AD400000100CEBC00000F50050C0F835329DF843
:10AD5000080000EB4003C3EBC01002EBC000807999
:10AD600003049DF8080000EB400CCCEBC01002EB94
:10AD7000C000C07943EA00239DF8080000EB400CB6
:10AD8000CCEBC01002EBC000007A03439DF8080032
:10AD900000EB001202EB002001EBC0019DF8200047
:10ADA00000EB001001EBC00000F50050C0F8393294
:10ADB000ACE08DF8247024E09DF8080000EB400121
:10ADC000C1EBC0109DF8241002EBC0000844C0780D
:10ADD00000F00F00092818D89DF8080000EB40018A
:10ADE000C1EBC0109DF8241002EBC0000844C078ED
:10ADF00000F0F000902808D89DF82400401C8DF841
:10AE000024009DF824000828D6D39DF824000828A3
:10AE1000C5F004839DF8080000EB4001C1EBC010B1
:10AE200002EBC00081799DF8080000EB4003C3EB02
:10AE3000C01002EBC000C07841EA00619DF8080034
:10AE400000EB4003C3EBC01002EBC0000079030429
:10AE50009DF8080000EB400CCCEBC01002EBC000EA
:10AE6000407943EA002001439DF8080000EB0013FD
:10AE700003EB002008EBC0039DF8200000EB00105E
:10AE800002E0D2E0FDE3FDE303EBC00000F500507B
:10AE9000C0F835129DF8080000EB4001C1EBC0106E
:10AEA00002EBC000817A9DF8080000EB4003C3EB81
:10AEB000C01002EBC000C07941EA00619DF80800B3
:10AEC00000EB4003C3EBC01002EBC000007A0304A8
:10AED0009DF8080000EB400CCCEBC01002EBC0006A
:10AEE000407A43EA002001439DF8080000EB00127D
:10AEF00002EB002008EBC0029DF8200000EB0010E0
:10AF000002EBC00000F50050C0F839129DF80800AF
:10AF100000EB001101EB002008EBC0029DF82000BF
:10AF2000414600EB001002EBC00000F5005090F825
:10AF30001C0203289DF8080004F0BB8500EB4002CA
:10AF400002EB00109DF8202001EB001000EB021036
:10AF500000F5805090F8860D800704F1CA859DF8B1
:10AF6000080000EB001202EB002004E04FE00AE1D1
:10AF70001CE032E1F9E301EBC0029DF8200000EB98
:10AF8000001002EBC00000F5005090F82A020128E2
:10AF900004F0B18505F042BA9DF8080000EB0013FB
:10AFA00003EB002008EBC00104F01BBE9DF8081065
:10AFB00001EB011303EB012100EBC1039DF820100D
:10AFC00001EB011103EBC10101F5005181F821B240
:10AFD0009DF8081001EB011202EB012100EBC10109
:10AFE00001F5005181F817629DF8081001EB41024C
:10AFF00002EB011109EB011004F0D2BD9DF808101D
:10B0000001EB011303EB012109EBC101CCE79DF832
:10B01000081001EB011202EB012100EBC10101F567
:10B02000005181F81772C322E8E79DF8081001EB80
:10B03000410303EB011100EB011101F5805191F87F
:10B04000601D00299DF8081001EB4103C3EBC111FD
:10B0500002EBC10152D0C9780B049DF8081001EB36
:10B06000410CCCEBC11102EBC101097943EA012388
:10B070009DF8081001EB410CCCEBC11108EBC101AC
:10B0800049790B439DF8081001EB011202EB0121F5
:10B0900000EBC1029DF8201001EB011102EBC10190
:10B0A00001F50051C1F8503200E0FCE39DF80810B2
:10B0B00001EB011202EB012100EBC1029DF820100F
:10B0C00001EB011102EBC10101F5005191F81C12D5
:10B0D000022932D09DF80810C52201EB011303EBC1
:10B0E000012100EBC1039DF8201001EB011103EBDE
:10B0F000C10101F5005181F82122F2E30B799DF89D
:10B10000081001EB410CCCEBC11108EBC101C9786F
:10B1100043EA01229DF8081001EB011303EB012122
:10B1200000EBC1039DF8201001EB011103EBC101FD
:10B1300001F50051C1F85022B6E79DF8081001EB67
:10B14000011202EB012100EBC10101F5005181F870
:10B1500017729DF80810032201EB011303EB012184
:10B1600000EBC1039DF8201001EB011103EBC101BD
:10B1700001F5005181F81C22D922FAE300F50050B4
:10B1800080F8177206E79DF8081001EB011202EB38
:10B19000012100EBC10101F5005181F817629DF812
:10B1A000081001EB011303EB012100EBC1039DF833
:10B1B000201001EB011103EBC10101F5005181F8F1
:10B1C00021B29DF8081001EB410202EB011109EBDD
:10B1D000011004F0EABD0270DCE69DF80810CE46CE
:10B1E00001EB410303EB011109EB011000F5805065
:10B1F00090F8600D00289DF80C0002D00E28C1D1F7
:10B200009FE00C28BED18DF8247024E09DF8081032
:10B2100001EB4100C0EBC1109DF8241002EBC0000F
:10B220000844C07800F00F00092818D89DF80810CD
:10B2300001EB4100C0EBC1109DF8241002EBC000EF
:10B240000844C07800F0F000902808D89DF8240049
:10B25000401C8DF824009DF824000A28D6D39DF8C0
:10B2600024000A288ED30020CDE90A0038468DF844
:10B2700024701FE0DDE90A31090241EA13611B0273
:10B28000CDE90A319DF8081001EB4103C3EBC11170
:10B290009DF8243002EBC1011944C978DDE90A3C6C
:10B2A000194340EA0C03CDE90A139DF82410491C08
:10B2B0008DF824109DF824100529DBD3DDE90A3C24
:10B2C0009DF8081001EB011808EB01210EEBC109F4
:10B2D0009DF82010F04601EB011109EBC10101F5C9
:10B2E0000059C9F83D324946C1F841C20023CDE9B1
:10B2F0000A338DF824001FE0DDE90A131B0243EA3C
:10B3000011630902CDE90A139DF8081001EB41030E
:10B31000C3EBC1119DF8243002EBC1011944097A35
:10B32000DDE90A3C194340EA0C03CDE90A139DF814
:10B330002410491C8DF824109DF824100529DBD316
:10B340009DE08DF8247024E09DF8081001EB410089
:10B35000C0EBC1109DF8241002EBC0000844C07877
:10B3600000F00F00092818D89DF8081001EB4100E3
:10B37000C0EBC1109DF8241002EBC0000844C07857
:10B3800000F0F000902808D89DF82400401C8DF8AB
:10B3900024009DF824000C28D6D39DF824000C2806
:10B3A000C5F03C800020CDE90A0038468DF82470B5
:10B3B0001FE0DDE90A31090241EA13611B02CDE910
:10B3C0000A319DF8081001EB4103C3EBC1119DF850
:10B3D000243002EBC1011944C978DDE90A3C194364
:10B3E00040EA0C03CDE90A139DF82410491C8DF89E
:10B3F00024109DF824100629DBD3DDE90A3C9DF8D2
:10B40000081001EB011808EB01210EEBC1099DF8B2
:10B410002010F04601EB011109EBC10101F50059C3
:10B42000C9F83D324946C1F841C20023CDE90A338B
:10B430008DF824001FE0DDE90A131B0243EA1163C3
:10B440000902CDE90A139DF8081001EB4103C3EB93
:10B45000C1119DF8243002EBC1011944497ADDE99C
:10B460000A3C194340EA0C03CDE90A139DF8241065
:10B47000491C8DF824109DF824100629DBD3DDE942
:10B480000A129DF8080000EB001303EB002008EB04
:10B49000C0039DF8200000EB001003EBC00000F596
:10B4A0000053C3F845121846C0F849229DF8080019
:10B4B000F04600EB001101EB00200EEBC0029DF8FE
:10B4C000200000EB001002EBC00000F5005090F8E7
:10B4D0001C229DF8080000EB001303EB00200EEB8C
:10B4E000C00000F5005090F8180282427DD194F817
:10B4F000A40780B19DF8080000EB400101EB0011AA
:10B5000008EB01109DF8201000EB01102844017891
:10B5100041F0080199E0C8F839709DF8080000EB87
:10B52000001101EB00219DF8200008EBC10100EBA8
:10B53000001001EBC00042F23D21014410220798A7
:10B54000FCF783FE9DF8080000EB001101EB0021E1
:10B550009DF8200008EBC10100EB001001EBC000DA
:10B5600000F2352000F500504146026841F81D2FD9
:10B57000406848609DF8080000EB400101EB0011B5
:10B5800008EB01109DF8201000EB011000F5805031
:10B5900090F8841D88F81C1004998A6EC8F83D2024
:10B5A000B1F86C10A8F841109DF8080000EB0011EC
:10B5B00001EB00219DF8200008EBC10100EB001019
:10B5C00001EBC00000F50050D0F85012C8F825106B
:10B5D0009DF8080000EB400101EB001108EB0110A1
:10B5E0009DF8201000EB011000E0BFE000F5805056
:10B5F000D0F8881DC8F84310D8F8580081B202204E
:10B60000FDF7A2FA00210620FEF7A8F8D8F8581096
:10B61000B8F81A00814204D2D8F85810491CC8F86A
:10B62000581000210520FEF799F89DF8080000EB5E
:10B63000400101EB001108EB01109DF8201000EB18
:10B6400001102844017821F0080101709DF80810CC
:10B650000220FEF783F89DF820009DF8081000EB0B
:10B660000110C117CDE90A0100EB8001C1EB801187
:10B6700001EB0800C0F87D709DF8081001EB011285
:10B6800001E02FE1ADE102EB01229DF8201008EB73
:10B69000C20201EB011102EBC10142F23D22114451
:10B6A00010226D30FCF7D1FD9DF8080000EB001171
:10B6B00001EB00219DF8200008EBC10100EB001018
:10B6C00001EBC0010A9801F2352100EB8002C2EBC8
:10B6D000801201F5005102EB08000A6840F8612F62
:10B6E000496841609DF8081001EB410202EB01122C
:10B6F00008EB02119DF8202001EB021101F58051A9
:10B7000091F8841D00F8011C04998A6E0262B1F858
:10B710006C1081849DF8081001EB011202EB0122EC
:10B720009DF8201008EBC20201EB011102EBC101F0
:10B7300001F50051D1F8501281609DF8081001EB1D
:10B74000410202EB011208EB02119DF8202001EBEF
:10B75000021101F58051D1F8881DC0F826100A9811
:10B7600081B20820FDF7FAFF11E0BEE09DF8080065
:10B7700000EB400101EB001108EB01109DF82010D7
:10B7800000EB01102844017841F0040101709DF89C
:10B79000080000EB001101EB002008EBC0029DF84F
:10B7A0002000414600EB001002EBC00000F5005005
:10B7B00080F85A729DF8080000EB001303EB00209C
:10B7C00008EBC0039DF8200000EB001003EBC00065
:10B7D00000F5005080F821B29DF8080000EB00123F
:10B7E00002EB002001EBC0029DF8200000EB0010EE
:10B7F00002EBC00000F5005090F81C02042844F051
:10B800000D869DF8080000EB400202EB00109DF849
:10B81000202001EB001000EB02102844027842F0D7
:10B82000800202709DF8080000EB001202EB00207D
:10B8300001EBC00000F5005080F817629DF8080089
:10B84000052200EB001303EB00209DF8203001EBF4
:10B85000C00003EB031300EBC30000F5005080F8B9
:10B860001C229DF8080000EB400202EB00109DF83E
:10B87000202001EB001000EB021000F5805090F842
:10B88000860D800744F1CA859DF8080000EB400250
:10B8900002EB00109DF8202001EB001000EB0210DD
:10B8A0002844027800E064E022F0020303709DF86F
:10B8B000080000EB400202EB00109DF8202001EB95
:10B8C000001000EB02102844027822F020030370DD
:10B8D0009DF8080000EB400202EB001008EB00109E
:10B8E000FEE3FEE35A46FFF789BB84F8E0669DF865
:10B8F000081001EB011202EB012100EBC1029DF8DF
:10B90000201001EB011102EBC10101F5005191F88A
:10B910001C1200299DF8081001EB011202EB012115
:10B920000ED000EBC1029DF8201001EB011102EBDB
:10B93000C10101F5005191F81E12B22928D021E46D
:10B9400000EBC10101F5005181F817729DF8081054
:10B9500001EB011202EB012100EBC1029DF8201066
:10B9600001EB011102EBC10101F5005181F81C62EC
:10B970005A469DF8081001EB011303EB012109EB76
:10B98000C10304F011BD00F5005080F8212223E42A
:10B990009DF8081001EB011202EB012100EBC1013F
:10B9A00001F5005181F817729DF80810B22201EBE1
:10B9B000011303EB012100EBC1039DF8201001EB03
:10B9C000011103EBC10101F5005181F821229DF81D
:10B9D000081001EB011202EB012109EBC10204F096
:10B9E00013BD84F8E0767DE79DF8080000EB400188
:10B9F000C1EBC010FE4911F83000042809D09DF8B1
:10BA0000080000EB4002C2EBC01011F8300015280E
:10BA100001D1ADF818009DF80800F54900EB40028F
:10BA2000C2EBC01001EBC00042789DF8080000EBAB
:10BA30004003C3EBC01011F8300042EA0020A0F52B
:10BA40008051303922D09DF8080000EB4001C1EB55
:10BA5000C010E74901EBC00042789DF8080000EBF8
:10BA60004003C3EBC01011F8300042EA0020A0F5FB
:10BA70008052313A0CD09DF8080000EB4002C2EB36
:10BA8000C01011F83000022804D019E0A62015E0FB
:10BA9000A72013E09DF8080000EB4002C2EBC010A5
:10BAA00001EBC00002799DF8080000EB4003C3EBF6
:10BAB000C01001EBC000C07842EA0020ADF81800C9
:10BAC0009DF80800DFF82C9300EB001101EB00213A
:10BAD00009EBC10101F5005191F816128DF8201003
:10BAE0009DF808109DF8202009EB0111114401F583
:10BAF000805181F8887B99F81800012810D19DF8B1
:10BB0000080000EB400101EB001109EB01109DF86A
:10BB1000201000EB01102844017841F080010170F1
:10BB2000BDF8180043F23002811A904272D009DC4D
:10BB3000042870D015286FD0A6280DD0A72844F06F
:10BB40006D8405E1B1F5C06F67D0A1F5C061013921
:10BB500079D00429F3D1FDE39DF8080000EB001132
:10BB600001EB002009EBC00000F50050494680F8C9
:10BB700017729DF8080000EB001202EB002009EBA1
:10BB8000C0029DF8200000EB001002EBC00000F5A1
:10BB9000005090F81C02032840D09DF8080000EBEC
:10BBA000001202EB002001EBC0029DF8200000EB28
:10BBB000001002EBC00000F5005090F81C020828AD
:10BBC00042D09DF8080000EB001202EB002001EBD0
:10BBD000C0029DF8200000EB001002EBC00000F551
:10BBE000005090F81C020D2843D09DF8080000EB8F
:10BBF000001202EB002001EBC0029DF8200000EBD8
:10BC0000001002EBC00000F5005090F82102A528BA
:10BC100044D054E02BE189E1A0E3CDE39DF8080096
:10BC2000042200EB001303EB002001EBC0039DF89E
:10BC3000200000EB001003EBC00000F5005080F87E
:10BC40001C22A822EEE3F7E39DF80800092200EB8E
:10BC5000001303EB002001EBC0039DF8200000EB74
:10BC6000001003EBC00000F5005080F81C22A92250
:10BC7000D8E39DF808000E2200EB001303EB002030
:10BC800001EBC0039DF8200000EB001003EBC000A7
:10BC900000F5005080F81C22A222C3E39DF80800A2
:10BCA00000EB400202EB00109DF8202001EB001099
:10BCB00000EB02102844027842F0040202709DF862
:10BCC000080000EB001202EB002001EBC0029DF81F
:10BCD000200000EB001002EBC00000F5005090F8CF
:10BCE0001E02A12804F09A839DF8080000EB0012C0
:10BCF00002EB002001EBC0029DF8200000EB0010D9
:10BD000002EBC00000F5005090F81E229DF80800DC
:10BD100000EB001303EB002001EBC0039DF82000B3
:10BD200000EB001003EBC00000F5005080F821226A
:10BD30009DF80800A12200EB001303EB002009EBA3
:10BD4000C0019DF8200000EB001001EBC000FCE3F7
:10BD50009DF8080000EB001101EB002009EBC0008A
:10BD600000F50050494680F817729DF8080000EB76
:10BD7000001202EB002009EBC0029DF8200000EB4E
:10BD8000001002EBC00000F5005090F81C020528DE
:10BD90009DF8080000EB001202EB00200ED001EB32
:10BDA000C0029DF8200000EB001002EBC00000F57F
:10BDB000005090F81C02092808D01FE001EBC000D9
:10BDC00000F5005080F81772062200E00A229DF864
:10BDD000080000EB001303EB002001EBC0039DF80B
:10BDE000200000EB001003EBC00000F5005003E062
:10BDF00080640020A412002080F81C229DF8080016
:10BE000000EB001202EB002001EBC0029DF82000C5
:10BE100000EB001002EBC00000F5005090F821028A
:10BE2000A42822D19DF8080000EB400202EB00108C
:10BE30009DF8202001EB001000EB0210284402784E
:10BE400042F0200202709DF8080000EB001202EBA5
:10BE5000002001EBC0029DF8200000EB001002EB77
:10BE6000C00000F5005080F85972A122DAE28DF886
:10BE7000247012A9FE4A13E09DF8080000EB40036D
:10BE8000C3EBC0109DF8243002EBC0001844C0780A
:10BE90009DF82430C8549DF82400401C8DF82400DF
:10BEA0009DF824000628E7D3062112A810F014F903
:10BEB000CDE91007109B000AC018B84647EB0801EF
:10BEC0004FF480720023FCF77DF99DF8080000EB29
:10BED000001101EB002009EBC0039DF8200000EBEE
:10BEE000001003EBC00000F5005080F820229DF800
:10BEF000080000EB001202EB002009EBC00000F587
:10BF0000005080F817829DF8080000EB001202EB49
:10BF1000002009EBC0029DF8200000EB001002EBAE
:10BF2000C00000F5005080F81C627AE29DF808001D
:10BF300000EB001101EB002109EBC1029DF820107C
:10BF4000484601EB011102EBC10101F5005191F8E6
:10BF50001C12062931D19DF8081001EB011202EBE9
:10BF6000012100EBC10101F5005181F817729DF824
:10BF70000810072201EB011303EB012100EBC103C1
:10BF80009DF8201001EB011103EBC10101F50051F7
:10BF900081F81C229DF80810A72201EB011303EB86
:10BFA000012100EBC1039DF8201001EB011103EB0F
:10BFB000C10101F5005181F821229DF8081001EB23
:10BFC000011202EB012100EBC1029DF8201001EBF0
:10BFD000011102EBC10101F5005191F81C12012978
:10BFE0009DF8081001EB011202EB01215ED000EB7D
:10BFF000C1029DF8201001EB011102EBC10101F516
:10C00000005191F81C1207299DF8081001EB01124C
:10C0100002EB012152D000EBC1029DF8201001EB90
:10C02000011102EBC10101F5005191F81C120B291D
:10C030009DF8081001EB011202EB01215CD000EB2E
:10C04000C1029DF8201001EB011102EBC10101F5C5
:10C05000005191F81C120C299DF8081001EB0112F7
:10C0600002EB012163D000EBC1029DF8201001EB2F
:10C07000011102EBC10101F5005191F81C120E29CA
:10C080005DD09DF8081001EB011202EB012100EBDD
:10C09000C1029DF8201001EB011102EBC10101F575
:10C0A000005191F81C120F297ED048E400EBC10129
:10C0B00001F5005181F81772022206E000EBC10180
:10C0C00001F5005181F8177208229DF8081001EB64
:10C0D000011303EB012100EBC1039DF8201001E0E7
:10C0E000CAE013E101EB011103EBC10101F50051BD
:10C0F00081F81C22A3223CE400EBC10101F50051B0
:10C1000081F817729DF808100C2201EB011303EB64
:10C11000012100EBC1039DF8201001EB011103EB9D
:10C12000C10101F5005181F81C22A12221E400EB9C
:10C13000C10101F5005181F817720D22C5E79DF884
:10C1400008100F2201EB011303EB012100EBC103E7
:10C150009DF8201001EB011103EBC10101F5005125
:10C1600081F81C229DF80810A12201EB011303EBBA
:10C17000012100EBC1039DF8201001EB011103EB3D
:10C18000C10101F5005181F821229DF8081001EB51
:10C19000011303EB012100EBC1039DF8201001EB1B
:10C1A000011103EBC10100E075E001F5005181F8D8
:10C1B0001E229DF8081001EB410202EB011100EB79
:10C1C00001129DF8201002EB011129440A7842F077
:10C1D00080020A709DF8081001EB410202EB011188
:10C1E0009DF8202000EB011101EB021129440A788F
:10C1F00042F004030B709DF8081001EB410202EBC2
:10C2000001119DF8202000EB011101EB021101F555
:10C21000805191F8861D890744F100819DF808102E
:10C2200001EB410202EB01119DF8202000EB01110E
:10C2300001EB021129440A7822F002030B709DF8E9
:10C24000081001EB410202EB01119DF8202000EBE8
:10C25000011101EB021129440A7822F020030B702E
:10C260009DF8081001EB410202EB011102E0000011
:10C270008064002009EB01109DF8201000EB0110F4
:10C280002844017841F0080101709DF8081002204F
:10C29000FDF764FA09E79DF8081001EB011202EBC3
:10C2A000012100EBC1029DF8201001EB011102EB0E
:10C2B000C10101F5005191F81E12A12930D09DF85D
:10C2C0000810A32201EB011303EB01219DF820309C
:10C2D00000EBC10103EB031301EBC30101F50051B6
:10C2E00081F821229DF8081001EB011202EB0121D7
:10C2F00000EBC1029DF8201001EB011102EBC1011E
:10C3000001F5005191F81E12A229C3D09DF8081022
:10C3100001EB011202EB012109EBC100FEF72EBF78
:10C320009DF80810A12201EB011303EB012100EBA2
:10C33000C1039DF8201001EB011103EBC10101F5D0
:10C34000005181F821229DF8081001EB011202EB47
:10C35000012100E0A3E309EBC100F5E39DF808002B
:10C36000A12200EB001101EB002009EBC0039DF8B6
:10C37000200000EB001003EBC00000F5005080F837
:10C380001E229DF8080000EB001303EB002009EBD0
:10C39000C0039DF8200000EB001003EBC00000F587
:10C3A000005080F821229DF8080000EB001202EBFB
:10C3B000002009EBC000B1E79DF8080000EB001178
:10C3C00001EB002009EBC0029DF82000494600EB7C
:10C3D000001002EBC00000F5005090F81C02062887
:10C3E00044F01C809DF8080000EB001202EB0020D6
:10C3F00001EBC00000F5005080F817729DF80800AE
:10C40000072200EB001303EB002001EBC0039DF8B3
:10C41000200000EB001003EBC00000F5005080F896
:10C420001C22A7229DF8080000EB001303EB00205C
:10C4300009EBC00103F0D5BBFFE79DF80800C84633
:10C4400000EB001101EB002009EBC00000F50050EB
:10C4500080F817729DF80800A72100EB001303EB8A
:10C46000002009EBC0029DF8200000EB001002EB59
:10C47000C00000F5005080F821129DF80800DFF898
:10C480007C9D00EB4001C1EBC01109EBC10040797C
:10C4900030289DF8080000EB400147D0C1EBC010E8
:10C4A00009EBC0004946407931289DF808007DD04D
:10C4B00000EB4002C2EBC01001EBC0004079332812
:10C4C0009DF8080073D000EB4002C2EBC01009EBEE
:10C4D000C000407934289DF8080000EB400101EBD2
:10C4E000001065D09DF8201008EB001000EB011043
:10C4F0002844017821F0010101709DF8080000EB4B
:10C50000400101EB00109DF8201008EB001000EB3B
:10C5100001102844017821F0020101700020CDE9CA
:10C520000A0001468DF824704B461AE201EB001018
:10C530009DF82020414608EB001000EB0210284433
:10C54000027822F00102027000E0FDE39DF808008D
:10C5500000EB400202EB00109DF8202008EB0010D9
:10C5600000EB02102844027822F0020303709DF8C9
:10C57000080000EB001202EB002001EBC0039DF865
:10C58000200000EB001003EBC00000F5005090F815
:10C590001F023128C2D19DF8080000EB400202EBD7
:10C5A000001001EB00109DF8202002E01BE03CE1B0
:10C5B00086E100EB02102844027822F0200202708B
:10C5C0009DF8080000EB001202EB002008EBC00110
:10C5D0009DF8200000EB001001EBC00000F50050BA
:10C5E00080F859729AE700EB001101EB002008EB8C
:10C5F000C0029DF82000414600EB001002EBC00095
:10C6000000F5005090F85A0200289DF8080000EB51
:10C61000001202EB00207DD001EBC0029DF820004B
:10C6200000EB001002EBC00000F5005080F85972DA
:10C630009DF8080000EB400202EB00109DF820205E
:10C6400001EB001000EB02102844027822F00102F6
:10C6500002709DF8080000EB400202EB00109DF80C
:10C66000202001EB001000EB02102844027822F099
:10C670000203037094F8A4070028B3D1487E012870
:10C68000B0D1886D4A8B9042ACD29DF8080000EB87
:10C69000001202EB002001EBC0029DF8200000EB2D
:10C6A000001002EBC00000F5005090F8590201287C
:10C6B00098D19DF8080000EB001202EB002001EB7E
:10C6C000C0029DF8200000EB001002EBC00000F556
:10C6D000005090F89302002884D19DF808004FF094
:10C6E000104200EB001303EB002001EBC0039DF8A8
:10C6F000200000EB001003EBC00000F50050C0F874
:10C7000024229DF8080000EB400202EB001001EB30
:10C71000001200E06CE09DF8200002EB001000F534
:10C72000805090F8842D9DF8080000EB001303EB77
:10C73000002001EBC00000F5005080F815229DF8A4
:10C74000080000EB001202EB002001EBC0029DF894
:10C75000200000EB001002EBC00000F5005090F844
:10C760001C229DF8080000EB001303EB002001EBF6
:10C77000C00000F5005090F81802824298D19DF850
:10C78000080000EB001202EB002001EBC0029DF854
:10C79000200000EB001002EBC00000F5005080F814
:10C7A00022729DF80800A42200EB001303EB002086
:10C7B00001EBC0039DF8200000EB001003EBC0006C
:10C7C00000F5005080F81E229DF80800A32200EB1F
:10C7D000001303EB002008EBC0019DF8200000EBE4
:10C7E000001001EBC00000F5005080F8212295E612
:10C7F0009DF8202001EBC00002EB021200EBC2000A
:10C8000000F5005080F859629DF8080000EB4002E6
:10C8100002EB00109DF8202001EB001000EB02104D
:10C820002844027842F0010212E700EB400101EBDC
:10C8300000109DF8201008EB001000EB01102844B8
:10C84000017841F0010101709DF8080000EB400102
:10C8500001EB00109DF8201008EB001000EB011018
:10C8600000F5805090F8860D800715D49DF80800DB
:10C8700000EB400101EB001108EB01109DF82010C6
:10C8800000EB01102844017841F0020101709DF88D
:10C8900008100220FCF762FF9DF80800A22100EBBF
:10C8A000001202EB00229DF8200008EBC20200EB10
:10C8B000001002EBC00000F5005080F81E122DE6BB
:10C8C0009DF8202008EB001000EB021028440278AD
:10C8D00022F0200202709DF8080000EB400202EBFB
:10C8E00000109DF8202008EB001000EB02102844F7
:10C8F000027822F0020202709DF80800A92200EBE3
:10C90000001303EB002008EBC0019DF8200000EBB2
:10C91000001001EBC00000F5005080F81E22FDE57C
:10C920000A98090141EA10710001CDE90A019DF858
:10C93000080000EB4001C1EBC0109DF8241003EB90
:10C94000C00008448079DDE90A2C3038C117104353
:10C9500041EA0C01CDE90A019DF82400401C8DF844
:10C9600024009DF824000628DAD39DF808000A9ACE
:10C9700000EB001101EB00209DF8201008EBC00037
:10C9800001EB011100EBC10000F50050C0F83522A9
:10C990000020CDE90A008DF8247021E0DDE90A01CC
:10C9A000090141EA10710001CDE90A019DF8080072
:10C9B00000EB4001C1EBC0109DF8241003EBC00058
:10C9C0000844407BDDE90A2C3038C117104341EAA6
:10C9D0000C01CDE90A019DF82400401C8DF82400CB
:10C9E0009DF824000428D9D39DF808000A9900EB8B
:10C9F000001202EB002008EBC0029DF8200000EBC3
:10CA0000001002EBC00000F50050C0F850120022E8
:10CA1000CDE90A2211468DF8247020E00A98090118
:10CA200041EA10710001CDE90A019DF8080000EB10
:10CA30004001C1EBC0109DF8241003EBC000084476
:10CA4000407CDDE90A2C3038C117104341EA0C0163
:10CA5000CDE90A019DF82400401C8DF824009DF8C2
:10CA600024000628DAD39DF808000A9900EB00128A
:10CA700002EB002008EBC0029DF8200000EB001044
:10CA800002EBC00000F50050C0F839129DF8080014
:10CA900000EB4001C1EBC01003EBC000FDE39DF8CB
:10CAA000080000EB001101EB002009EBC00000F5CD
:10CAB000005080F817729DF8080000EB001202EB9E
:10CAC000002009EBC0019DF8200000EB001001EBF5
:10CAD000C00000F5005090F81C020A2835D09DF8DF
:10CAE000080000EB001101EB002009EBC0029DF8EB
:10CAF0002000494600EB001002EBC00000F500509A
:10CB000090F81C229DF8080000EB001303EB0020B6
:10CB100009EBC00000F5005090F81802824227D1BE
:10CB200094F8A40728B39DF808009DF8201000EBA6
:10CB3000400202EB001009EB001000EB011028444A
:10CB4000017841F008019BE0FEE39DF808000B210D
:10CB500000EB001202EB00229DF8200009EBC2025C
:10CB600000EB001002EBC00000F5005080F81C1232
:10CB70008CE0C846C1F839709DF8080000EB001140
:10CB800001EB00219DF8200009EBC10100EB001032
:10CB900001EBC00042F23D21014410220798FBF74F
:10CBA00054FB9DF8080000EB001101EB00219DF8FB
:10CBB000200008EBC10100EB001001EBC00000F207
:10CBC000352000F500504146026841F81D2F4068AD
:10CBD00048609DF8080000EB400101EB001108EBF4
:10CBE00001109DF8201000EB011000F5805090F826
:10CBF000841D88F81C109DF8080000EB001101EB63
:10CC000000219DF8200008EBC10100EB001001EBB2
:10CC1000C00000F50050D0F85012C8F82510049953
:10CC200040468A6E40F83D2FB1F86C108180D8F8EC
:10CC3000580081B20220FBF787FF00210620FCF795
:10CC40008DFDD8F85810B8F81A00814204D2D8F8EF
:10CC50005810491CC8F8581000210520FCF77EFD2B
:10CC60009DF8080000EB400101EB001108EB0110FA
:10CC70009DF8201000EB01102844017821F00801F4
:10CC800001709DF808100220FCF768FD9DF808006F
:10CC9000A72100EB001202EB002009EBC0029DF877
:10CCA0002000CC4600EB001002EBC00000F5005065
:10CCB00080F821129DF80800A22100EB001202EB7F
:10CCC000002009EBC0029DF8200000EB001002EBF1
:10CCD000C00000F5005080F81E129DF8080000EB1F
:10CCE000001101EB00200CEBC0019DF8200000EBCF
:10CCF000001001EBC00000F5005080F85A720021CE
:10CD0000CDE90A118DF82470DFF8F08422E0DDE926
:10CD10000A10000140EA11700901CDE90A109DF8DE
:10CD2000080000EB4001C1EBC0109DF8241008EB97
:10CD3000C0000844C07ADDE90A233038C117104327
:10CD40001943CDE90A0100E00BE29DF82400401CE4
:10CD50008DF824009DF824000A28D8D3DDE90A12B2
:10CD60009DF8080000EB001303EB00200CEBC00360
:10CD70009DF8200000EB001003EBC00000F500530D
:10CD8000C3F83D121846C0F841220021CDE90A112E
:10CD90008DF8247020E0DDE90A01090141EA1071F3
:10CDA0000001CDE90A019DF8080000EB4001C1EB4C
:10CDB000C0109DF8241008EBC0000844407DDDE958
:10CDC0000A233038C11710431943CDE90A019DF8F1
:10CDD0002400401C8DF824009DF824000A28DAD392
:10CDE000DDE90A129DF8080000EB001303EB0020B8
:10CDF0000CEBC003FEE39DF8080000EB4001C1EB23
:10CE0000C010FE4911F83000042809D09DF8080030
:10CE100000EB4002C2EBC01011F83000152801D120
:10CE2000ADF818009DF80800894600EB4002C2EBFF
:10CE3000C01001EBC00042789DF8080000EB4003F1
:10CE4000C3EBC01011F8300042EA0020A0F5805179
:10CE5000303922D09DF8080000EB4001C1EBC01032
:10CE600009EBC000494642789DF8080000EB4003FA
:10CE7000C3EBC01019F8300042EA0020A0F5805240
:10CE8000313A0CD09DF8080000EB4002C2EBC01014
:10CE900011F83000022804D019E0A62015E0A720E0
:10CEA00013E09DF8080000EB4002C2EBC01001EB5C
:10CEB000C00002799DF8080000EB4003C3EBC010EE
:10CEC00009EBC000C07842EA0020ADF818009DF8D8
:10CED000080000EB001101EB0021C94800EBC10183
:10CEE00001F5005191F816228DF820209DF80810C8
:10CEF00000EB01129DF82010114401F5805181F8DA
:10CF0000887B017E012910D19DF8081001EB4102B8
:10CF100002EB01119DF8202000EB011101EB021141
:10CF200029440A7842F080020A70BDF81810A72937
:10CF30007DD007DC04297BD015297AD0A62943F0BF
:10CF40006D823DE001F51D61B1F5804104D01129EC
:10CF500070D01229F3D1FDE39DF8081001EB011206
:10CF600002EB012100EBC1029DF8201001EB011141
:10CF700002EBC10101F5005191F81C120029DED12C
:10CF80009DF8081001EB011202EB012100EBC10139
:10CF900001F5005181F817729DF8081001EB01129C
:10CFA00002EB012100EBC1029DF8201001EB011101
:10CFB00002EBC10101F5005181F81C62A7229EE13C
:10CFC0009DF8081001EB011202EB012100EBC101F9
:10CFD00001F5005181F817729DF8081001EB01125C
:10CFE00002EB012100EBC1029DF8201001EB0111C1
:10CFF00002EBC10101F5005191F81C1202292DD05C
:10D000009DF8081001EB011202EB012100EBC102B7
:10D010009DF8201001EB011102EBC10101F5005157
:10D0200091F81C1205292ED09DF8081003E09EE00F
:10D03000F0E065E28AE201EB011202EB012100EB74
:10D04000C1029DF8201001EB011102EBC10101F5B5
:10D05000005191F82112A5292AD03AE09DF8081034
:10D06000032201EB011303EB012100EBC1039DF847
:10D07000201001EB011103EBC10101F5005181F812
:10D080001C22A9223BE19DF80810062201EB0113A6
:10D0900003EB012100EBC1039DF8201001EB01110E
:10D0A00003EBC10101F5005181F81C22A22226E107
:10D0B0009DF8081001EB410202EB01119DF82020C0
:10D0C00000EB011101EB021129440A7842F004023D
:10D0D0000A709DF8081001EB011202EB012100EB30
:10D0E000C1029DF8201001EB011102EBC10101F515
:10D0F000005191F81E12A12903F090819DF80810AB
:10D1000001EB011202EB012100EBC1029DF820109E
:10D1100001EB011102EBC10101F5005191F81E2252
:10D120009DF8081001EB011303EB012100EBC10393
:10D130009DF8201001EB011103EBC10101F5005135
:10D1400081F821229DF80810A12201EB011303EBC5
:10D15000012100EBC1039DF8200000EB001003EB60
:10D16000C00000F5005080F81E2203F057B99DF86A
:10D17000081001EB011202EB012100EBC1029DF846
:10D18000201001EB011102EBC10101F5005191F8F2
:10D190002112A42922D19DF8081001EB410202EBD3
:10D1A00001119DF8202000EB011101EB021129442F
:10D1B0000A7842F020020A709DF8081001EB011273
:10D1C00002EB012100EBC1029DF8201001EB0111DF
:10D1D00002EBC10101F5005181F859729DF8081068
:10D1E00001EB011202EB012100EBC10101F500513D
:10D1F00081F81772A1229DF8081003E080640020D6
:10D20000A412002001EB011303EB012100EBC1018B
:10D2100002F0E7BC9DF8081001EB011202EB0121BE
:10D2200000EBC1029DF8201001EB011102EBC101DE
:10D2300001F5005191F81C1201299DF8081001EB2D
:10D24000011202EB012138D000EBC1029DF8201041
:10D2500001EB011102EBC10101F5005191F81C1223
:10D2600004299DF8081001EB011202EB01212CD0DA
:10D2700000EBC1029DF8201001EB011102EBC1018E
:10D2800001F5005191F81C1206299DF8081001EBD8
:10D29000011202EB01213CD000E0FCE300EBC102F3
:10D2A0009DF8201001EB011102EBC10101F50051C5
:10D2B00091F81C1207297DD057E700EBC10101F559
:10D2C000005181F81772022206E000EBC10101F55E
:10D2D000005181F8177205229DF8081001EB011327
:10D2E00003EB012100EBC1039DF8201001EB0111BC
:10D2F00003EBC10101F5005181F81C22A3229DF826
:10D30000081001EB011303EB012100EBC10303F053
:10D310004BB800EBC10101F5005181F817729DF87F
:10D320000810072201EB011303EB012100EBC103FD
:10D330009DF8201001EB011103EBC10101F5005133
:10D3400081F81C22A12200E0D5E09DF8081001EB35
:10D35000011303EB012100EBC1039DF8201001EB49
:10D36000011103EBC10101F5005181F821229DF863
:10D37000081001EB410202EB011100EB01129DF8D4
:10D38000201002EB011129440A7842F080020A7051
:10D390009DF8081001EB410202EB011100EB0112B4
:10D3A0009DF8201002EB01114A19117841F0040395
:10D3B000137000E03EE09DF8081001EB410202EB23
:10D3C000011100EB01129DF8201002EB011101F593
:10D3D000805191F8861D890743F120809DF808103F
:10D3E00001EB410202EB01119DF8202000EB01113D
:10D3F00001EB021129440A7822F002030B709DF818
:10D40000081001EB410202EB01119DF8202000EB16
:10D41000011101EB021129440A7822F020030B705C
:10D420009DF8081001EB410202EB011100EB011025
:10D43000FEF722BF9DF8081001EB011202EB01215B
:10D4400000EBC1029DF8201001EB011102EBC101BC
:10D4500001F5005191F81E12A12931D09DF8081054
:10D46000A32201EB011303EB01219DF8203000EB17
:10D47000C10103EB031301EBC30101F5005181F876
:10D4800021229DF8081001EB011202EB012100EBB3
:10D49000C1029DF8201001EB011102EBC10101F561
:10D4A000005191F81E12A22902F0B8879DF80810C9
:10D4B00001EB011202EB012100EBC100FDF75EBEA2
:10D4C0009DF80810A12201EB011303EB012100EBF1
:10D4D000C1039DF8201001EB011103EBC10101F51F
:10D4E000005181F821229DF8081001EB011202EB96
:10D4F000012100EBC10000F5005080F8176234E60E
:10D500009DF80810A12201EB011303EB012100EBB0
:10D51000C1039DF8201001EB011103EBC10101F5DE
:10D52000005181F821229DF8081001EB011303EB53
:10D53000012100EBC1039DF8201001EB011103EB69
:10D54000C10101F5005181F81E22AFE79DF80810D6
:10D55000804601EB011202EB012200EBC20000F554
:10D56000005080F817729DF80800A72200EB001306
:10D5700003EB002008EBC0019DF8200000EB001039
:10D5800001EBC00000F5005080F821229DF8080052
:10D5900000EB4001C1EBC01109EBC100407930281C
:10D5A0009DF8080000EB400154D0C1EBC01009EB1E
:10D5B000C0004946407931289DF808007ED000EB34
:10D5C0004002C2EBC01001EBC000407933289DF847
:10D5D000080074D000EB4002C2EBC01001EBC000A9
:10D5E000407934289DF808006AD000EB4002C2EB75
:10D5F000C01000E0FEE309EBC0004079352871D08F
:10D600009DF8080000EB400101EB00109DF8201090
:10D6100008EB001000EB01102844017821F0010113
:10D6200001709DF8080000EB400101EB00109DF82F
:10D63000201008EB001000EB01102844017821F0C5
:10D64000020101700020CDE90A0001468DF8247026
:10D65000CC460EE201EB00109DF82020414608EB7D
:10D66000001000EB02102844027822F00102027040
:10D670009DF8080000EB400202EB00109DF820200E
:10D6800008EB001000EB02102844027822F002039D
:10D6900003709DF8080000EB001202EB002001EB84
:10D6A000C0039DF8200000EB001003EBC00000F564
:10D6B000005090F81F023128C4D102E013E037E196
:10D6C0006FE19DF808009DF8201000EB400202EB8E
:10D6D000001008EB001000EB01102844017821F045
:10D6E0002001AEE791E100EB001101EB002008EB17
:10D6F000C0029DF82000414600EB001002EBC00084
:10D7000000F5005090F85A0200289DF8080000EB40
:10D71000001202EB00207CD001EBC0039DF820003A
:10D7200000EB001003EBC00000F5005080F85972C8
:10D730009DF8080000EB400202EB00109DF820204D
:10D7400001EB001000EB02102844027822F00103E4
:10D75000037000E060E29DF8080000EB400202EB7D
:10D7600000109DF8202001EB001000EB021028446F
:10D77000027822F00203037094F8A40700289BD1DA
:10D78000487E012898D1886D4A8B9042BFF45AAFE9
:10D790009DF8080000EB001202EB002001EBC00234
:10D7A0009DF8200000EB001002EBC00000F50050D7
:10D7B00090F859020128E2D19DF8080000EB001210
:10D7C00002EB002001EBC0029DF8200000EB0010EE
:10D7D00002EBC00000F5005090F893020028CED173
:10D7E0009DF808004FF0104200EB001303EB0020FF
:10D7F00001EBC0039DF8200000EB001003EBC0001C
:10D8000000F50050C0F824229DF8080000EB40020B
:10D8100000E070E002EB001001EB00129DF8200028
:10D8200002EB001000F5805090F8842D9DF8080060
:10D8300000EB001303EB002001EBC00000F50050EB
:10D8400080F815229DF8080000EB001202EB002082
:10D8500001EBC0029DF8200000EB001002EBC000BD
:10D8600000F5005090F81C229DF8080000EB001312
:10D8700003EB002001EBC00000F5005090F8180207
:10D88000824298D19DF8080000EB001202EB0020C4
:10D8900001EBC0029DF8200000EB001002EBC0007D
:10D8A00000F5005080F822729DF80800A42200EBD9
:10D8B000001303EB002001EBC0039DF8200000EBF8
:10D8C000001003EBC00000F5005080F81E229DF808
:10D8D0000800A32200EB001303EB002008EBC001BB
:10D8E0009DF8200000EB001001EBC00000F5005097
:10D8F00080F82122A6E69DF8202001EBC00002EB73
:10D90000021200EBC20000F5005080F859629DF849
:10D91000080000EB400202EB00109DF8202001EB14
:10D92000001000EB02102844027842F001030FE7D8
:10D9300000EB400101EB00109DF8201008EB0010F7
:10D9400000EB01102844017841F0010101709DF8BD
:10D95000080000EB400101EB00109DF8201008EBDF
:10D96000001000EB011000F5805090F8860D800744
:10D9700015D49DF8080000EB400101EB001108EB05
:10D9800001109DF8201000EB01102844017841F0AF
:10D99000020202709DF808100220FBF7DFFEA221B0
:10D9A00034E000EB400101EB00109DF8202008EB73
:10D9B000001000EB02102844027822F020020270CE
:10D9C0009DF8080000EB400202EB00109DF82020BB
:10D9D00008EB001000EB02102844027822F002024B
:10D9E00002709DF80800A92200EB001303EB002051
:10D9F00008EBC0019DF8200000EB001001EBC00017
:10DA000000F5005080F81E221CE6A1219DF80800B8
:10DA100000EB001202EB00229DF8200008EBC2028E
:10DA200000EB001002EBC00000F5005080F81E1261
:10DA300008E60A98090141EA10710001CDE90A01DE
:10DA40009DF8080000EB4001C1EBC0109DF82410C8
:10DA50000CEBC00008448079DDE90A233038C11797
:10DA600010431943CDE90A019DF82400401C8DF8AC
:10DA700024009DF824000828DBD39DF808000A99AB
:10DA800000EB001202EB002008EBC0029DF8200022
:10DA900000EB001000E089E002EBC00000F5005050
:10DAA000C0F835120021CDE90A118DF8247020E06C
:10DAB000DDE90A01090141EA10710001CDE90A011D
:10DAC0009DF8080000EB4001C1EBC0109DF8241048
:10DAD0000CEBC0000844C07BDDE90A233038C117D5
:10DAE00010431943CDE90A019DF82400401C8DF82C
:10DAF00024009DF824000628DAD39DF808000A992E
:10DB000000EB001202EB002008EBC0029DF82000A1
:10DB100000EB001002EBC00000F50050C0F85012FE
:10DB20000021CDE90A118DF8247020E0DDE90A0119
:10DB3000090141EA10710001CDE90A019DF80800D0
:10DB400000EB4001C1EBC0109DF824100CEBC000AD
:10DB50000844407DDDE90A233038C11710431943DA
:10DB6000CDE90A019DF82400401C8DF824009DF8A1
:10DB700024000828DAD39DF808000A9900EB001267
:10DB800002EB002008EBC0029DF8200000EB001023
:10DB900002EBC00000F50050C0F839129DF80800F3
:10DBA00000EB4001C1EBC0100CEBC00041799DF8C7
:10DBB000080000EB001202EB002008EBC0029DF809
:10DBC000200000EB001002EBC00000F5005080F8D0
:10DBD0001F129DF8080000EB400101EB001008EB5C
:10DBE00000119DF8200001EB001000F5805090F826
:10DBF000861D9DF8080000EB001202EB002008EBE8
:10DC0000C0029DF8200000EB001002EBC00000F500
:10DC1000005080F8341272E49DF80810804601EB41
:10DC2000011202EB012200EBC20000F5005080F867
:10DC300017729DF8080000EB001202EB002008EBC1
:10DC4000C0019DF8200000EB001001EBC00000F5C2
:10DC5000005090F81C02032834D09DF8080000EB17
:10DC6000001101EB002008EBC0029DF820004146A6
:10DC700000EB001002EBC00000F5005090F81C22F1
:10DC80009DF8080000EB001303EB002008EBC00038
:10DC900000F5005090F81802824226D194F8A407AB
:10DCA00020B39DF808009DF8201000EB400202EB25
:10DCB000001008EB001000EB01102844017841F03F
:10DCC00008019BE09DF80800042100EB001202EB24
:10DCD00000229DF8200008EBC20200EB001002EBCE
:10DCE000C00000F5005080F81C128DE0C1F83970BA
:10DCF0009DF8080000EB001101EB00219DF82000C9
:10DD000008EBC10100EB001001EBC00042F23D2125
:10DD1000014410220798FAF798FA9DF8080000EBE2
:10DD2000001101EB00219DF8200008EBC10100EB80
:10DD3000001001EBC00000F2352000F50050414614
:10DD4000026841F81D2F406848609DF8080000EB0C
:10DD5000400101EB001108EB01109DF8201000EBD1
:10DD6000011000F5805090F8841D88F81C109DF873
:10DD7000080000EB001101EB00219DF8200008EBEA
:10DD8000C10100EB001001EBC00000F50050D0F81D
:10DD90005012C8F82510049940468A6E40F83D2F6D
:10DDA000B1F86C108180D8F8580081B20220FAF7DF
:10DDB000CBFE00210620FBF7D1FCD8F85810B8F8AC
:10DDC0001A00814204D2D8F85810491CC8F85810DB
:10DDD00000210520FBF7C2FC9DF8080000EB400184
:10DDE00001EB001108EB01109DF8201000EB011071
:10DDF000284400E0B8E0017821F0080101709DF8A6
:10DE000008100220FBF7AAFC9DF8080000EB0011A7
:10DE100001EB002008EBC0019DF8200000EB001092
:10DE200001EBC00000F5005080F85A729DF8080020
:10DE3000A72100EB001202EB002008EBC0029DF8C6
:10DE4000200000EB001002EBC00000F5005080F84D
:10DE500021129DF80800A22100EB001202EB002025
:10DE600008EBC0029DF8200000EB001002EBC000A0
:10DE700000F5005080F81E120021CDE90A118DF83E
:10DE80002470CC4620E0DDE90A10000140EA117060
:10DE90000901CDE90A109DF8080000EB4001C1EB33
:10DEA000C0109DF824100CEBC0000844C07ADDE9D6
:10DEB0000A233038C11710431943CDE90A019DF8F0
:10DEC0002400401C8DF824009DF824000C28DAD38F
:10DED000DDE90A019DF8082002EB021303EB0222A0
:10DEE00008EBC2039DF8202002EB021203EBC202F2
:10DEF00002F50053C3F83D021A46C2F84112002051
:10DF0000CDE90A0001468DF824701FE00A98090146
:10DF100041EA10710001CDE90A019DF8080000EB0B
:10DF20004001C1EBC0109DF824100CEBC000084468
:10DF3000C07DDDE90A233038C11710431943CDE90C
:10DF40000A019DF82400401C8DF824009DF824004F
:10DF50000C28DBD3DDE90A129DF8080000EB001362
:10DF600003EB002008EBC0039DF8200000EB00103D
:10DF700003EBC00000F50053C3F845121846C0F883
:10DF8000492248E6FE4B9DF808009DF8201003EB5F
:10DF90000010084400F5805080F8887B9DF8080048
:10DFA000DFF8E08300EB4001C1EBC01008EBC000DC
:10DFB000407870280AD19DF8080000EB4001C1EBC1
:10DFC000C01008EBC0008078FA282DD09DF808001A
:10DFD00000EB4001C1EBC01008EBC00040789DF899
:10DFE000080000EB4001C1EBC01018F830009DF8AC
:10DFF000080000EB001101EB002003EBC00000F56E
:10E00000005090F816028DF820009DF808009DF849
:10E01000201003EB0010084400F5805080F8887B46
:10E02000187E012804D014E0B120ADF81800DEE716
:10E030009DF8080000EB400101EB00109DF8201056
:10E0400003EB001000EB01102844017841F080013F
:10E050000170BDF8180001284BD065287DD0B1288B
:10E060008FD0B6288DD19DF8080000EB001101EB90
:10E07000002003EBC0019DF8200000EB001001EB35
:10E08000C00000F5005090F81C020128EAD19DF86C
:10E09000080000EB001101EB002003EBC00000F5CD
:10E0A000005080F817729DF8080000EB001101EB9A
:10E0B000002003EBC0019DF8200000EB001001EBF5
:10E0C000C00000F5005080F81C629DF80800B121E6
:10E0D00000EB001202EB002003EBC0029DF82000D1
:10E0E00000EB001002EBC00000F5005080F8211298
:10E0F00091E59DF8080000EB4001C1EBC01008EB72
:10E10000C00000790128F3D00228F1D00328EFD015
:10E110000528EDD19DF8080000EB001101EB00206F
:10E1200003EBC0019DF8200000EB001001EBC000E4
:10E1300000F5005090F81C020028D9D19DF8080085
:10E1400000EB001101EB002003EBC00000F50050D4
:10E1500080F817729DF8080000E036E000EB00112F
:10E1600001EB002003EBC0019DF8200000EB001044
:10E1700001EBC00000F5005080F81C629DF808001B
:10E18000B62100EB001202EB002003EBC0029DF869
:10E19000200000EB001002EBC00000F5005080F8FA
:10E1A00021129DF80800B22100EB001202EB0020C2
:10E1B00003EBC0029DF8200000EB001002EBC00052
:10E1C00000F5005080F81E1225E59DF8080000EBD0
:10E1D0004001C1EBC01008EBC0000079B922ADF8D6
:10E1E00018209DF8080000EB4001C1EBC01008EBBF
:10E1F000C000007900F00F018DF814108DF8247024
:10E200001FE09DF8080000EB400101EB001003EB5C
:10E2100000119DF8240001EB001000F5805090F8EB
:10E22000851D9DF8080000EB400CCCEBC01018F8E1
:10E2300030005038814214D09DF82400401C8DF8E5
:10E2400024009DF8080000EB400101EB001003EBF7
:10E25000001000F5805090F85B0D9DF82410884266
:10E26000CFD89DF824009DF8141008448DF82000A4
:10E270009DF8080000EB001101EB002003EBC00C3F
:10E280009DF8200000EB00100CEBC00000F50050E2
:10E2900090F81C02012813D09DF8080000EB001133
:10E2A00001EB002003EBC0019DF8200000EB001003
:10E2B00001EBC00000F5005090F81C0201287DD150
:10E2C0009DF8080000EB001101EB002003EBC000FB
:10E2D00000F5005080F817729DF80800022100EB4D
:10E2E000001C0CEB002003EBC00C9DF8200000EBA1
:10E2F00000100CEBC00000F5005080F81C129DF8D7
:10E30000080000EB001101EB002003EBC001F8E373
:10E310009DF8080000EB400101EB0011184800EBEC
:10E32000011000F5805090F8600D20B1012873D0E5
:10E330000228C4D19BE2DFF848909DF8081009EB51
:10E34000410000F58040B0F83404801F81B29DF890
:10E350000800DFF8308000EB4002C2EBC01208EB8F
:10E36000C200401CFAF77AFFCDE910079DF80810AB
:10E3700009EB410000F58040B0F83414414403E05B
:10E38000A4120020806400209DF8080000EB4002E9
:10E39000C2EBC0106FF0040202EBC000084404217D
:10E3A00009F062FFC117CDE90A01DDE9103201462B
:10E3B0000B98594050400143BBD100E001E39DF868
:10E3C000080009EB001000F5805080F8887B9DF86C
:10E3D000080000EB4002C2EBC012404600EBC20056
:10E3E0000079ADF81800BDF818003128A1D19DF8CA
:10E3F000081009EB410000F58040B0F834044121D9
:10E40000183890FBF1F0C117CDE90A0184F88405B2
:10E410008DF82470B846CCE0D5E09DF8080000EBFC
:10E420004001C1EBC011FE4800EBC1019DF8240082
:10E4300000EB80100844017D9DF8242009EB0200C8
:10E4400000F5805080F885159DF8080000EB40012C
:10E45000C1EBC011F24800EBC1019DF8240000EBB4
:10E460008010084408211A3009F0CAFE8DED010A17
:10E4700010EE100A9DF8242009EB021101F58051DD
:10E48000C1F895059DF8080000EB4001C1EBC011F3
:10E49000E34800EBC1019DF8240000EB8010084424
:10E4A0000821323009F0ACFE8DED010A10EE100AA1
:10E4B0009DF8242009EB021101F58051C1F8910566
:10E4C0009DF8080000EB4001C1EBC011D44800EBFF
:10E4D000C1019DF8240000EB8010084408213A3067
:10E4E00009F08EFE8DED010A10EE100A9DF8242031
:10E4F00009EB021101F58051C1F899059DF808005A
:10E5000000EB4001C1EBC011C54800EBC1019DF813
:10E51000240000EB801008440821423009F070FE0E
:10E520008DED010A10EE100A9DF8242009EB02116E
:10E5300001F58051C1F89D059DF8080000EB4001F0
:10E5400001EB001109EB01109DF8241000EB011004
:10E550002844017841F0800101709DF8081009EB12
:10E56000410000F58040B0F83414AD4801449DF8F6
:10E57000080000EB4002C2EBC0104FF0FF3202EB8C
:10E58000C000095C9DF8080000EB001202EB0022BD
:10E590009DF8200009EBC20300EB001003EBC00064
:10E5A00000F5005080F858129DF82400401C8DF8AA
:10E5B00024009DF82400DDE90A12401A78EB0200DD
:10E5C000FFF62BAFDDE49DF80800DFF8548200EB86
:10E5D0004001C1EBC01008EBC000437D9DF808006E
:10E5E00000EB4002C2EBC01008EBC000807D43EAA4
:10E5F0000020C317CDE90A039DF80800152100EBA0
:10E600004002C2EBC01008EBC000FAF711FECDE9E2
:10E610001007DDE90A01109B794058400843D1D129
:10E620009DF8080000EB4001C1EBC011404618F80E
:10E630003120521E8DF82020DFF8E8919DF8081057
:10E640004A4609EB01139DF82010194401F5805149
:10E6500081F8887B9DF82010494401F5805181F8AC
:10E6600085759DF8201009EB011101F58051C1F865
:10E6700095759DF8081001EB4103C3EBC11100EB48
:10E68000C1018B799DF8081001EB410CCCEBC11155
:10E6900000EBC101497943EA012100EE101AF8EEBE
:10E6A000400A9FED610A9DF8081080EE801A01EB88
:10E6B0004103C3EBC11100EBC1010B799DF80810B8
:10E6C00001EB410CCCEBC11100EBC101C97843EA6D
:10E6D000012100EE901A9DF82010F8EE600A71EE0C
:10E6E000200A10EE903A02EB011101F58051C1F8B9
:10E6F00091359DF8081001EB4103C3EBC11100EB0C
:10E70000C1018B7A9DF8081001EB410CCCEBC111D3
:10E7100000EBC101497A43EA012100EE901A9DF80D
:10E720000810B8EE601AC1EE000A01EB4103C3EB1A
:10E73000C11100EBC1010B7A9DF8081001EB410CEF
:10E74000CCEBC11100EBC101C97943EA012100EE14
:10E75000101A9DF82010B8EE400A30EE800A10EE34
:10E76000103A02EB011101F58051C1F899359DF87D
:10E77000081001EB4102C2EBC11100EBC100C07AED
:10E7800000069DF8080000EB4001C1EBC01008EB4B
:10E79000C000027B9DF8080000EB4003C3EBC010F3
:10E7A00008EBC000C07A42EA00200AD400EE100A4A
:10E7B000DFED1E0AB8EE400A20EE200A10EE100A25
:10E7C0000BE0404280B2F9F70DFF9FED191B53ECAF
:10E7D000112BF9F715FEF9F76AFF9DF8202009EBD8
:10E7E000021101F58051C1F89D059DF808009DF8C2
:10E7F000202000EB400101EB001009EB001000EBC2
:10E8000002102844027842F0800202709DF808004D
:10E8100000EB4002C2EBC01208EBC200C27D0BE06D
:10E8200080640020A412002000FF7F470000803D8C
:10E83000000000000000B0BF9DF8080000EB0013CE
:10E8400003EB002009EBC0039DF8200000EB001053
:10E8500003EBC00000F5005080F858229DF8080036
:10E8600000EB400202EB001009EB0010D0E09DF835
:10E870000800DFF8809400EB4001C1EBC01009EB09
:10E88000C000C3799DF8080000EB4002C2EBC01045
:10E8900009EBC000007A43EA0020C317CDE90A0360
:10E8A0009DF80800072100EB4002C2EBC01009EB05
:10E8B000C000FAF7BDFCCDE91007DDE90A01109BA5
:10E8C0007940584008437CD19DF8080000EB400196
:10E8D000C1EBC01119F83100401E8DF82000DFF89F
:10E8E00018849DF8081008EB011000F5805080F89E
:10E8F000887B9DF8201008EB010000F5805080F81F
:10E9000085759DF8080000EB4001C1EBC01109EBD3
:10E91000C1008079F9F766FE41EC110B9FEDF70B12
:10E920000CF07EFA9DF80800B0EE408AF0EE608AA6
:10E9300000EB4001C1EBC01109EBC10002799DF869
:10E94000080000EB4001C1EBC01109EBC100C07829
:10E9500042EA0020F9F746FE53EC182BF9F7C2FD06
:10E96000F9F7A5FE9DF8201008EB011101F5805183
:10E97000C1F895059DF8201008EB011000F58050B6
:10E98000C0F891759DF8201008EB011000F580503B
:10E99000C0F899759DF8201008EB011000F5805023
:10E9A000C0F89D759DF8080000EB400101EB0011D7
:10E9B00008EB01109DF8201000EB011028440178AD
:10E9C00000E093E241F0800202709DF8080000EB45
:10E9D0004001C1EBC01109EBC100427A9DF808006B
:10E9E00000EB001101EB00219DF8200008EBC103B2
:10E9F00000EB001003EBC00000F5005080F8582237
:10EA00009DF8080000EB400101EB001108EB01103C
:10EA100000F5805090F85B0D84F88405D2E59DF8F0
:10EA20000800DFF8D08200EB4001C1EBC01008EB1A
:10EA3000C0004146C3789DF8080000EB4002C2EBDD
:10EA4000C01008EBC000807843EA00208DF80C006D
:10EA50009DF8080000EB4002C2EBC0109DF80C20AE
:10EA600008EBC000104443789DF8080000EB40021A
:10EA7000C2EBC0109DF80C2001EBC000805C43EAA3
:10EA80000020C317CDE90A039DF808009DF80C107B
:10EA900000EB4002C2EBC01008EBC000FAF7C8FB65
:10EAA000CDE91007DDE90A10109B78405940014379
:10EAB000B4D19DF8080000EB4001C1EBC01008EB99
:10EAC000C00040788DF820008DF824708A491CE041
:10EAD0009DF8080000EB400202EB00109DF8242096
:10EAE00001EB001000EB021000F5805090F8850D4E
:10EAF0009DF8202090429DF8240003D18DF820003D
:10EB000013E0FDE3401C8DF824009DF8080000EBA5
:10EB1000400202EB001001EB001000F5805090F86D
:10EB20005B0D9DF824209042D2D89DF8080000EBA0
:10EB3000400202EB001001EB00129DF8200002EBF6
:10EB400000102844027842F0800202709DF808000C
:10EB500000EB4002C2EBC01008EBC0000079ADF83A
:10EB600018009DF808009DF8202001EB00101044CB
:10EB700000F5805080F8887BBDF81800F32806D097
:10EB800006DC05287DD0F12807D0F22890D155E287
:10EB9000F42877D0F6288BD152E29DF8080000EBDC
:10EBA000001202EB002001EBC0029DF8200000EBF8
:10EBB000001002EBC00000F5005090F81C02002885
:10EBC0009DF8080025D000EB400202EB00109DF8F4
:10EBD000202001EB001000EB021000F5805090F8AF
:10EBE0008D0DC00714D09DF808008C4600EB001274
:10EBF00002EB002001EBC0029DF8200000EB0010AA
:10EC000002EBC00000F5005090F8A202C00724D02B
:10EC1000C0E000EB001202EB002001EBC0029DF807
:10EC2000200000EB001002EBC00000F5005080F85F
:10EC30001C629DF80800F42200EB001303EB002097
:10EC400001EBC0039DF8200000EB001003EBC000B7
:10EC500000F5005080F821229CE09DF8080000EBB0
:10EC6000001202EB00200CEBC0029DF8200000EB2C
:10EC7000001002EBC00000F5005090F89402C0B301
:10EC800001E058E2F0E18DF824702AE09DF80800D8
:10EC900000EB001202EB00209DF820200CEBC000DE
:10ECA00002EB021200EBC2009DF82420104400F594
:10ECB000005090F895229DF8080000EB400303EB0C
:10ECC00000109DF824300CEB0010184400F5805023
:10ECD00090F8620D824208D19DF82400401C8DF806
:10ECE00024009DF824000428D0D39DF82400042893
:10ECF00031D04FE080640020A4120020000000000A
:10ED0000000024409DF8080000EB001202EB0020F8
:10ED10000CEBC0029DF8200000EB001002EBC000DD
:10ED20009DF82420104400F5005090F895029DF8BD
:10ED3000082002EB420303EB02129DF824300CEB97
:10ED400002121A4402F5805292F8622D904208D1C4
:10ED50009DF82400401C8DF824009DF824000A280A
:10ED6000D0D39DF824000A2814D09DF8080000EBA9
:10ED7000001202EB002001EBC0029DF8200000EB26
:10ED8000001002EBC00242F2A2201044027842F0CE
:10ED9000010202709DF80C00112844D09DF80C006F
:10EDA00014289DF8080000EB400202EB00107CD014
:10EDB0009DF8202001EB001000EB0210284402789F
:10EDC00022F0040303709DF8080000EB001202EB30
:10EDD000002001EBC0039DF8200000EB001003EBC6
:10EDE000C00000F5005090F8A202C0077ED09DF848
:10EDF000080000EB001202EB002001EBC0029DF8BE
:10EE0000200000EB001002EBC00000F50050A0F85D
:10EE1000A07205229DF8080000EB001303EB002010
:10EE200001EBC0016CE29DF8080000EB400202EB30
:10EE3000001001EB00129DF8200002EB00104219B7
:10EE4000107840F0040313708DF82470424625E0DA
:10EE50009DF8080000EB4003C3EBC01002EBC003B9
:10EE60009DF82400184443799DF8080000EB001C2D
:10EE70000CEB002001EBC00C9DF8200000EB001013
:10EE80000CEBC00C9DF82400604400F5005080F8A5
:10EE90005B329DF824305B1C8DF824309DF82400F3
:10EEA0000A28D5D38DF8247028E02CE09DF80800BE
:10EEB00000EB4003C3EBC0109DF8243002EBC00010
:10EEC0001844C37B9DF8080000EB001C0CEB0020ED
:10EED00001EBC00C9DF8200000EB00100CEBC00013
:10EEE0009DF824C0604400F5005000E08EE280F8F8
:10EEF00074329DF82400401C8DF824009DF82400F5
:10EF00000228D3D382E201EB00129DF8200002EB2D
:10EF100000104219107840F0040313708DF824702B
:10EF2000424625E09DF8080000EB4003C3EBC0100B
:10EF300002EBC0039DF82400184443799DF80800B3
:10EF400000EB001C0CEB002001EBC00C9DF8200036
:10EF500000EB00100CEBC00C9DF82400604400F5A1
:10EF6000005080F85B329DF824305B1C8DF8243013
:10EF70009DF824000A28D5D38DF824701FE09DF851
:10EF8000243002EBC0001844C37B9DF8080000EB5E
:10EF9000001C0CEB002001EBC00C9DF8200000EBE6
:10EFA00000100CEBC0009DF824C0604400F5005038
:10EFB00080F874329DF82400401C8DF824009DF8E0
:10EFC000240002289DF8080000EB4003C3EBC010AA
:10EFD000D5D302EBC0039DF824001844407C030401
:10EFE0009DF8080000EB400CCCEBC01002EBC00C0D
:10EFF0009DF824006044807C43EA00239DF80800CB
:10F0000000EB400CCCEBC01008EBC0029DF82400D4
:10F010001044C07C03439DF8080000EB001202EB93
:10F02000002001EBC0019DF8200000EB001001EB77
:10F03000C00000F50050C0F88832E7E1F122E9E6AF
:10F040009DF80800032200EB001303EB002001EB06
:10F05000C0039DF8200000EB001003EBC00000F59A
:10F06000005080F81C22E9E79DF80800022200EB1E
:10F07000001303EB002001EBC0039DF8200000EB20
:10F08000001003EBC00000F5005080F81C229DF832
:10F090000800F62200EB001303EB002001EBC00395
:10F0A0009DF8200000EB001003EBC00000F50050BD
:10F0B00080F821229DF8080000EB001202EB0020EE
:10F0C00001EBC0029DF8200000EB001002EBC00035
:10F0D00000F5005080F894628DF82470424625E0D7
:10F0E0009DF8080000EB4003C3EBC0109DF82430EE
:10F0F00002EBC000184443799DF8080000EB001CA7
:10F100000CEB002001EBC00C9DF8200000EB001080
:10F110000CEBC0009DF824C0604400F5005080F85E
:10F1200095329DF82400401C8DF824009DF82400A1
:10F130000A28D5D36AE19DF8080000EB4002C2EB33
:10F14000C01008EBC00083799DF8080000EB400C6C
:10F15000CCEBC01008EBC000407943EA00229DF8D8
:10F16000080000EB001303EB002001EBC0039DF847
:10F17000200000EB001003EBC00000F50050A0F8E9
:10F18000A0229DF8080000EB001202EB002001EB2A
:10F19000C0029DF8200000EB001002EBC00000F55B
:10F1A0000050B0F8A0229DF8080000EB400303EBEC
:10F1B000001001EB001000F58050B0F86E0D824297
:10F1C000B8D39DF80800F12200EB001303EB0020F8
:10F1D00001EBC00C9DF8200000EB00100CEBC00010
:10F1E00000F5005080F821229DF8080000EB001285
:10F1F00002EB002001EBC0019DF8200000EB0010A5
:10F2000001EBC00042F2A2210844017821F0010183
:10F210000170FBE09DF8080000EB4001C1EBC0105D
:10F22000FE4A02EBC00000798DF820008DF80070D6
:10F23000DFF8EC831BE09DF808009DF8001000EB60
:10F24000400303EB001008EB001000EB011000F589
:10F25000805090F8850D9DF8201088429DF80000A0
:10F2600002D18DF8200012E0401C8DF800009DF8BE
:10F27000080000EB400101EB001008EB001000F566
:10F28000805090F85B0D9DF800309842D3D89DF8DF
:10F29000080000EB4001C1EBC01002EBC000C078D9
:10F2A000ADF81800BDF81800182812D2DFE800F0F9
:10F2B000110C0E11797971797311111175797979B0
:10F2C00079771111791179791A2000E00D208DF8E4
:10F2D0000C009DF80C00001FC1B29DF8080091467B
:10F2E00000EB4003C3EBC01302EBC300C01CF9F7F3
:10F2F000CDFD8DF804009DF8080000EB400100E012
:10F30000F6E3C1EBC01109EBC1009DF80C100844F5
:10F3100010F8010C9DF80410884277D19DF8080080
:10F320004A4600EB4001C1EBC01009EBC000407839
:10F3300000286BD09DF8080000EB4001C1EBC01025
:10F340009DF80C1002EBC0000844C3789DF808003B
:10F3500000EB001101EB002108EBC10C9DF820101F
:10F36000404601EB01110CEBC10101F5005181F8A0
:10F3700058329DF8081008EB01139DF8201019442D
:10F3800001F5805181F8887B98F8181001290AD07E
:10F390001AE007209BE7082099E70C2097E70A204E
:10F3A00095E7062093E79DF8081001EB410303EB76
:10F3B00001119DF8203000EB011101EB03112944EC
:10F3C0000B7843F080030B70BDF81810CE2912D0D3
:10F3D00012DCB9297ED008DC5A29AAD0B2297AD009
:10F3E000B52977D0B62998D1FEE3C32974D0C529B1
:10F3F00073D0CA2991D1DDE3E1296FD007DCD5298B
:10F400000AD0D72995D0D92987D1DDE237E3E5297C
:10F4100065D0E729E7D1E8E39DF8081001EB410347
:10F42000C3EBC11109EBC101C97884F8E2119DF861
:10F43000081001EB410202EB0112014600EB021041
:10F440009DF8202000EB021094F8E2212844A6EB5E
:10F45000D213027863F3000202709DF8080000EBFB
:10F46000400202EB00109DF8202001EB001000EBA1
:10F47000021094F8E22128445309027863F3410210
:10F4800002709DF8080000EB400202EB001001EB57
:10F4900000129DF8200002EB001000F5805090F85B
:10F4A000860DC0F340029DF8080000EB001303EB4B
:10F4B000002008EBC0019DF8200000EB001001EBDC
:10F4C000C00000F5005090F83402C0F340008242C2
:10F4D00057D005E070E3FCE33CE3FBE36AE3FAE3C7
:10F4E0009DF8080000EB001101EB002008EBC002C2
:10F4F0009DF82000414600EB001002EBC00042F2F4
:10F50000342210449DF8082002EB420303EB021260
:10F510009DF8203008EB021202EB031202F5805234
:10F5200092F8862D5308027863F3410202709DF829
:10F53000080000EB400202EB00109DF8202001EBD8
:10F54000001000EB021000F5805090F8860D800747
:10F5500018D59DF80800D92200EB001303EB00201A
:10F5600008EBC0019DF8200000EB001001EBC0008B
:10F5700000F5005080F821229DF808100220FAF7CB
:10F58000EDF847E09DF8080000EB001202EB0020C8
:10F5900001EBC0029DF8200000EB001002EBC00060
:10F5A00000F5005080F829629DF80800D92200EB90
:10F5B000001303EB002001EBC0039DF8200000EBDB
:10F5C000001003EBC00000F5005080F821229DF8E8
:10F5D000080000EB400202EB001001EB00129DF866
:10F5E000200002EB00104219107820F02003137065
:10F5F0009DF8080000EB001202EB002008EBC001B0
:10F600009DF8200000EB001001EBC00000F5005059
:10F6100080F85A629DF8080004E000008064002031
:10F62000A412002000EB400101EB001008EB0011D8
:10F630009DF82000434601EB001000F5805090F843
:10F64000860D00F001019DF8080000EB001202EBAE
:10F65000002008EBC0029DF8200000EB001002EB38
:10F66000C00000F5005090F8340200F00100814223
:10F6700071D09DF808009DF8202000EB001101EBEF
:10F680000020194603EBC00002EB021200EBC2009F
:10F6900042F2342210449DF8082002EB420303EBAF
:10F6A00002129DF8203001EB021202EB031202F568
:10F6B000805292F8862D037862F3000303709DF860
:10F6C000080000EB400202EB00109DF8202001EB47
:10F6D000001000EB021000F5805090F8860DC00776
:10F6E0009DF8080038D000EB001202EB002001EB7F
:10F6F000C0029DF8200000EB001002EBC00000F5F6
:10F70000005090F85A0200289DF8080000EB001203
:10F7100002EB002001EBC0029DF8200000EB00107E
:10F7200002EBC00000F5005038D080F859729DF807
:10F73000080000EB400202EB001001EB00129DF804
:10F74000200002EB00104219107820F00103137022
:10F7500094F8A40728B3DBE000EB400202EB0010B2
:10F760009DF8202001EB001000EB021028440278E5
:10F7700022F0200303709DF8080000EB001202EB5A
:10F78000002001EBC0019DF8200000EB001001EB10
:10F79000C00000F5005080F85972B9E080F8596255
:10F7A000D6E7487E012868D1886D4A8B904264D2A2
:10F7B0009DF8080000EB001202EB002001EBC002F4
:10F7C0009DF8200000EB001002EBC00000F5005097
:10F7D00090F85902012850D19DF8080000EB001262
:10F7E00002EB002001EBC0029DF8200000EB0010AE
:10F7F00002EBC00000F5005090F89302E8BB9DF8C2
:10F80000080000EB400202EB001001EB00129DF833
:10F81000200002EB001000F5805090F8842D9DF838
:10F82000080000EB001303EB002001EBC00000F523
:10F83000005080F815229DF80800C32200EB001349
:10F8400003EB002001EBC0039DF8200000EB00104B
:10F8500003EBC00000F5005080F821229DF808005D
:10F8600000EB400202EB001008EB00119DF82000B5
:10F8700001EB001000F5805000E049E0C0F8887D01
:10F880009DF808100220F9F769FF8DF824704146B1
:10F8900019E09DF8080000EB001202EB002001EBDC
:10F8A000C0029DF8200000EB001002EBC0009DF8A4
:10F8B0002420104400F5005080F85B729DF824006D
:10F8C000401C8DF824009DF824001428E1D38DF805
:10F8D000247019E09DF8080000EB001202EB0020F4
:10F8E00001EBC0029DF8200000EB001002EBC0000D
:10F8F0009DF82420104400F5005080F877729DF8A0
:10F900002400401C8DF824009DF824000A28E1D32F
:10F910009DF808009DF8202000EB400101EB00104D
:10F92000414608EB001000EB021000F5805090F803
:10F93000860D800712D59DF80800D92200EB001330
:10F9400003EB002001EBC0039DF8200000EB00104A
:10F9500003EBC00000F5005080F821229DF808005C
:10F9600000EB001202EB002001EBC0029DF820002A
:10F9700000EB001002EBC00000F5005090F81C02F4
:10F9800001287CD19DF8080000EB001202EB00205A
:10F9900001EBC00000F5005080F817729DF80800D8
:10F9A000022200EB001303EB002001EBC0039DF8E3
:10F9B000200000EB001003EBC00000F5005080F8C1
:10F9C0001C22B622FBF7E8BA9DF8081001EB4103B0
:10F9D00003EB011108EB011000F5805090F8600D69
:10F9E00000289DF80C0002D00A28CAD130E008286F
:10F9F000C7D18DF8247025E09DF8080000EB400188
:10FA0000C1EBC0109DF8241002EBC0000844C07880
:10FA100000F00F0009283BF663A99DF8080000EBF1
:10FA20004001C1EBC0109DF8241002EBC000084457
:10FA3000C07800F0F0009028EDD89DF82400401C1C
:10FA40008DF824009DF824000628D5D3FBF748B98B
:10FA50008DF8247027E09DF8080000EB4001C1EB11
:10FA6000C0109DF8241002EBC0000844C07800F0DC
:10FA70000F0009283BF6C9A99DF8080000E02CE218
:10FA800000EB4001C1EBC0109DF8241002EBC00058
:10FA90000844C07800F0F0009028EBD89DF82400CE
:10FAA000401C8DF824009DF824000828D3D3FBF7D0
:10FAB000ACB900EB001202EB002001EBC00000F536
:10FAC000005080F817729DF80800042200EB001324
:10FAD00003EB002001EBC0039DF8200000EB0010B9
:10FAE00003EBC00000F5005080F81C22C52269E736
:10FAF00077E05A4666E79DF8080000EB001202EB3B
:10FB0000002001EBC0029DF8200000EB001002EB8A
:10FB1000C00000F5005080F82A729DF80800B62257
:10FB200000EB001303EB002001EBC0039DF8200065
:10FB300000EB001003EBC00000F5005080F821221C
:10FB40009DF8080000EB001202EB002008EBC0005B
:10FB5000FBF714BB9DF8081001EB011303EB012127
:10FB600000EBC1039DF8201001EB011103EBC10173
:10FB700001F5005181F821B29DF8081001EB011246
:10FB800002EB012100EBC10101F5005181F8176280
:10FB90009DF8081001EB410202EB011108EB011086
:10FBA0009DF8201000EB01102844017841F020025C
:10FBB000FBF711BB5A460CE09DF8081001EB01124F
:10FBC00002EB012100EBC10101F5005181F8177230
:10FBD000C3229DF8081001EB011303EB012108EB90
:10FBE000C1019DF8200001E006E0FCE300EB0010FD
:10FBF00001EBC000FBF7C7BE9DF8081001EB410305
:10FC000003EB011100EB011101F5805191F8601D2A
:10FC100000299DF8081001EB4103C3EBC11102EB71
:10FC2000C1015CD0C9780B049DF8081001EB410CB0
:10FC3000CCEBC11102EBC101097943EA01239DF824
:10FC4000081001EB410CCCEBC11109EBC101497962
:10FC50000B439DF8081001EB011202EB012100EBB0
:10FC6000C1029DF8201001EB011102EBC10101F569
:10FC70000051C1F850329DF8081001EB011202EB5F
:10FC8000012100EBC1029DF8201001EB011102EBF4
:10FC9000C10101F5005191F81C1202293ED09DF8D6
:10FCA0000810C52201EB011303EB012100EBC10396
:10FCB0009DF8201001EB011103EBC10101F500518A
:10FCC00081F821229DF8081001EB011202EB0121BD
:10FCD00002E044E072E01BE308EBC10038E70B7977
:10FCE0009DF8081001EB410CCCEBC11109EBC101EF
:10FCF000C97843EA01229DF8081001EB011303EBD8
:10FD0000012100EBC1039DF8201001EB011103EB71
:10FD1000C10101F50051C1F85022ACE79DF808106F
:10FD200001EB011202EB012100EBC10101F50051D1
:10FD300081F817729DF80810032201EB011303EB01
:10FD4000012100EBC1039DF8201001EB011103EB31
:10FD5000C10101F5005181F81C22D9221CE39DF854
:10FD6000081001EB011202EB012100EBC10101F5CA
:10FD7000005181F817629DF8081001EB011303EBA5
:10FD8000012100EBC1039DF8201001EB011103EBF1
:10FD9000C10101F5005181F821B29DF8081001EB75
:10FDA000410202EB011108EB01109DF8201000EB5D
:10FDB00001102844017841F00402F9E69DF808108A
:10FDC000C64601EB410303EB011108EB011000F5FE
:10FDD000805090F8600D00289DF80C0002D00E288D
:10FDE0007BD1A0E00C2878D18DF8247024E09DF818
:10FDF000081001EB4100C0EBC1109DF8241002EB8C
:10FE0000C0000844C07800F00F00092818D89DF8F9
:10FE1000081001EB4100C0EBC1109DF8241002EB6B
:10FE2000C0000844C07800F0F000902808D89DF881
:10FE30002400401C8DF824009DF824000A28D6D305
:10FE40009DF824000A2848D30020CDE90A0038464E
:10FE50008DF824701FE0DDE90A31090241EA1361DF
:10FE60001B02CDE90A319DF8081001EB4103C3EBF9
:10FE7000C1119DF8243002EBC1011944C978DDE9B4
:10FE80000A3C194340EA0C03CDE90A139DF82410FB
:10FE9000491C8DF824109DF824100529DBD3DDE9D9
:10FEA0000A3C9DF8081001EB011808EB01210EEB4C
:10FEB000C1099DF82010F04601EB011109EBC101C9
:10FEC00001F50059C9F83D324946C1F841C2002345
:10FED000CDE90A338DF8240020E0D2E0DDE90A13F1
:10FEE0001B0243EA11630902CDE90A139DF80810C9
:10FEF00001EB4103C3EBC1119DF8243002EBC101BA
:10FF00001944097ADDE90A3C194340EA0C03CDE9BA
:10FF10000A139DF82410491C8DF824109DF8241014
:10FF20000529DBD39CE08DF8247024E09DF80810AF
:10FF300001EB4100C0EBC1109DF8241002EBC000A2
:10FF40000844C07800F00F00092818D89DF8081060
:10FF500001EB4100C0EBC1109DF8241002EBC00082
:10FF60000844C07800F0F000902808D89DF82400DC
:10FF7000401C8DF824009DF824000C28D6D39DF851
:10FF800024000C287DD30020CDE90A0038468DF8E6
:10FF900024701FE0DDE90A131B0243EA1163090222
:10FFA000CDE90A139DF8081001EB4103C3EBC11121
:10FFB0009DF8243002EBC1011944C978DDE90A3CFF
:10FFC000194340EA0C03CDE90A139DF82410491C9B
:10FFD0008DF824109DF824100629DBD3DDE90A3CB6
:10FFE0009DF8081001EB011808EB01210EEBC10987
:10FFF0009DF82010F04601EB011109EBC10101F55C
:020000040801F1
:100000000059C9F83D324946C1F841C20023CDE943
:100010000A338DF824001FE0DDE90A131B0243EACE
:1000200011630902CDE90A139DF8081001EB4103A1
:10003000C3EBC1119DF8243002EBC1011944497A88
:10004000DDE90A3C194340EA0C03CDE90A139DF8A7
:100050002410491C8DF824109DF824100629DBD3A8
:10006000DDE90A129DF8080000EB001303EB002005
:1000700008EBC0039DF8200000EB001003EBC0006C
:1000800000E044E100F50053C3F845121846C0F8FB
:1000900049229DF80800F04600EB001101EB00201A
:1000A0000EEBC0029DF8200000EB001002EBC00038
:1000B00000F5005090F81C229DF8080000EB00139A
:1000C00003EB00200EEBC00000F5005090F8180282
:1000D00082427DD194F8A40780B19DF8080000EB1E
:1000E000400101EB001108EB01109DF8201000EB1E
:1000F00001102844017841F0080187E0C8F8397000
:100100009DF8080000EB001101EB00219DF8200094
:1001100008EBC10100EB001001EBC00042F23D21F1
:10012000014410220798F8F790F89DF8080000EBBA
:10013000001101EB00219DF8200008EBC10100EB4C
:10014000001001EBC00000F2352000F500504146E0
:10015000026841F81D2F406848609DF8080000EBD8
:10016000400101EB001108EB01109DF8201000EB9D
:10017000011000F5805090F8841D88F81C109DF83F
:10018000080000EB001101EB00219DF8200008EBB6
:10019000C10100EB001001EBC00000F50050D0F8E9
:1001A0005012C8F82510049940468A6E40F83D2F39
:1001B000B1F86C108180D8F8580081B20220F8F7AD
:1001C000C3FC00210620F9F7C9FAD8F8581000E05E
:1001D00023E0B8F81A00814204D2D8F85810491C1C
:1001E000C8F8581000210520F9F7B8FA9DF8080062
:1001F00000EB400101EB001108EB01109DF820100D
:1002000000EB01102844017821F0080101709DF8ED
:1002100008100220F9F7A2FA10E09DF8080000EBA0
:10022000400101EB001108EB01109DF8201000EBDC
:1002300001102844017841F0040101709DF8080084
:1002400000EB001101EB002008EBC0029DF820003C
:10025000414600EB001002EBC00000F5005080F8B2
:100260005A729DF8080000EB001303EB002008EB26
:10027000C0039DF8200000EB001003EBC00000F568
:10028000005080F821B29DF8080000EB001202EB4C
:10029000002001EBC0029DF8200000EB001002EBF3
:1002A000C00000F5005090F81C0204282FD19DF8E2
:1002B000080000EB400202EB00109DF8202001EB4B
:1002C000001000EB02102844027842F08002027015
:1002D0009DF8080000EB001202EB002001EBC000CB
:1002E00000F5005080F817629DF80800052200EB29
:1002F000001303EB002008EBC0019DF8200000EB89
:10030000001001EBC00000F5005080F81C2285E0D1
:1003100084F8E0669DF8081001EB011202EB012160
:1003200000EBC1029DF8201001EB011102EBC101AD
:1003300001F5005191F81C1200299DF8081001EBFD
:10034000011202EB01210ED000EBC1029DF820103A
:1003500001EB011102EBC10101F5005191F81E12F0
:10036000B22928D05AE000EBC10101F5005181F813
:1003700017729DF8081001EB011202EB012100EB4E
:10038000C1029DF8201001EB011102EBC10101F542
:10039000005181F81C625A469DF8081001EB0113C8
:1003A00003EB012108EBC1039DF8200000EB0010D6
:1003B00003EBC0001EE49DF8081001EB011202EBF4
:1003C000012100EBC10101F5005181F817729DF880
:1003D0000810B22201EB011303EB012100EBC10372
:1003E0009DF8201000E037E001EB011103EBC101A3
:1003F00001F5005181F821229DF8081001EB01124E
:1004000002EB012108EBC1029DF8200000EB001077
:1004100002EBC00000F5005080F81E7294F8E7036C
:10042000B0B121489DF8081000EB410000F5804074
:10043000B0F834149DF80800012300EB4002C2EB31
:10044000C0121A4800EBC2009DF80820F9F7DEFD43
:100450008DF82470154913E084F8E076FFF7AABB05
:100460009DF8080000EB4002C2EBC0109DF824206C
:1004700001EBC00087549DF82400401C8DF8240037
:100480009DF824001428EBD30948017842781144E0
:1004900082781144C278D14279F479AF1FB0BDECB3
:1004A000028BBDE8F08F0000A412002080640020C1
:1004B000120000202DE9F74F8EB00020ADF80000AB
:1004C000ADF80400ADF80400ADF804008DF810009C
:1004D0008DF814008DF81800CDE90800CDE908006A
:1004E000ADF83400F8A1D1E90023F9A1CDE9022348
:1004F000D1E90023F849CDE90A2308710E98F74A9B
:1005000000EB400101EB001002EB001000F5805100
:100510008A4691F85A1D8DF810100E9902EB0113BE
:100520000F990793194401F58051894691F8883B4A
:100530000E994FF0310E01EB011404EB012114462A
:1005400004EBC10C0F99042B01EB01110CEBC1075B
:100550000F9907F5005500EB011101F5805B1FD1E4
:10056000052389F8883B002185F81C129BF8861D1D
:1005700021F080038BF8863D9AF85A3DA121072B84
:100580000ED2DFE803F00D040B0B06080A00E5218C
:1005900004E0B12102E0714600E0F12185F821126A
:1005A000117E01297BD09DF810800E99109B01EBE4
:1005B000011404EB0121C94CC94E04EBC10101F542
:1005C000005101910E99A13BC1EB011101EB810496
:1005D000B8F1080F7BD2DFE818F07A000800470274
:1005E000AD0342051E06940661089BF8850D4FF089
:1005F0000008414601F0A4FF8DF8140095F81C1284
:10060000019890F81802814203D10198012180F8E5
:10061000171299F8880B401C89F8880B1098CE287F
:100620007ED010DCB9287CD006DCB2287AD0B52880
:1006300036D0B6284BD1EEE3C32874D0C52873D08A
:10064000CA28F7D1E8E3E1286FD06FDCD52807D0BE
:10065000D7286CD0D928EDD10EE0E728EAD1FAE30B
:10066000F52006F834009DF8140006EBC405687008
:10067000A220A870D5200AE0F52006F834009DF8E5
:10068000140006EBC4056870A220A870D920E87099
:100690002846032101F085FE2871052053E2FDE381
:1006A000F52006F834009DF8140006EBC4077870B6
:1006B0009AF8600D0028D5F8240209D0B0F1104F47
:1006C00038D34FF010400021CDE9080136E059E25F
:1006D000B0F5100F05D34FF410000021CDE908014B
:1006E00003E0D5F82412CDE90818A520B8704046DB
:1006F0000FE0BDF80000C0F10200C200DDE9080112
:10070000F7F791FDBDF800103944C870BDF800003E
:10071000401CADF80000BDF800000328E9D307E055
:1007200009E127E088E0EEE3EEE3DBE0EDE3EDE373
:10073000B520C0E0D5F82412CDE90818A620B8707D
:1007400040460FE0BDF80000C0F10300C200DDE943
:100750000801F7F768FDBDF800103944C870BDF80E
:100760000000401CADF80000BDF800000428E9D3EB
:10077000B520D9E0F52006F834009DF8140006EB0A
:10078000C40778709AF8600D0028D5F824020AD0C2
:10079000B0F1104F30D0D5F82402CDE90808A620DA
:1007A000B87040463EE0B0F5100F07D0D5F82412DF
:1007B000CDE90818A520B870404615E04FF41000A8
:1007C0000021CDE90801F5E7BDF80000C0F1020005
:1007D000C200DDE90801F7F726FDBDF80010394435
:1007E000C870BDF80000401CADF80000BDF8000066
:1007F0000328E9D3B9205EE04FF010400021CDE995
:100800000801CCE7BDF80000C0F10300C200DDE93B
:100810000801F7F708FDBDF800103944C870BDF8AD
:100820000000401CADF80000BDF800000428E9D32A
:10083000B92079E0092031E7F52006F834009DF869
:10084000140006EBC40778709AF8600D18B1A52063
:10085000B870404628E0A420B87040460EE0D5F8B5
:100860005002BDF80010C1F10101C900C840BDF837
:1008700000103944C870BDF80000401CADF80000FD
:10088000BDF800000228EAD3FEE3D5F85002BDF817
:100890000010C1F10201C900C840BDF80010394480
:1008A000C870BDF80000401CADF80000BDF80000A5
:1008B0000328EAD3B220B8713846062101F071FD51
:1008C000F8710820EAE6000001693230313030006A
:1008D000016932304530300012000020A41200209F
:1008E000205B0020F52006F834009DF8140006EB8C
:1008F000C4077870A620B87040460EE0D5F85402C0
:10090000BDF80010C1F10301C900C840BDF80010D6
:100910003944C870BDF80000401CADF80000BDF8B7
:1009200000000428EAD3E120F8713846072101F0DD
:1009300038FD38727EE7F52006F834009DF8140083
:1009400006EBC40568709AF8600D18B1AE20A87067
:1009500040465CE0AC20A870404615E007F500502A
:10096000D0F83D0207F50051D1F84112BDF8002042
:10097000C2F10402D200F7F756FCBDF8001029447A
:10098000C870BDF80000401CADF80000BDF80000C4
:100990000528E3D3404615E007F50050D0F845029E
:1009A00007F50051D1F84912BDF80020C2F1040248
:1009B000D200F7F738FCBDF8001029440872BDF8E2
:1009C0000000401CADF80000BDF800000528E3D38E
:1009D000CE20687328460D2101F0E3FCA8730F2098
:1009E000B1E007F50050D0F83D0207F50051D1F80D
:1009F0004112BDF80020C2F10502D200F7F713FC46
:100A0000BDF800102944C870BDF80000401CADF8C6
:100A10000000BDF800000628E3D3404615E007F5C6
:100A20000050D0F8450207F50051D1F84912BDF841
:100A30000020C2F10502D200F7F7F5FBBDF8001067
:100A400029444872BDF80000401CADF80000BDF814
:100A500000000628E3D3CE20E87328460F2101F0DA
:100A6000A0FC287411206EE09BF8850D8DF8140011
:100A700095F81C12019890F81802814203D1019850
:100A8000012180F8171299F8880B401C89F8880B0F
:100A90009DF8140020B19DF81400401E8DF814003C
:100AA0000A2B6FD2DFE803F043F7588FF8F5F4050F
:100AB000F36F022006F834009DF8140006EBC4071B
:100AC000403078704120B8703020F870387195F857
:100AD00020020009787178790A28787901D23030BB
:100AE00000E03730787195F8200200F00F00B871FF
:100AF000B8790A28B87901D2303000E03730B871BF
:100B00000320F871781C0721F8F7C0F93872092022
:100B1000ADF8340095F81C02042802D1052085F8B0
:100B20001C020198002180F81712062028E00422F8
:100B300006F834209DF8141006EBC40040314170D3
:100B4000512145E1072035E2287103206871681CB6
:100B50000521F8F79BF9E9E3042206F834209DF813
:100B6000141006EBC4004031417041218170052111
:100B7000C170ADF8342095F81C02022802D1032080
:100B800085F81C0229E1022006F834009DF81400C3
:100B900006EBC405403068704120A87085F803E07A
:100BA0003220287103206871681C0521F8F76EF95E
:100BB000A8710720ADF834009BF8860D20F02001C5
:100BC0008BF8861D09E1022006F834009DF8140018
:100BD00006EBC407403078704120B870704687F843
:100BE00003E030213971D5F82422B2F5100F00D27C
:100BF0003221797195F82212012903D095F8220249
:100C000028B100E0B8710021ADF8001015E03220E5
:100C1000F8E7D5F82402BDF80020C2F105029200E1
:100C2000D040BDF8002000F00F003A443030D071C1
:100C3000BDF80000401CADF80000BDF8000006281B
:100C4000E7D332207873ADF8001013E0D5F85002E6
:100C5000BDF80010C1F103018900C840BDF80010C3
:100C600000F00F00394430308873BDF80000401C9C
:100C7000ADF80000BDF800000428E7D30320B874E5
:100C8000781C1221F8F702F9F874142092E186E03A
:100C900062E162E100E073E0022006F834009DF8B2
:100CA000140006EBC407403078704120B870322041
:100CB000F87087F804E07871B8710021ADF8001081
:100CC00013E0D5F85002BDF80020C2F103029200F3
:100CD000D040BDF8002000F00F003A443030D07111
:100CE000BDF80000401CADF80000BDF8000004286D
:100CF000E7D3ADF80010302108E0BDF8000038441B
:100D0000C172BDF80000401CADF80000BDF8000045
:100D10001928F2D3032087F82400781C2421F8F73F
:100D2000B5F887F82500262044E106EBC401487099
:100D300002203FE19BF8850D8DF8140095F81C12F8
:100D4000019890F81802814203D10198012180F89E
:100D5000171299F8880B401C89F8880B9DF814002D
:100D600020B19DF81400401E8DF814000A2B34D2D7
:100D7000DFE803F005062453F4F3F2331534D6E626
:100D8000022006F834009DF8140006EBC40540303C
:100D900068704120A87085F803E03520D4E6022071
:100DA00006F834009DF8140006EBC4054030687066
:100DB0004120A8703220E8703020C5E6042206F8F1
:100DC00034209DF8141006EBC400403141704121DD
:100DD00081700521C170ADF834201BE2022006F8B5
:100DE00034009DF8140006EBC405403068704120C3
:100DF000A87085F803E03220287103206871681C10
:100E00000521F8F743F8A8719BF8860D20F0200122
:100E10008BF8861D96E6FDE3FDE3022006F834001C
:100E20009DF8140006EBC407403078704120B8707C
:100E3000714687F803E03871D5F82402B0F1104FFD
:100E40000AD03220787195F82202012806D095F850
:100E5000220228B106E0FAE33020F3E7B97101E09D
:100E60003220B8710022ADF8002013E0D5F824023A
:100E7000BDF80010C1F107018900C840BDF800109D
:100E800000F00F0039443030C871BDF80000401C3C
:100E9000ADF80000BDF80000082800E0FDE3E5D350
:100EA0003220F873ADF8002013E0D5F85002BDF8F9
:100EB0000010C1F105018900C840BDF8001000F024
:100EC0000F00394430300874BDF80000401CADF804
:100ED0000000BDF800000628E7D33021B975ADF851
:100EE000002008E0BDF800003844C175BDF80000DE
:100EF000401CADF80000BDF800000628F2D3797759
:100F0000ADF800200CE0F0E3F0E3F0E3F0E3BDF82F
:100F1000000038448177BDF80000401CADF80000A7
:100F2000BDF800000628F2D387F82410ADF80020A1
:100F300009E0BDF80000384480F82510BDF8000035
:100F4000401CADF80000BDF800000628F1D387F87A
:100F50002B10ADF800200CE07CE076E02BE0BDF833
:100F60000000384480F82C10BDF80000401CADF89B
:100F70000000BDF800000628F1D387F83210ADF864
:100F8000002009E0BDF80000384480F83310BDF8B7
:100F90000000401CADF80000BDF800000628F1D3A9
:100FA000032087F83900781C3921F7F76FFF87F89D
:100FB0003A003B20CEE3022006F834009DF81400EE
:100FC00006EBC407403078704120B8703220F870CA
:100FD00087F804E033217971B8710021ADF8001071
:100FE00013E0D5F85002BDF80020C2F105029200CE
:100FF000D040BDF8002000F00F003A443030D071EE
:10100000BDF80000401CADF80000BDF80000062847
:10101000E7D3ADF80010302108E0BDF800003844F7
:101020004173BDF80000401CADF80000BDF80000A1
:101030001928F2D3032087F82600781C2621F7F719
:1010400025FF87F82700282084E3102006F83400C5
:1010500030206AE6102006F83400704665E69BF8FA
:10106000851D8DF81410BDF8001001EB01110CEB7B
:10107000C10101F5005191F81C22019991F8181253
:101080008A4205D1012200E0EEE3019981F817229E
:1010900099F8881B491C89F8881B0027ADF8007057
:1010A00010E0BDF8001000EB011101F5805191F83E
:1010B000851D9DF8142091420AD0BDF80010491CEE
:1010C000ADF800109AF85B1DBDF800209142E8D8F9
:1010D000BDF8001000EB011000F5805090F8841D61
:1010E0000F98401A401C8DF818009DF8140020B18C
:1010F0009DF81400401E8DF8140095F81D020F286D
:1011000005D295F81D02401C85F81D0201E085F806
:101110001D7210996520B13909297BD2DFE801F0F1
:10112000050C437A7A647A1D2F009DF81400503024
:1011300006F83400202166E09DF81400503006F8CF
:10114000340095F81D0206EBC40540F030006870CD
:101150000120A870E8702F7136E09DF8141050310E
:1011600006F8341095F81D1206EBC40541F0300165
:101170006970A8700120E8709DF8180023E09DF8C0
:101180001410503106F8341095F81D1206EBC40502
:1011900041F030016970A8700120E8709DF81800D6
:1011A00040F010000FE09DF81400503006F83400B5
:1011B00095F81D0206EBC40540F030006870012070
:1011C000A870E8700520287128460521F8F71CFA58
:1011D000CDE9080768710898000AA8710320E87132
:1011E000FA202872FFF726BB95F81E0285F8210227
:1011F00085F81E729DF81400503006F8340095F8FA
:101200001D0240F0C00106EBC4004170FA2181705C
:1012100003209FE289E0BDF800100798084441F6DA
:10122000883108440178491C01709AF8600D38B182
:101230000F99491CC9B2012836D0022875D144E063
:101240001098312802D04528F8D116E00020ADF8DA
:10125000000002A90CE0BDF80000BDF8003006EB6C
:10126000C402085CD054BDF80000401CADF800007A
:10127000BDF800000728EED364E40020ADF80000BC
:101280000AA90CE0BDF80000BDF8003006EBC4026E
:10129000085CD054BDF80000401CADF80000BDF85B
:1012A00000000728EED34DE48DF814109DF81400CB
:1012B00006F8340006EBC405032068700027AF7001
:1012C0000220E8702F7109200EE08DF814109DF8AF
:1012D000140006F8340006EBC405032068700027EC
:1012E000AF70EF702F710220687128460621F7F762
:1012F0009FFFCDE90807000AE8710898A871FFF779
:10130000E0BA99F8881B491C89F8881B9BF8851D51
:101310008DF814101099F3296FD008DC05296DD0D1
:10132000F12909D0F22989D114E015E23EE1F4292E
:101330007DD0F62988D1FDE0F52006F834009DF82F
:10134000140006EBC40568700027AF700520E87034
:10135000F12021E1F52006F834009DF8141006EB89
:10136000C400804641704FF0000980F80290F221DD
:10137000017195F89212417195F8920201281DD0E1
:1013800095F89202202870D00620ADF83400BDF800
:10139000340088F803004046BDF83410F7F748FFE2
:1013A000CDE90809BDF83420000A08F80200BDF8AC
:1013B0003420089908EB02004170B7E02520ADF811
:1013C00034004946ADF8009010E0BDF80000384404
:1013D00000F5005090F86522BDF8003008EB0300DE
:1013E0008271BDF80000401CADF80000BDF800009F
:1013F0000F28EAD3ADF8001012E051E0D8E0BDF8B4
:101400000000384400F5005090F87722BDF8003015
:1014100008EB03004275BDF80000401CADF8000069
:10142000BDF800000A28EAD395F88C2200E0A6E077
:1014300088F81F20ADF8001011E0BDF80000384416
:1014400000F5005090F88D12BDF8002008EB020066
:1014500080F82010BDF80000401CADF80000BDF879
:1014600000000528E9D392E7FFE70A20ADF8340031
:1014700048460EE0BDF80000384400F5005090F8F2
:101480008D12BDF8002008EB02008171BDF800004C
:10149000401CADF80000BDF800000428EAD376E750
:1014A000F52006F834009DF8141006EBC4008046C1
:1014B00041704FF0000980F80290F322027195F814
:1014C000922242710C22ADF8342095F88C22827160
:1014D000ADF8009010E0BDF80000384400F5005071
:1014E00090F88D12BDF8002008EB0200C171BDF824
:1014F0000000401CADF80000BDF800000528EAD34C
:10150000BDF8340088F803004046BDF83410F7F702
:101510008FFECDE90809BDF83420000A08F8020062
:10152000BDF83420089808EB0201B4E0BDF834009F
:10153000801C0FE10620ADF83400F52006F83400D9
:101540009DF8140006EBC40568700027AF70BDF865
:101550003400E870F62028719BF88C0D68712846DD
:10156000BDF83410F7F764FECDE90807BDF8341074
:10157000000A6854BDF83410089829448BE0F5201F
:1015800006F834009DF8140006EBC40568700027C7
:10159000AF700520E870F420287128460521F7F780
:1015A00047FECDE90807000A68710898A87131E480
:1015B00040F21321ADF83410F52106F834109DF8EF
:1015C000141006EBC4077970BDF83410090AB9701D
:1015D000BDF83410F970052139714FF0000841460B
:1015E0000DE0BDF80010014401F5805191F8621D35
:1015F000BDF800303B445971BDF80010491CADF8EE
:101600000010BDF800100A29EBD3BAF86E0D914610
:10161000000A01E0E0E0E2E0F873BAF86E0D387419
:10162000B5F8A002000A7874B5F8A002B874B5F84D
:10163000A0120E9801EB802081B20320F7F718FA70
:101640004546ADF800804FF40072484610E055E280
:10165000BDF80010014401F5805191F8E611BDF884
:1016600000303B44D974BDF80010491CADF800109F
:10167000BDF800109142EBD33846BDF83410F7F7AF
:10168000D7FDCDE90805BDF83410000A7854BDF83F
:10169000341008983944487048E794E29BF8850D67
:1016A0004FF00008414600F04BFF8DF8140095F80C
:1016B0001C12019890F81802814203D1019801216F
:1016C00080F8171299F8880B401C89F8880B10983D
:1016D000C5280BD012DCB6287ED00ADC012847D002
:1016E000142825D0B22837D107E1E2E06FE10FE0FE
:1016F00010E2B92877D0C3282ED1DAE0E1286DD0E6
:1017000006DCCA286BD0CE286AD0D72824D101E2C3
:10171000E5287EF4A2AFF52006F834009DF8140009
:1017200006EBC4056870A220A870E520FEF7AFBFE5
:10173000FA2006F8340006EBC4056870A87010980B
:10174000E8709DF81400287128460221F7F79EFBE7
:1017500068710620ADF834000E99FB48FB4D002956
:101760007ED001297DD002297CD003297BD10BE2D8
:10177000FA2006F8340006EBC4077870B8701098A9
:10178000F8709DF814003871D5F82402B0F1104FAC
:1017900005D34FF410000021CDE9080103E0D5F88E
:1017A0002402CDE9080840460FE0BDF80000C0F172
:1017B0000200C200DDE90801F6F735FDBDF80010B2
:1017C00039444871BDF80000401CADF80000BDF878
:1017D00000000328E9D304E083E004E0D4E074E0EF
:1017E00001E1FEF7C5BFF52006F834009DF81400AE
:1017F00006EBC40778709AF8600D0028D5F824022B
:101800000AD0B0F1104F36D0D5F82412CDE908181F
:10181000A620B870404644E0B0F5100F07D0D5F8C8
:101820002412CDE90818A520B870404615E04FF401
:1018300010000021CDE90801F5E7BDF80000C0F176
:101840000200C200DDE90801F6F7EDFCBDF800106A
:101850003944C870BDF80000401CADF8000004E039
:1018600064E175E180E19EE16FE0BDF800000328CE
:10187000E3D3FEF7BFBF4FF010400021CDE90801D0
:10188000C6E7BDF80000C0F10300C200DDE90801B1
:10189000F6F7C9FCBDF800103944C870BDF8000067
:1018A000401CADF80000BDF800000428E9D3FEF7A5
:1018B000BFBFF52006F834009DF8140006EBC40500
:1018C0006870A220A870C32030E7F52006F8340025
:1018D0009DF8140006EBC4056870A220A870CA2009
:1018E00024E7F52006F834009DF8140006EBC40543
:1018F0006870A220A870B62018E7F52006F834001A
:101900009DF8140006EBC40778709AF8600D18B1C2
:10191000A520B87040462FE0A420B87040460EE0E5
:10192000D5F85002BDF80010C1F10101C900C8404E
:10193000BDF800103944C870BDF80000401CADF877
:101940000000BDF800000228EAD3B22078713846C2
:10195000052100F026FDB8718EE4D5F85002BDF8DF
:101960000010C1F10201C900C840BDF8001039449F
:10197000C870BDF80000401CADF80000BDF80000C4
:101980000328EAD3FEF796BFF52006F834009DF849
:10199000140006EBC4077870A620B87040460EE02D
:1019A000D5F85402BDF80010C1F10301C900C840C8
:1019B000BDF800103944C870BDF80000401CADF8F7
:1019C0000000BDF800000428EAD3FEF7ACBFF52004
:1019D00006F834009DF8140006EBC4056870A220D8
:1019E000A870C520A2E6F52006F834009DF8140082
:1019F00006EBC40568709AF8600D18B1AE20A870A7
:101A0000404655E0AC20A870404615E007F5005070
:101A1000D0F83D0207F50051D1F84112BDF8002081
:101A2000C2F10402D200F6F7FEFBBDF80010294413
:101A3000C870BDF80000401CADF80000BDF8000003
:101A40000528E3D3404615E007F50050D0F84502DD
:101A500007F50051D1F84912BDF80020C2F1040287
:101A6000D200F6F7E0FBBDF8001029440872BDF87B
:101A70000000401CADF80000BDF800000528E3D3CD
:101A8000FEF7A6BF07F50050D0F83D0207F500515C
:101A9000D1F84112BDF80020C2F10502D200F6F7DC
:101AA000C2FBBDF800102944C870BDF80000401CFE
:101AB000ADF80000BDF800000628E3D3404615E06D
:101AC00007F50050D0F8450207F50051D1F849124A
:101AD000BDF80020C2F10502D200F6F7A4FBBDF864
:101AE000001029444872BDF80000401CADF8000009
:101AF000BDF800000628E3D3FEF7ADBFF52006F8D9
:101B000034009DF8140006EBC4056870A220A8708C
:101B1000E7200BE6F52006F834009DF8140006EBEC
:101B2000C4056870A220A870D720FFE5BDF8341066
:101B3000C9B38021F8F745FABDF83400C5F8A40010
:101B400002480121A0302CE0000C0240006002405D
:101B5000BDF8341039B30821F8F733FABDF8340072
:101B6000686701211B481CE0BDF83400D8B14FF470
:101B700080711948F8F725FABDF83400C5F8BC00A3
:101B80001448012148300CE0BDF8341059B14FF42D
:101B90008061F8F716FABDF83400E8650D480121B8
:101BA0001838F7F79BFB0D4890F8E703002807D09B
:101BB00006EBC4000023BDF834100E9AF8F726FA9D
:101BC00011B0BDE8F08F99F8880B401C89F8880B9C
:101BD000F6E700007060024000000240A4220020EE
:101BE0002DE9F04700242DED048B804689469FEDBA
:101BF0001E9B25462646E20040464946F6F713FB63
:101C0000C7B22046F6F7EEFC41EC110BB0EE490AE4
:101C1000F0EE690A09F004F9380907F00F0100EB4A
:101C20008000B0EE408AF0EE608A01EB4000F6F7EB
:101C3000D9FC53EC182BF6F7E3FB41EC180B2846C4
:101C40003146F6F7DCFC53EC182BF6F732FBF6F7CF
:101C500009FD641CE4B205460E46082CCBD3BDEC4E
:101C6000048BBDE8F0870000000000000000594030
:101C700070B50E4D40F224442146284608F089FDF7
:101C8000012812D1298828462A1D1188214608F0EA
:101C90001DFD0748012180F8291B0648D0F88C005B
:101CA0000549C0F57A70A1F83C0470BD00440040BD
:101CB000A422002000600240A452002010B50B4C6A
:101CC00040F22441204608F064FD01280DD120880F
:101CD000201D00880648012180F8351B0548406C0E
:101CE0000549C0F57A70A1F83E0410BD004C0040D3
:101CF000A422002000600240A452002010B50B4C2A
:101D000040F22441204608F044FD01280CD12088EF
:101D1000A0880748012180F8411B06484069064910
:101D2000C0F57A70A1F8400410BD000000500040DA
:101D3000A422002000600240A452002010B50B4CE9
:101D400040F22441204608F024FD01280DD12088CE
:101D5000201D00880648012180F84D1B0548C06AF7
:101D60000549C0F57A70A1F8420410BD0048004052
:101D7000A422002000600240A452002010B5124CA2
:101D800010492046F7F794FA00212046F7F7A6FA03
:101D90000E4C4021204608F0F5FC0028F9D08021A7
:101DA0000B48F8F710F9084C0A49183C2046F7F799
:101DB0007FFA01212046F7F791FA074901200871BF
:101DC00010BD000000802020A060024000440040C0
:101DD000000C0240008800201200002010B5124CB8
:101DE00010492046F7F764FA00212046F7F776FA03
:101DF0000E4C4021204608F0C5FC0028F9D00821EF
:101E00000B48F8F7E0F8084C0A49303C2046F7F751
:101E10004FFA01212046F7F761FA074901200871BE
:101E200010BD00002080002070600240004C004087
:101E3000000C0240008020101200002010B5124C4F
:101E400010492046F7F734FA00212046F7F746FA02
:101E50000E4C4021204608F095FC0028F9D04FF4A4
:101E600080710B48F8F7AFF8074C0A49A83C2046A8
:101E7000F7F71EFA01212046F7F730FA064901204C
:101E8000087110BD00800028B8600240005000407A
:101E900000000240208000101200002010B5124CFB
:101EA00010492046F7F704FA00212046F7F716FA02
:101EB0000E4C4021204608F065FC0028F9D04FF474
:101EC00080610B48F8F77FF8074C0A49303C204600
:101ED000F7F7EEF901212046F7F700FA064901204D
:101EE000087110BD00800018586002400048004092
:101EF000000C024000880010120000202DE9F0477D
:101F0000012190B0480505F0CBFE8648F7F7F0F9BF
:101F1000402738010024CDE90540C5010794089405
:101F2000CDE9094546040C940D94DFF8FC917F48F7
:101F30000B94CDE90207CDE9006969460E94794812
:101F4000F7F77EFA012210217648F7F763FADFF8F7
:101F5000D4A1AAF1180A5046F7F7CAF94FF47A78D3
:101F6000CDE90348E811CDE9054007940894CDE98F
:101F700009456F480B940C940D9400960E94CDE98E
:101F8000019069465046F7F75BFA01215046F7F792
:101F9000A5F9DFF890A1AAF1300A5046F7F7A8F9A1
:101FA000E811CDE9054007940894CDE909450C9462
:101FB0000D94DFF8809160480B94CDE90207CDE9DC
:101FC000006969460E945046F7F73AFA012210214B
:101FD0005046F7F71FFADFF84CA1AAF1600A504605
:101FE000F7F786F9CDE90348E811CDE905400794F4
:101FF0000894CDE9094551480B940C940D94009632
:102000000E94CDE9019069465046F7F719FA01217F
:102010005046F7F763F9DFF80CA10AF1180A5046A9
:10202000F7F766F9E811CDE9054007940894CDE982
:1020300009450C940D94DFF8089142480B94CDE9C2
:102040000207CDE9006969460E945046F7F7F8F9A2
:10205000012210215046F7F7DDF9DFF8C8A0AAF1F8
:10206000900A5046F7F744F9CDE90348E811CDE965
:10207000054007940894CDE9094533480B940C9426
:102080000D9400960E94CDE9019069465046F7F7FD
:10209000D7F901215046F7F721F9DFF88890A9F127
:1020A00048094846F7F724F90397E811CDE90540B8
:1020B00007940894CDE9094525480B940C940D9498
:1020C000224F00960E94CDE9017069464846F7F715
:1020D000B7F9012210214846F7F79CF9DFF8449040
:1020E000A9F178094846F7F703F9CDE90348E81163
:1020F000CDE9054007940894CDE9094515480B94AE
:102100000C940D9400960E94CDE9017069464846F2
:10211000F7F796F901214846F7F7E0F810B0BDE867
:10212000F0870000A060024004440040205B0020D3
:1021300080640020044C0040785D00206868002026
:1021400004500040D05F0020506C00200448004044
:1021500028620020387000202DE9FC41012108464A
:1021600005F09EFD0121042005F09AFD01210820C3
:1021700005F096FD0121402005F092FDDFF8FC807E
:10218000072205214046F7F705FF072206214046B2
:10219000F7F700FF072208214046F7F7FBFE07226A
:1021A00009214046F7F7F6FE354F08220A21384646
:1021B000F7F7F0FE08220B213846F7F7EBFE08226E
:1021C00002214046F7F7E6FE08220C213846F7F7D1
:1021D000E1FE02268DF8056000244FF459708DF859
:1021E0000640012500908DF807508DF8046069467F
:1021F0004046F7F793FE8DF805604FF4E0508DF8F8
:10220000064000908DF807508DF804606946384606
:10221000F7F784FE4FF4916000908DF806408DF83A
:10222000045069464046F7F779FE280200908DF881
:1022300006408DF8045069461248F7F76FFE8DF896
:1022400006404FF4F040104C00908DF80450694661
:102250002046F7F763FEA9032046F7F7B2FE6903AD
:102260002046F7F7AEFEA1142046F7F7AAFEE114C8
:102270002046F7F7A6FEBDE8FC810000000C0240F6
:1022800000080240000002400018024070B500241F
:10229000FFF762FFFFF732FE00F01EF80C48002146
:1022A0000170817041700121C1704FF47A718160B9
:1022B000084D042085F8240B04E0204600F062F964
:1022C000641CE4B295F8240BA042F6D870BD00005F
:1022D00024570020A4220020F8B511208DF800001A
:1022E00002258DF8015001248DF802408DF803403D
:1022F000684601F0AFF926208DF800008DF8014006
:1023000000268DF802608DF80340684601F0A2F9BE
:102310000E208DF800008DF801508DF802408DF8E8
:102320000340684601F096F927208DF800008DF8EB
:1023300001408DF802608DF80340684601F08AF98B
:102340000F208DF800008DF801508DF802408DF8B7
:102350000340684601F07EF934208DF800008DF8C6
:1023600001408DF802608DF80340684601F072F973
:102370002F208DF800008DF801508DF802408DF867
:102380000340684601F066F935208DF800008DF8AD
:1023900001408DF802608DF80340684601F05AF95B
:1023A000F8BD01B9102110F8012B10F8013B491EAE
:1023B0005A400904090CF8D102F07F007047000070
:1023C0002DE9FF5F14460F464FF480564FF48068A6
:1023D0004FF4C0694FF00C0A40F2244B002580B145
:1023E000012830D0022851D0032871D1012188045E
:1023F00005F07AFC0097012C6DD0022C70D094B3BC
:1024000077E00121480405F06FFC0097012C03D010
:10241000022C06D054B10DE0ADF80460ADF8088090
:1024200008E0ADF80460ADF8089003E0ADF80450A2
:10243000ADF80850ADF80650ADF80C50ADF80AA054
:1024400069463B4C5DE00121C80405F04DFC009756
:10245000012C03D0022C07D05CB10EE0ADF8046073
:10246000ADF8088009E040E0ADF80460ADF80890F0
:1024700003E0ADF80450ADF80850ADF80650ADF8E3
:102480000C50ADF80AA069462A4C3AE00121080533
:1024900005F02AFC0097012C03D0022C06D054B181
:1024A0000DE0ADF80460ADF8088008E0ADF8046018
:1024B000ADF8089003E0ADF80450ADF80850ADF861
:1024C0000650ADF80C50ADF80AA069461A4C18E059
:1024D0002CE000E004E0ADF80460ADF8088008E00E
:1024E000ADF80460ADF8089003E0ADF80450ADF825
:1024F0000850124CADF80650ADF80C50ADF80AA0DB
:102500006946204608F07CF90121204608F0E1F8F0
:1025100001225946204608F05BF91021204608F0B8
:10252000D5F80122C021204608F0DDF8BDE8FF9F64
:1025300000440040004C0040005000400048004073
:102540002DE9FC410024CDE900446F4664220023BC
:10255000F5F738FE0E460546104619460A220023B6
:10256000F5F730FE010102F00F000818385504F1AC
:102570000104E4B228463146082CE7D3DDE9000126
:10258000BDE8FC812DE9F84F8F4E804600250420E0
:1025900086F8240B08EB480101EB0810A6F58057DC
:1025A00007EB001B0BF5805494F8610D012803D153
:1025B0000021404600F010F908EB4802BA4607EB4C
:1025C0008207A7F59B6707F500574FF0000987F8CA
:1025D000009087F8029087F8019087F80390052112
:1025E000B96087F8309087F83290012087F8310081
:1025F00087F83300D4F85C0D00EB80004000B8632E
:1026000094F8592DD4F8541D4046A7F62837FFF703
:10261000D7FE94F85A1D08EB081202EB08206B4A0B
:10262000072902EBC000009000F5005015D2DFE84A
:1026300001F01404060A0C0E1A00052100E00F2117
:1026400080F8181209E00721FAE70421F8E7D4F826
:102650005C1D64225143C7F8601B9AF81810D046DD
:10266000012902D017E00321EAE780F8189201203F
:10267000C7F8300B564F80213846F7F7A4FC0821E5
:102680003846F7F7A0FCB9155248F7F79CFC391506
:102690003846F7F798FC4FF0A10EC2466FE000985D
:1026A00005EB051200EBC20000F5077000F50050C5
:1026B00000210173012282734173C173D4F85C2D30
:1026C00094F85B7D7A4302EB8202920042610BEB4D
:1026D000051202F5805292F8867D27F0800782F875
:1026E000867D017094F85A1DA0F50770072944D221
:1026F000DFE801F0430408080A0C0E00E52180F829
:1027000021123AE07146FAE7B121F8E73121F6E704
:10271000F12180F8211200212BE001EB011303EBE2
:1027200001230AEBC30701EB410303EB01130AEB9F
:102730000313002003F5805915E003EB001C0CF592
:10274000805C9CF884CD92F88C8DC44509D192F8B8
:1027500084CD00EB001807EBC80808F5005888F88E
:1027600093C2401CC0B299F85BCD8445E5D8491CA2
:10277000C9B296F8240B8842CFD86D1CEDB294F8FC
:102780005B0D5346A8428AD8002086F8250B00EB43
:10279000400101EB001103EB011101F5805191F8AB
:1027A0005A2D052A09D291F85A2D32B196F8252BC7
:1027B00091F85B1D114486F8251B401CC0B204280B
:1027C000E5D3BDE8F88F0000A4220020A412002069
:1027D000000C0240000002402DE9F041054663482C
:1027E0004FF480425310066861488414C71439B10D
:1027F000C5B1012D18D0022D18D0032D1BD117E023
:1028000035B1012D06D0022D06D0032D13D105E0E0
:10281000114604E0194602E0214600E03946F7F788
:10282000D2FB08E0114604E0194602E0214600E030
:102830003946F7F7C6FB642009F038FC00224FF454
:1028400016512846FFF7BCFD4A4905EB450001EB50
:10285000800000F58050002280F85A2BC0F85C2BD5
:1028600005EB450000EB051001EB001000F5805072
:10287000D0F85C3D01F58041C1F88834012381F82E
:10288000813490F85A1D3C4C962305EB850020447A
:1028900006290AD2DFE801F009030505073376218E
:1028A00002E0837001E06E218170C5EB0511334BAE
:1028B00001EB8101C02403F8314003EBC1046270D5
:1028C0000821A170E27006F00F0105EB051211441A
:1028D0002171807860712020A071E17180202072C8
:1028E0004C2060725420A0722548264F0B2645B11B
:1028F000012D0FD0022D25D0032D14D12DE06621FE
:10290000D2E78021F7F75DFBC7F8A4601D480121DD
:10291000A03006E00821F7F754FB7E671948012133
:102920007030F6F7DBFC184890F8E70328B1204632
:1029300000232A460B21F7F769FBBDE8F04164202C
:1029400009F0B4BB4FF480711048F7F73AFBC7F8B1
:10295000BC600C480121B830E3E74FF48061F7F721
:1029600030FBFE65074801215830DAE7187AFF1F6F
:1029700000180240A412002020740020205B0020D8
:10298000000C024000600240A4220020000002402F
:102990002DE9F04700252DED028B8EB08DF82850E3
:1029A0008DF82C508DF83050CDE90855CDE9005503
:1029B0008DF808508DF80C508DF810508DF814508B
:1029C000ADF818509FEDFE0AFE4C07958DED090AF3
:1029D00094F83A0D4FF0010908B384F83A5DB4F861
:1029E000520DF94E3168C1F57A71884217D13068BD
:1029F000C0F57A70A4F8500D371F00213846F6F75D
:102A00006DFCF2493846F6F753FCF14981F8009025
:102A10004FF47A70306001213846F6F75FFC94F885
:102A2000DA0CEB4FBF1C02280AD0042801D005287D
:102A300003D184F8469DC4F8485D8DF8285055E2CE
:102A4000E048603090F8D80BDFF8888341F6865A6A
:102A500008F1020606F5805600287DD001287CD0BA
:102A60000228E6D1F879397A40EA0120C117CDE988
:102A70000001D7480721801CF6F7DAFBCDE90805ED
:102A8000DDE90001089B694058400843D1D13878FE
:102A9000401E8DF8100086F82C5D9DF8100046460B
:102AA000404400F5805080F88555B879F5F79AFDD7
:102AB00041EC110B9FEDC80B08F0B2F93879B0EE7C
:102AC000408AF0EE608AF97840EA0120F5F78AFD45
:102AD00053EC182BF5F706FDF5F7E9FD9DF81010FE
:102AE00006EB011101F58051C1F895059DF8100024
:102AF00006EB001000F58050C0F891559DF81000CD
:102B000006EB001000F58050C0F899559DF81000B4
:102B100006EB001000F58050C0F89D559DF80800A8
:102B200000EB400101EB00109DF8101006EB0010C7
:102B300000EB011101EB0A00017841F08001017006
:102B4000797A9DF8080000EB001202EB002006EBFA
:102B5000C0029DF8100001E017E00BE100EB00104F
:102B600002EBC00000F5005080F858129DF80800F4
:102B700000EB400101EB001006EB001000F5805067
:102B800090F85B0D84F8840553E79DF8081008EB76
:102B9000410000F58040B0F83414781C891FF6F726
:102BA0005DFBC117CDE908019DF8081008EB410055
:102BB00000F58040B0F834148548C01E0844042154
:102BC00005F052FBC117CDE90001DDE908320146ED
:102BD0000198594050400143D6D186F82C5D387990
:102BE000ADF81800BDF818003128CDD19DF80800C7
:102BF000464608EB400000F58040B0F8340441211F
:102C0000183890FBF1F0C117CDE9000184F8840574
:102C10008DF82850A4E09DF8280000EB801038447F
:102C2000017D9DF82800304400F5805080F885151E
:102C30009DF82800082100EB801038441A3005F078
:102C4000DFFA00EE100AB8EEC00A8DED090A10EEA8
:102C5000100A9DF8281006EB011101F58051C1F80A
:102C600095059DF82800082100EB8010384432308B
:102C700005F0C6FA00EE100AB8EEC00A8DED090A9A
:102C800010EE100A9DF8281006EB011101F5805195
:102C9000C1F891059DF82800082100EB8010384408
:102CA0003A3005F0ADFA00EE100AB8EEC00A8DED2C
:102CB000090A10EE100A9DF8281006EB011101F523
:102CC0008051C1F899059DF82800082100EB80107B
:102CD0003844423005F094FA00EE100AB8EEC00A0B
:102CE0008DED090A10EE100A9DF8281006EB01116F
:102CF00001F58051C1F89D059DF8080000EB4001E9
:102D000001EB00109DF8281006EB001000EB0111FC
:102D100001EB0A00017841F0800101709DF8080084
:102D200006EB400000F58040B0F834142848401C01
:102D3000095C9DF8080000EB001202EB002006EB96
:102D4000C0029DF8100000EB001002EBC00000F57F
:102D5000005080F858129DF82800401C8DF828007B
:102D60009DF82810DDE90023891A75EB0300FFF6B2
:102D700052AF5EE6787DB97D40EA0120C117CDE90A
:102D8000000113481521801CF6F752FACDE9080519
:102D9000DDE90010089B684059400143E9D13878CB
:102DA000401E8DF8100086F82C5D9DF810004646F8
:102DB000404400F5805080F885559DF810000FE0E4
:102DC00000000000A42200202C64024000880010B3
:102DD000CE0A0020A41200200000000000002440C1
:102DE00008EB001000F58050C0F89555B879797956
:102DF00040EA012000EE100AF8EE400A9FED400A7A
:102E0000387980EE801AF97840EA012000EE900AC5
:102E10009DF81000F8EE600A71EE200A10EE901A8C
:102E200006EB001000F58050C0F89115B87A797A59
:102E300040EA012000EE900A387AB8EE601AC1EE3E
:102E4000000AF97940EA012000EE100A9DF81010FE
:102E5000B8EE400A30EE800A10EE100A06EB0111BF
:102E600001F58051C1F89905F87A0006387BF97AA6
:102E700040EA01200AD400EE100ADFED220AB8EE83
:102E8000400A20EE200A10EE100A0BE0404280B209
:102E9000F5F7A8FB9FED1C1B53EC112BF5F7B0FACF
:102EA000F5F705FC9DF8101006EB011101F58051B6
:102EB000C1F89D059DF8080000EB400101EB0010F2
:102EC0009DF8101006EB001000EB011101EB0A0059
:102ED000017841F080010170F97D32E69DF828000B
:102EE0003D549DF82800401C8DF828009DF82800CE
:102EF0001428F3D30EB0BDEC028BBDE8F0870000C0
:102F000000FF7F470000803D000000000000B0BFD0
:102F10002DE9F34F8246F2A085B0D0E90010CDE94B
:102F20000110F1A00026D0E90010CDE90310F0490E
:102F300035463746B046B3464E70EE4A02EB0A00BD
:102F400000F5805090F82C1D042921D1052180F82E
:102F50002C1D594680F8DEBC90F8BC3C23F0800361
:102F600080F8BC3C5046BAF1020F07D0042803D0C9
:102F7000BAF1050F0CD105E0DF4805E0DE4831214C
:102F8000801E01E0DC48401C00F5005080F8E31C86
:102F9000D8480AEB4A0100EB011000F58050814649
:102FA00090F8D22BD548D64C4FF48071022A7DD0B0
:102FB000042A0FD0052A0AD194F82C0D401C84F85D
:102FC0002C0D99F8D11BD9F8CC0B00F0FDFA07B005
:102FD000BDE8F08F94F8DC2C002AF8D0F6F7F1FF6A
:102FE000C44E99F8D11BD9F8CC0B00F0EDFA94F847
:102FF000DC0C012802D0022841D11BE094F8DB1C34
:1030000001EB8100C0EB8110304490F86080B94A38
:1030100050F8617F02F64173C2F8217F4768C2F819
:10302000257F8268C6F8292F026A1A60808C9880F2
:103030000F0924E096F8208F1DE007EB470101EB14
:10304000071106EB0112002002F5805109E002EBA6
:10305000001303F5805393F884CDC44505D0401C7C
:1030600080B291F85B3D8342F1D891F85B1D8142BB
:1030700005D87F1CBFB294F8240BB842DDD8404677
:103080000021FFF75DFA02460B4606210020CDF82D
:1030900000B004F05BFD07EB470000EB071006EB08
:1030A0000017A7F5247707F5005700E0ADE0387862
:1030B000C0F381000090D6F8212F00230721184685
:1030C00006F6297604F042FD387800F003000090FF
:1030D00056F8042C00230821184604F037FD3878F0
:1030E000C0F301100090326800230921184604F053
:1030F0002DFD322004F8C70F30206070717F00EB87
:103100001111A170717F01F00F013031E1702D219B
:103110002171327F00EB12126271327F02F00F02D6
:103120003032A271E171F17E00EB11112172F17E5A
:1031300001F00F0130316172B17E00EB1111E172CB
:10314000B17E01F00F01303121733A216173727E3B
:1031500000EB1212A273727E02F00F023032E273A1
:103160002174317E00EB11106074307E00F00F008E
:103170003030A07400202021624F40F28A22C73CE8
:10318000A6F629763954401C80B29042FAD34FF00B
:103190000A0C87F800C087F801C00021002006EB68
:1031A0004112131893F85B3F202B03D1401C80B2CF
:1031B0002028F6D31F280DD20020131893F85B3F68
:1031C00000EB451807F80830401C80B22028F4D3E3
:1031D0006D1CADB2491C89B21429DFD307EB451031
:1031E00080F820C080F821C080F822C080F823C079
:1031F00080F824C080F825C0252000EB451000048D
:10320000000C84F8DCBC55D1E1E60F468046F6F7A9
:10321000DAFE4FF400714046F6F7D5FE354D99F8C9
:10322000D11BD9F8CC0B00F0CFF994F82C0D401C31
:1032300084F82C0D0AEB4A0101EB0A1005EB001093
:1032400000F5805090F8600DE8B1022501240326B6
:1032500001283AD00228D7D139464046F6F7B3FEC6
:10326000284F3C707E7087F802B087F803B087F86B
:1032700004B07D7106212348F5F7DAFF010AF971E0
:10328000B871082016E0069831280AD04528BBD12D
:103290001C4803A98A5D8255761CB6B2072EF9D365
:1032A00007E0184801A98A5D8255761CB6B2072E40
:1032B000F9D307201449086013480121001FF6F7CD
:1032C0000DF80B4981F801B081E60E4F3C707E701D
:1032D00087F802B0FD7087F804B009207871C9E75B
:1032E0000169323031303000016932304530300010
:1032F000CE0A0020A4120020A802002000080240EC
:10330000A4220020B80E0020A464024070B50D4C29
:1033100040F224452946204607F03BFA002810D009
:103320002946204607F0D2F92088201D008806484B
:10333000012180F8391D05490968C1F57A71A0F8A5
:10334000521D70BD00140140A42200202C640240D4
:1033500010B5124C10492046F5F7AAFF002120466F
:10336000F5F7BCFF0E4C4021204607F00BFA002871
:10337000F9D04FF400710B48F6F723FE074C0A49C9
:10338000783C2046F5F794FF01212046F5F7A6FF8B
:1033900006490120487010BD00802020A064024032
:1033A000001401400008024000880010CE0A0020EE
:1033B0002DE9F04301218FB0880504F071FCDFF89E
:1033C00094904846F5F794FF4020050103900024AF
:1033D000CDE90545C60207940894CDE909464FF0AA
:1033E00020681E480B940C940D941B4FCDF8008060
:1033F0000E94CDE9017069464846F6F721F801229E
:1034000010214846F6F706F8DFF84890A9F1780948
:103410004846F5F76DFF4FF47A70CDE90340CDE9EA
:10342000054507940894CDE909460D480B940C9482
:103430000D94CDF800800E94CDE9017069464846A0
:10344000F5F7FEFF01214846F5F748FF0FB0BDE84C
:10345000F0830000A064024004140140B80E002074
:10346000D00A00207CB50121042004F019FC184E7C
:10347000082206213046F6F78DFD08220721304646
:10348000F6F788FD02218DF8051000258DF806500D
:103490000124C0208DF8074000908DF80410694683
:1034A0003046F6F73BFD4FF4407000908DF8044035
:1034B0008DF8065003208DF805008DF80740694609
:1034C0003046F6F72BFD61023046F6F77AFD7CBDFB
:1034D000000802402DE9F0410024FFF7C3FF00215E
:1034E0004FF4E13000F070F8FFF762FF00F04EF8A3
:1034F00024480023037083704370C37002218160ED
:103500000373837301264673C6734FF47A71416166
:103510001D4A04EB440102EB8100A0F5447000F564
:103520000050037083704670C67002EB011505F5FC
:103530008055D5F8D41B01EB81014900816095F8D5
:10354000D21BA0F54F60022909D0042901D005291A
:1035500011D1101900F5805080F8E33C0BE03121C7
:10356000171907F5805787F8E31CD5F8D41B642595
:103570006943C0F8F81C641CE4B2052CC9D3BDE84B
:10358000F0810000DC2F0020A412002038B5452077
:103590008DF8000002208DF8010001248DF8024012
:1035A0008DF80340684600F055F847208DF800007C
:1035B0008DF8014000208DF802008DF80340684628
:1035C00000F048F838BD00007FB50C4605460121E3
:1035D000202004F0A1FB00204FF480510095012C25
:1035E00003D0022C06D064B10FE0ADF804104FF404
:1035F000806103E0ADF804104FF4C061ADF808102D
:1036000003E0ADF80400ADF80800ADF80400ADF833
:103610000600ADF80C000C200D4CADF80A00694610
:10362000204607F0EDF80121204607F052F801226C
:1036300040F22441204607F0CBF81021204607F045
:1036400045F80122C021204607F04DF87FBD00005B
:103650000014014030B50F23C27801780125FAB17A
:10366000144A126801F1E02102F4E062C2F5E0625E
:10367000C2F30722C2F10404D3404278A240847806
:103680001C401443220181F80024007800F01F013F
:103690008D404009800000F1E020C0F8005130BDAD
:1036A00001F01F0085404809800000F1E020C0F8CB
:1036B000805130BD0CED00E0024A11400143024848
:1036C0000160704780FFFF1F08ED00E010B500218A
:1036D000074B0A46002003EBC004401CC0B26254F2
:1036E0008028F8D3491CC9B20829F3D310BD0000C3
:1036F000237E00202DE9FE4F0026171A8146701EFA
:103700003546A3EB010A8846002F02DD4FF0010188
:1037100002E003D14FF00001019102E0C7F1000780
:103720000190BAF1000F02DD4FF0010002E003D179
:103730004FF00000009002E0C7F1000A00905046F0
:10374000574501DD3C4600E00446601C4FF0000B8D
:10375000029016E008F0FF0109F0FF000C9A00F05B
:1037600015F83E445544A64202DD0199361B8944B2
:10377000A54202DD00992D1B88440BF101001FFAC0
:1037800080FB02998B45E5DBBDE8FE8F30B5CC08A8
:1037900001F0070301259D40EBB2064D05EBC00586
:1037A000C808285C0AB1184302E063EA0000C0437D
:1037B000285530BD237E00202DE9FC4101210A203F
:1037C00004F06EFA01248DF8044000264FF4C05036
:1037D0008DF80660032700908DF805708DF807407E
:1037E00069464648F6F79AFB8DF804408DF8066066
:1037F0008DF80570A5028DF80740414C009569468B
:103800002046F6F78BFBC82008F050FC29462046DE
:10381000F6F7D7FBC82008F049FC29462046F6F702
:10382000D2FBC82008F042FC0021FD2000F054FA31
:103830000021122000F050FA0021AE2000F04CFAD6
:103840000021D52000F048FA0021A02000F044FA21
:103850000021A82000F040FA00213F2000F03CFAAF
:103860000021D32000F038FA0021084600F034FA95
:103870000021402000F030FA0021A02000F02CFAB6
:103880000021C02000F028FA0021DA2000F024FAFC
:103890000021122000F020FA0021812000F01CFA03
:1038A00000217F2000F018FA0021D92000F014FA3E
:1038B0000021822000F010FA0021DB2000F00CFA39
:1038C0000021342000F008FA0021A42000F004FABE
:1038D0000021A62000F000FA0021202000F0FCF9D1
:1038E0000021084600F0F8F9FFF7F0FE0021AF20B4
:1038F00000F0F2F900F054F8BDE8FC81000C024041
:10390000000402400346012000E05843491EC9B2AA
:10391000FBD270472DE9F84F82460A980D46504376
:103920006421B0FBF1F0984600F0FF0B4FF0010965
:103930000AEB02072B4600245046FAB21946CDF88E
:103940000090FFF7D7FE05EB0806F3B2FAB2F1B22A
:103950005046CDF80090FFF7CDFE5246F3B229460F
:103960001046CDF80090FFF7C5FEF3B2FAB2F8B2F8
:103970002946CDF80090FFF7BDFE4F460AEB0B0637
:1039800009E02819C3B2C1B2F2B250460097FFF75E
:10399000B1FE641CE4B24445F3D3BDE8F88F0000E7
:1039A00070B50025B020294600F096F900210846A0
:1039B00000F092F90021102000F08EF9084E00244A
:1039C00006EBC4000121405D00F086F9641CE4B2FE
:1039D000802CF5D36D1CEDB2082DF0D370BD000026
:1039E000237E002070B50B4C05460221204604F0D2
:1039F00021FB0028F9D02946204604F024FB0121B0
:103A0000204604F017FB0028F9D0204604F019FBEB
:103A1000C0B270BD003800402DE9FC4F1D468846FD
:103A200081468B460090082B0ED0680700D00120FD
:103A300000EBD500690810FB01F0C0B2203A02F09B
:103A4000FF0A0026019046E00620F7E7082D10D077
:103A50000C2D14D0102D16D0182D3FD121490AEB72
:103A6000CA0001EB80000027845DE0070FD00B9AAD
:103A700010E01D490AEB4A0001EB4000F3E70AEBB6
:103A80004A001A49EDE71A4901EB0A10EBE70B98D7
:103A900030B3002241464846FFF778FE7F1C640899
:103AA00008F10100FFB200F0FF08082FDDD309F193
:103AB000010000F0FF09082D0AD00099A9EB0100D0
:103AC000B0EB550F04D10BF10800894600F0FF0B55
:103AD000761CD846F6B201988642B7D3BDE8FC8F73
:103AE0000122D7E7C8DE01083CD2010864D40108EE
:103AF000D8D801082DE9FF4F81B04FF00005DDE96E
:103B00000F7ADDF838B05FEA030980462E4612D1FD
:103B10000398F4F767FD41EC100B07F0E9F89FED0F
:103B2000331B51EC100B53EC112BF4F7C2FBF4F7E1
:103B30007AFD00F0FF09082F00D10225D94510D8E1
:103B4000BBF1000F0DD03B463022CDF800A040461F
:103B50000299FFF761FF05EB570101EB080000F048
:103B6000FF08002431E0A9EB0B01A1420DD105EBC8
:103B7000570101FB0480C0B23B462E22CDF800A0C5
:103B80000299FFF749FF01261DE0001B401EC1B24C
:103B90000A20FFF7B7FE0399CDF800A0B1FBF0F0C3
:103BA0000A21B0FBF1F201FB120106EB0800A1B102
:103BB00005EB570202FB04003031C0B2CAB23B46EB
:103BC0000299FFF729FF641CE4B209EB0600A0424A
:103BD000C9D805B04846BDE8F08F05EB570101FB99
:103BE0000400C0B23B463022EAE7000000000000BB
:103BF0000000F03F2DE9FF4F81B0064600900F46D0
:103C00004FF0000A8946580700D0012000EBD3008E
:103C10000490002032E0002029E00E98002410F8E3
:103C20000A500AF101001FFA80FAE80701D00F9A42
:103C300002E00F9848B3002239463046FFF7A6FD50
:103C40007F1C641C6D08E4B2FFB2082CEDD3761C17
:103C50000098F6B2311A0398814204D109F10800A4
:103C6000009E00F0FF0908F101004F46C0B2039921
:103C700080468842D1D30BF10100C0B2049983463B
:103C80008842C8D305B0BDE8F08F0122D4E72DE902
:103C9000F8431D46DDE908781646894604460EE0DD
:103CA0003B4649462046CDF80080FFF7B5FE082F79
:103CB0000ED004EB5700C4B26D1EEDB2761C002D81
:103CC00004D03278202A01D37E2AE9D9BDE8F883CE
:103CD000A41DE4B2F0E700002DE9F041114C0646C6
:103CE0004FF4006500292946204602D0F6F76BF90B
:103CF00001E0F6F766F94FF4805739462046F6F7AB
:103D000060F939460848F6F75EF93046FFF76AFE73
:103D100039462046F6F757F929462046BDE8F041D6
:103D2000F6F751B9000C0240000402402DE9F04FB3
:103D300089B04FF00009C846ADF80090ADF8049086
:103D4000ADF80890ADF80C90ADF81090ADF8149067
:103D5000F74C4D4694F8E206A4F5805A0106F54E5C
:103D60000AF580404FF0010B069001F1348701F015
:103D700038BF94F8A607022805D194F8A50710B11A
:103D80000720ADF81400BDF8140030448079BDF868
:103D900014103144C97840EA0160BDF81410314470
:103DA0000979BDF8142009043244527941EA02210C
:103DB0000843E1494A6890424CD04860BDF814007D
:103DC00030448078BDF814103144497840EA012528
:103DD000B4F86A16BDF814002844801C814239D317
:103DE000B4F86A06BDF81410401B401A801EA4F8EF
:103DF0006A06BDF8140029463044F5F719FABDF8F3
:103E00001410294431444978BDF814202A44B25C86
:103E100041EA0221814241F0BF8694F8E70340B1B4
:103E2000A81C81B2BDF81400012330440422F6F727
:103E3000EDF8BDF814003044007900F0010008905E
:103E4000BDF81400304480790027C0F34200EB1F16
:103E5000079012E0A4F86A8609B0BDE8F08F3844F4
:103E60003044C079DDE90721F5F7E4FBBDF8141013
:103E700039443144C8717F1CBFB2BDF814009F4261
:103E8000EDDB3044C07984F8A4B74146C4F8A88675
:103E900084F8A686069A82F87684C2F8788494F824
:103EA000A627032A03D094F8A627012A02D1A34B00
:103EB000C3F888B2ADF80C1012287DD00CDCA0F14C
:103EC0000B00072816D2DFE810F0D10A330B6C0B79
:103ED000660B780D20002C0CA2286FD006DC14286D
:103EE0006DD015286CD0A12804D12EE3A32868D06A
:103EF000A42867D00020BDF814200244B154401C0F
:103F000080B20528F7D301F042BE88464046F3E16F
:103F1000BDF80000574600EB400101EB00100AEB32
:103F2000001000F5805090F85A0D07287DD2DFE888
:103F300000F07C040404047CA60040468BE0BDF83D
:103F40001400BDF80C1008443044007AA8B30128CE
:103F500002D0022877D113E0BDF8000000EB400149
:103F600001EB0010BDF8041007EB001000EB01108E
:103F700041F686510844017821F00401017062E0A5
:103F8000BDF8000000EB400101EB0010BDF804108B
:103F900007EB001000EB011041F686510844017850
:103FA00021F008010170BDF8000000EB400202EBB7
:103FB000001007EB001006E0FEE344E0FDE3FDE344
:103FC000FDE3FDE3FDE3BDF8042000EB021000F586
:103FD0008050C0F8888DBDF800100220F5F7BEFBB8
:103FE00000204246BDF8001001EB011303EB012154
:103FF00007EBC103BDF8041001EB011103EBC10194
:10400000014401F5005181F85B22401C80B2142864
:10401000E8D30020BDF8001001EB011303EB0121F0
:1040200007EBC103BDF8041000E062E101EB0111F0
:1040300003EBC101014401F5005181F87722401CD6
:1040400080B20A28E6D3BDF80C00401CADF80C0085
:10405000BDF80400401CADF80400BDF8000000EB02
:10406000400101EB001007EB001000F5805090F8C4
:104070005B0DBDF8041088423FF661AF39E1C446DC
:10408000ADF8048024E1BDF81400BDF80C1008441C
:104090003044007A042805D005DC58B101284FD0FF
:1040A00002287DD132E108287BD010287AD0202840
:1040B00076D1E7E1BDF8000000EB001101EB002034
:1040C00007EBC001BDF8040000EB001001EBC000DD
:1040D00000F5005090F89202102824D1BDF800009D
:1040E00000EB001101EB002007EBC001BDF804005C
:1040F00000EB001001EBC00000F5005080F892C208
:10410000BDF80000F32100EB001202EB002007EBEA
:10411000C002BDF8040000EB001002EBC00000F587
:10412000005080F82112BDF80C00401CC9E00000CE
:10413000A422002034740020180200200000404215
:10414000BDF80000F22100EB001202EB002007EBAB
:10415000C002BDF8040000EB001002EBC00000F547
:10416000005080F82112BDF8000000EB400101EB87
:104170000010BDF8041007EB001000EB011041F631
:1041800086510844017821F004010170BDF8140043
:10419000BDF80C1008443044017ABDF8000002E07C
:1041A00091E0B3E0F2E000EB001202EB002007EB3D
:1041B000C002BDF8040000EB001002EBC00000F5E7
:1041C000005080F892120020BDF81410BDF80C20A9
:1041D0001144014431444A7ABDF8001001EB011347
:1041E00003EB012107EBC103BDF8041001EB011142
:1041F00003EBC101014401F5005181F86522401C27
:1042000080B20F28E0D30020BDF81410BDF80C20B8
:104210001144014431440A7EBDF8001001EB011342
:1042200003EB012107EBC103BDF8041001EB011101
:1042300003EBC101014401F5005181F87722401CD4
:1042400080B20A28E0D3BDF81400BDF80C10084471
:10425000304490F82210BDF8000000EB001202EB91
:10426000002007EBC002BDF8040000EB001002EBD9
:10427000C00000F5005080F88C120020BDF814102A
:10428000BDF80C2011440144314491F82320BDF8BD
:10429000001001EB011303EB012107EBC103BDF893
:1042A000041001EB011103EBC101014401F50051C0
:1042B00081F88D22401C80B20528DFD3BDF80C00A8
:1042C0002030ADF80C00BDF80400401CADF804002F
:1042D000BDF8000000EB400101EB001007EB0010FF
:1042E00000F5805090F85B0DBDF8041088423FF651
:1042F000CAAEBDF80000401CADF8000094F8240BD5
:10430000BDF8001088423FF603AEFCE5BDF80000A2
:10431000F22100EB001202EB002007EBC002BDF817
:10432000040000EB001002EBC00000F5005080F824
:104330002112BDF8000000EB400101EB0010BDF8B8
:10434000041007EB001000EB011041F68651084401
:10435000017821F004010170BDF81400BDF80C10C3
:1043600008443044017ABDF8000000EB001202EB73
:10437000002007EBC002BDF8040000EB001002EBC8
:10438000C00000F5005080F89212CCE6BDF80000A5
:10439000F32100EB001202EB002007EBC002BDF896
:1043A000040000EB001002EBC00000F5005080F8A4
:1043B0002112BDF8000000EB400101EB0010BDF838
:1043C000041007EB001000EB011041F68651084481
:1043D000017821F004010170BDF81400BDF80C1043
:1043E00008443044017ABDF8000000EB001202EBF3
:1043F000002007EBC002BDF8040000EB001002EB48
:10440000C00000F5005080F89212BDF81400BDF80D
:104410000C1008443044417ABDF8000000EB001253
:1044200002EB002007EBC002BDF8040000EB001017
:1044300002EBC00000F5005080F88C120020BDF89F
:104440001410BDF80C201144014431448A7ABDF89F
:10445000001001EB011303EB012107EBC103BDF8D1
:10446000041001EB011103EBC101014401F50051FE
:1044700081F88D22401C80B20528E0D3BDF80C00E5
:10448000C01D1EE7BDF80000F22100EB001202EB98
:10449000002007EBC002BDF8040000EB001002EBA7
:1044A000C00000F5005080F82112BDF8000000EBBC
:1044B000400101EB0010BDF8041007EB001000EB09
:1044C000011041F686510844017821F00401017081
:1044D000BDF81400BDF80C1008443044017ABDF852
:1044E000000000EB001202EB002007EBC002BDF859
:1044F000040000EB001002EBC00000F5005080F853
:1045000092120020BDF81410BDF80C201144014493
:1045100031444A7ABDF8001001EB011303EB01218D
:1045200007EBC103BDF8041001EB011103EBC1015E
:10453000014401F5005181F88D22401C80B204280D
:10454000E0D3BDF80C00401DBBE6A81E0D2290FB79
:10455000F2F0C0B288460790404609E2ADF8048008
:104560005746E1E1BDF8000000EB400101EB00100F
:10457000BDF8041007EB001000EB011000F58050AF
:1045800090F8860D80077DD409EB890101EBC90005
:10459000BDF8141008443044007A0021FDF720FBD8
:1045A000BDF8002002EB420303EB0212BDF8043019
:1045B00007EB021202EB031202F5805292F8842DEF
:1045C00088EA010342401A435CD1BDF8000000EBC9
:1045D000001101EB002007EBC001BDF8040000EB67
:1045E000001001EBC00000F5005090F859020128BE
:1045F0007ED1BDF814003044417ABDF8000000EBD4
:10460000001202EB002007EBC002BDF8040000EB33
:10461000001002EBC00000F5005080F82212BDF837
:1046200014003044407BBDF814103144897A40EACC
:104630000161BDF814003044C07ABDF814200004B4
:104640003244127B40EA02200143BDF8000000EB37
:10465000001202EB002007EBC002BDF8040000EBE3
:10466000001002EBC00000F50050C0F82412BDF8A5
:1046700014003044007DBDF814103144497C40EAF8
:10468000016000E04BE1BDF814103144897CBDF8B5
:10469000142009043244D27C41EA02210843BDF8C7
:1046A000001001EB410202EB0111BDF8042007EB01
:1046B000011101EB021101F58051C1F8880DBDF81F
:1046C000000000EB400101EB0010BDF8041007EB07
:1046D000001000EB011041F686510844017841F0CA
:1046E00020010170BDF800100220F5F737F800E056
:1046F00089E0BDF8000000EB400101EB0010BDF8BF
:10470000041007EB001000EB011000F5805090F84A
:10471000841DBDF8000000EB001202EB002007EB47
:10472000C00000F5005080F81512BDF8000000EB45
:10473000400101EB001007EB001000F5805090F8ED
:104740005A0D012806D0022860D003285ED0072821
:1047500059D1C8E0BDF8000000EB001101EB0020CA
:1047600007EBC001BDF8040000EB001001EBC00036
:1047700000F5005090F8220210B1012843D143E027
:10478000BDF8000000EB400101EB001007EB00104A
:1047900000F5805090F8600D0028BDF8000000EB97
:1047A000001101EB002007EBC001BDF8040000EB95
:1047B000001001EBC00005E0EEE3DCE1EDE3EDE32A
:1047C00025E30AE100F50050D0F8240203D0B0F14F
:1047D000104F03D104E0B0F5100F01D0B52100E077
:1047E000C321BDF8000000EB001202EB002007EB34
:1047F000C002BDF8040000EB001002EBC00000F5A1
:10480000005080F8211283E0B921EAE7BDF80000EA
:1048100000EB001101EB002007EBC001BDF8040024
:1048200000EB001001EBC00000F5005090F81C12E6
:10483000BDF8000000EB001202EB002007EBC00007
:1048400000F5005090F81802814261D1BDF81400C3
:104850003044807BBDF8141000043144C97B40EA29
:104860000121BDF814003044007C0143BDF8000074
:1048700000EB001202EB002007EBC002BDF80400C1
:1048800000EB001002EBC00000F50050C0F8501221
:10489000BDF814003044417ABDF8000000EB00126E
:1048A00002EB002007EBC002BDF8040000EB001093
:1048B00002EBC00000F5005080F82212BDF80000A5
:1048C000A42100EB001202EB002007EBC002BDF8B0
:1048D000040000EB001002EBC00000F5005080F86F
:1048E0001E12A3217DE7BDF8000000EB001101EBD3
:1048F000002007EBC001BDF8040000EB001001EB45
:10490000C00000F5005090F82202D8B301285DD015
:1049100009F10100079900F0FF09894515D2BDF89A
:104920000400401CADF80400BDF8000000EB40019D
:1049300001EB001007EB001000F5805090F85B0DC4
:10494000BDF8041088423FF60DAEBDF8000000EB44
:10495000400101EB001107EB011000F5805090F8C9
:104960005B0DBDF8041088427ED8BDF80000401CE5
:10497000ADF8000094F8240BBDF8001088423FF613
:10498000EDADC2E4FFE7BDF8000000EB400101EB34
:10499000001007EB001000F5805090F8600D002823
:1049A000BDF8000000EB001101EB002007EBC00197
:1049B000BDF8040000EB001001EBC00000F5005052
:1049C000D0F8240204D0B0F1104F04D0594608E7C3
:1049D000B0F5100FFAD1052103E78846404649E0BB
:1049E000ADF80480574620E0BDF814003044007A4A
:1049F0000021FDF7F5F8BDF8002002EB420303EBC0
:104A00000212BDF8043007EB021202EB031202F5AA
:104A1000805292F8842D88EA010342401A4332D032
:104A2000BDF80400401CADF80400BDF8000000EB28
:104A3000400101EB001007EB001000F5805090F8EA
:104A40005B0DBDF804108842CED8BDF8000000EB25
:104A5000400101EB001107EB011000F5805090F8C8
:104A60005B0DBDF8041000E04AE1884289D8BDF82A
:104A70000000401CADF8000094F8240BBDF80010B5
:104A80008842ADD841E4BDF80000BDF8042000EB39
:104A9000400101EB0010394607EB001000EB02105B
:104AA00000F5805090F8842DBDF8000000EB001355
:104AB00003EB002007EBC00000F5005080F8152242
:104AC000BDF8000000EB400202EB001007EB001005
:104AD00000F5805090F85A0D012838D0022801D0F6
:104AE0000328B2D1BDF8000000EB001202EB002059
:104AF00001EBC002BDF8040000EB001002EBC000A7
:104B000000F5005090F81C22BDF8000000EB0013E7
:104B100003EB002001EBC00000F5005090F81802F4
:104B2000824292D1BDF80000AA2200EB001303EBF1
:104B3000002001EBC003BDF8040000EB001003EB04
:104B4000C00000F5005080F81E22A32200E0CA2217
:104B5000BDF8000000EB001303EB002007EBC001E1
:104B6000BDF8040000EB001001EBC00000F50050A0
:104B700080F8212269E78846404646E0ADF8048087
:104B800020E0BDF814003044007A0021FDF728F839
:104B9000BDF8002002EB420303EB02130AEB031201
:104BA000BDF8043002EB031202F5805292F8842D16
:104BB00088EA010342401A4330D0BDF80400401C8B
:104BC000ADF80400BDF8000000EB400101EB00115E
:104BD0000AEB011000F5805090F85B0DBDF8041051
:104BE0008842CED8BDF8000000EB400101EB001177
:104BF0000AEB011000F5805090F85B0DBDF8041031
:104C000088427DD8BDF80000401CADF8000094F843
:104C1000240BBDF800108842B0D8B2E6BDF8000001
:104C2000BDF8042000EB400101EB001051460AEBF7
:104C3000001000EB021000F5805090F8842DBDF8B4
:104C4000000000EB001303EB00200AEBC00000F5AE
:104C5000005080F81522BDF814003044407ABDF8A9
:104C6000142000043244927A40EA0222BDF8140073
:104C70003044C07A0243BDF8000000EB001303EBA0
:104C8000002001EBC003BDF8040000EB001003EBB3
:104C9000C00000F50050C0F85022BDF8000000EB45
:104CA000400202EB001001EB001000F5805090F87C
:104CB0005A0D01284CD0022801D0032892D1BDF80A
:104CC000000000EB001202EB002001EBC002BDF877
:104CD000040000EB001002EBC00000F5005090F85B
:104CE0001C22BDF8000000EB001303EB002001EBD9
:104CF000C00000F5005090F818028242DED100E0BA
:104D0000EEE2BDF80000A52200EB001303EB00204B
:104D100001EBC003BDF8040000EB001003EBC00082
:104D200000F5005080F81E22BDF80000A32200EB21
:104D3000001303EB00200AEBC001BDF8040000EBF8
:104D4000001001EBC00000F5005080F8212249E777
:104D5000BDF8000000EB001202EB002001EBC002E6
:104D6000BDF8040000EB001002EBC00000F500509D
:104D700090F81C22BDF8000000EB001303EB0020AC
:104D800001EBC00000F5005090F818028242DED11D
:104D9000BDF80000B22200EB001303EB002001EB92
:104DA000C003BDF8040000EB001003EBC00000F5E9
:104DB000005080F81E22BDF80000E52200EB001331
:104DC00003EB002001EBC003BDF8040000EB001072
:104DD00003EBC00000F5005080F82122002FB6D16F
:104DE000BDF804000128B2D1BDF8000000EB0012AC
:104DF00002EB00200AEBC001BDF8040000EB00103C
:104E000001EBC00000F50050D0F85002EAE6BDF812
:104E100014003044007A0528BDF814003044007AAC
:104E20007ED2401EADF8000000205746BDF800209D
:104E300002EB420303EB021207EB021202EB001239
:104E400002F5805282F8841DBDF8002002EB420377
:104E500003EB021207EB021202EB001202F5805282
:104E600082F8851DBDF8002002EB420303EB02121D
:104E700007EB021202EB001202F5805282F88C1D41
:104E8000401C80B21028D1D3BDF814003044807B80
:104E900088460021FCF7A4FE08437CD0BDF814002E
:104EA0003044407ABDF8141000043144897A40EA55
:104EB0000120BDF814103144C97A0843C117FCF72A
:104EC0008FFEBDF8001001EB410202EB011107EB70
:104ED000011101F58051C1F8540DBDF814003044A2
:104EE000007B0021FCF77CFEBDF8001001EB4102C5
:104EF00002EB011107EB011101F5805181F8580D0A
:104F0000BDF814003044407B0021FCF769FEBDF879
:104F1000001001EB410202EB011107EB011100E06F
:104F2000DFE101F5805181F8590DBDF814003044DE
:104F3000807B0021FCF754FEBDF8001001EB41021C
:104F400002EB011107EB011101F5805181F85A0DB7
:104F5000BDF814003044C07B0021FCF741FEBDF8D1
:104F6000001001EB410202EB011107EB011101F509
:104F7000805181F85B0DBDF814003044007C0021A5
:104F8000FCF72EFEBDF8001001EB410202EB01110F
:104F900007EB011103E0E4E0CCE3FCE3FCE301F503
:104FA0008051C1F85C0DBDF814003044407C0021F4
:104FB000FCF716FEBDF8001001EB410202EB0111F7
:104FC00007EB011101F5805181F8600DBDF800007B
:104FD00000EB400101EB001007EB001000F58050E2
:104FE00090F85A0D062840465AD0A7E0BDF81400A4
:104FF000BDF8041008443044807C0021FCF7F0FD2B
:10500000BDF804200321B2FBF1F2BDF8001001EB62
:10501000410303EB011107EB011101EB021101F553
:10502000805181F8840DBDF81400BDF804100844C7
:105030003044C07C0021FCF7D3FDBDF804200321DF
:10504000B2FBF1F2BDF8001001EB410303EB0111DB
:1050500007EB011101EB021101F5805181F8850D7B
:10506000BDF81400BDF8041008443044007D002150
:10507000FCF7B6FDBDF804200321B2FBF1F2BDF848
:10508000001001EB410303EB011107EB011101EBF0
:10509000021101F5805181F88C0DBDF80400C01C8F
:1050A000ADF80400BDF8000000EB400101EB00107A
:1050B00007EB001000F5805090F85B0DBDF8041070
:1050C00000EB4000884291D84BE0BDF81400BDF8D9
:1050D000041008443044807C0021FCF781FDBDF8B9
:1050E000001001EB410202EB0111BDF8042007EBB7
:1050F0000111520801EB021101F5805181F8840D74
:10510000BDF81400BDF8041008443044C07C0021F0
:10511000FCF766FDBDF8001001EB410202EB011146
:10512000BDF8042007EB0111520801EB021101F553
:10513000805181F8850DBDF80400801CADF8040095
:10514000BDF8000000EB400101EB001007EB001080
:1051500000F5805090F85B0DBDF80410B1EB400FE6
:10516000B3D3BDF80400123085427DD9BDF80000EC
:1051700000EB400101EB001007EB001000F5805040
:1051800090F85A0D012837D0BDF8000000EB40011F
:1051900001EB001007EB001000F5805090F85A0D5D
:1051A000032829D0BDF8000000EB400101EB0010FE
:1051B00007EB001000F5805090F85A0D02281BD024
:1051C000BDF8000000EB400101EB001007EB001000
:1051D00000F5805090F85A0D07280DD0BDF800005A
:1051E00000EB400101EB001007EB001000F58050D0
:1051F00090F85A0D04285FD1BDF8140028443044BB
:1052000010F8020C00F00F00042814D2BDF80000C2
:1052100000EB400101EB001007EB001141F670506C
:105220000844BDF814102944314411F8022C0178C7
:1052300062F301010170BDF814002844304410F8F5
:10524000010C0421B1EB101F17D9BDF8000000EBD1
:10525000400101EB001007EB001141F670500844CB
:10526000BDF81410294400E026E0314411F8011C77
:105270000A09017862F383010170BDF81400284423
:10528000304410F8010C00F00F00042814D2BDF8CF
:10529000000000EB400101EB001007EB001141F6AC
:1052A00070500844BDF814102944314411F8011C11
:1052B000027861F305120270BDF800100220F4F7C5
:1052C0004DFABDF80000C0B2FDF75CF9BDF8000072
:1052D00000EB400007EB800000F5805080F8B1B68D
:1052E0001EE20528FCD1BDF814000930ADF80C0011
:1052F000BDF80C00305C84F8C80BBDF80C00401CF5
:10530000ADF80C00ADF80010A2E0BDF80C00305C68
:105310000021FCF765FCBDF80010574601EB410188
:105320000AEB011101F5805181F8D30BBDF80C0097
:10533000401CADF80C00BDF80C00305C0021FCF7FF
:105340004FFCBDF8001001EB410107EB011101F525
:10535000805181F8D20BBDF80C00401CADF80C0058
:10536000BDF80C00305CBDF80C10000431444978E5
:1053700040EA0120BDF80C10314489780843C11778
:10538000FCF72EFCBDF8001001EB410107EB011109
:1053900001F58051C1F8CC0BBDF80C00C01CADF874
:1053A0000C00BDF80C00305C0021FCF719FCBDF8C6
:1053B000001001EB410107EB011101F5805181F86B
:1053C000D00BBDF80C00401CADF80C00BDF80C0073
:1053D000305C0021FCF704FCBDF8001001EB41013A
:1053E00007EB011101F5805181F8D10BBDF80C00DC
:1053F000401CADF80C00BDF80C00305C0021FCF73F
:10540000EFFBBDF8001001EB410107EB011101F5C5
:105410008051C1F8D40BBDF80C00401CADF80C0055
:10542000BDF80C0030444078BDF80C10715C40EAC7
:105430000120BDF80C10891CADF80C10BDF80C1043
:105440000844ADF80C00BDF80000401CADF80000A9
:1054500094F8C80BBDF8001088423FF656AF002103
:105460000A20F4F77BF9FEF735F890E3BDF8140055
:105470003044007A84F8ED03BDF814003044407ADB
:1054800084F8EC03BDF814003044807A84F8EB0310
:10549000BDF814003044C07A84F8EA03BDF8140063
:1054A0003044007B84F8E903BDF814003044407BAD
:1054B00084F8E80304F57A74F4F772F8F4F734F832
:1054C0002078A4F57A74FF2829D1F3F7E3FFBDF81B
:1054D00014003044007A84F8ED03BDF81400304421
:1054E000407A84F8EC03BDF814003044807A84F8E4
:1054F000EB03BDF814003044C07A84F8EA03BDF829
:1055000014003044007B84F8E903BDF814003044F3
:10551000407B84F8E803F4F743F8F4F705F8DAF889
:10552000580008B10F2000E00E2084F8A8072EE3F1
:10553000102084F8A807BDF814003044007A84F8DD
:10554000ED03BDF814003044407A84F8EC03BDF854
:1055500014003044807A84F8EB03BDF81400304422
:10556000C07A84F8EA03BDF814003044007B84F864
:10557000E903BDF814003044407B84F8E80304F5E7
:105580007A74F4F70DF802F035FCA060A068A0680A
:10559000A4F57A74FBE20E2084F8A80784F8E111E0
:1055A000F5E2ADF8001057463EE0ADF8041016E005
:1055B000BDF8000000EB400202EB0010BDF8042033
:1055C00007EB001000EB021000F5805090F8860DFC
:1055D000C00714D1BDF80400401CADF80400BDF8AC
:1055E000000000EB400202EB001007EB001000F59A
:1055F000805090F85B0DBDF804209042D8D8BDF8DB
:10560000000000EB400202EB001007EB001000F579
:10561000805090F85B0DBDF80420904208D8BDF88A
:105620000000401CADF80000BDF800000428BCD309
:10563000BDF8000004286AD3FE4A88465170FE492E
:10564000C1F888B2C1F888B294F8E501002870D09A
:105650000D2084F8A807BDF814003044407ABDF846
:1056600014103144097A40EA0120ADF80800BDF871
:1056700014003044C07ABDF814103144897A40EAED
:105680000120508000204FF4007CBDF8141001442C
:105690003144097B3B1803F5805383F8E611401C25
:1056A00080B26045F1D3E348408800F2FF3081B218
:1056B0000120F3F749FA00283BD084F8E181DD4866
:1056C000418864225143BDF80820B1FBF2F184F80F
:1056D000E01187F807B04188491C41804088BDF837
:1056E0000810884225D994F8DC0140F0010084F8C4
:1056F000DC0194F8DC0120F00600801C84F8DC0159
:10570000BDF80800A4F8DE01002101204DE11020C1
:1057100084F8A80794F8DC0140F0800084F8DC01EC
:1057200035E2BDF814003044007A84F8E10111201C
:10573000FBE699E0ADF80010574641E0ADF80410E3
:1057400016E0BDF8000000EB400202EB0010BDF8CF
:10575000042007EB001000EB021000F5805090F8D9
:10576000860DC00714D1BDF80400401CADF804003C
:10577000BDF8000000EB400202EB001007EB001048
:1057800000F5805090F85B0DBDF804209042D8D809
:10579000BDF8000001E030E186E100EB400202EBE1
:1057A000001007EB001000F5805090F85B0DBDF87D
:1057B0000420904208D8BDF80000401CADF800005D
:1057C000BDF800000428B9D3BDF800000428A7D311
:1057D000DFF860C288468CF801109749C1F888B29A
:1057E000C1F888B294F8E501F0B3122084F8A80754
:1057F000BDF814003044007A84F8E10194F8E10126
:10580000401EADF800000020BDF8141001443144E2
:105810004A7ABDF8001001EB410303EB011107EBDD
:105820000111014401F5805181F8622D401C80B2C4
:105830000A28E9D3BDF814003044007DBDF81410E7
:105840003144C97C40EA0120ADF80800BDF81400DD
:105850003044807DBDF814103144497D40EA012078
:10586000ACF80200002000E05AE04FF40071BDF8EF
:10587000142002443244D37D3A1802F5805282F853
:10588000E631401C80B28842F1D36A484088BDF8B6
:10589000001000EB8120401E81B20320F3F754F981
:1058A000F0B36448418864225143BDF80820B1FB3D
:1058B000F2F184F8E0113A4687F807B04188491CB4
:1058C00041804188BDF80830994243D9002041F613
:1058D0008D53BDF8001001EB410707EB011102EBFE
:1058E000011101EB001119440F7847F001070F7007
:1058F000401C80B21028ECD3BDF8000000EB400142
:1059000001EB001002EB001041F66C5108440378E3
:1059100043F001030370BDF8000000EB400300E01A
:1059200045E003EB001002EB00100844017821F081
:105930000601891C0170BDF80810BDF8000000EBDD
:10594000400303EB001002EB001000F58050A0F8BC
:105950006E1D27E04088012829D1002041F68D5393
:10596000BDF8001001EB410707EB011102EB01113B
:1059700001EB001119440F7827F001070F70401C4C
:1059800080B21028ECD3BDF8000000EB400101EB21
:10599000001002EB001041F66C510844017821F030
:1059A00001010170BDF800100220F3F7D7FE224973
:1059B000C1F88882C1F88882E9E0DAF858005746D1
:1059C0000A22B0FBF2F0BDF814203244127A904261
:1059D00012D1BDF814003044007A18B1B86D0A38FD
:1059E000B86503E0B965102084F8A80700210520F8
:1059F000F3F7B4FE87F807B0C9E00021202257462C
:105A0000002007EB411303EB000C8CF85B2F401CCC
:105A100080B22028F7D3491C89B21429F0D314216D
:105A200084F8A817BDF814003044007AADF80800D7
:105A300004E000001802002000004242BDF81400FB
:105A40003044407AADF81000BDF80800142801D9A0
:105A5000ADF80810BDF81000202801D9ADF81020CD
:105A6000002118E0002007EB411C0EE0BDF81020DB
:105A7000BDF8143001FB026203441A44927A0CEB25
:105A8000000383F85B2F401C80B2BDF810209042C9
:105A9000ECD3491C89B2BDF808008142E2D3002151
:105AA0000720F3F75BFE72E0152084F8A807BDF825
:105AB00014003044017A50468AF8201FBDF81410B3
:105AC0003144097BBDF814203244527A41EA026124
:105AD000BDF814203244927ABDF8143012043344D5
:105AE000DB7A42EA03221143C0F8251FBDF81410E7
:105AF0003144097CBDF814203244527B41EA0261F2
:105B0000BDF814203244927BBDF8143012043344A3
:105B1000DB7B42EA03221143C0F8211FBDF81410B9
:105B20003144497CBDF8142009043244927C41EA96
:105B30000221BDF814203244D27C1143C0F8291F41
:105B4000BDF814103144097D80F8461FBDF81410CB
:105B50003144497D80F8451FBDF814103144897DDA
:105B600080F8441FBDF814103144C97D80F8431FEC
:105B7000BDF814103144097E80F8421FBDF814109E
:105B80003144497E80F8411F022084F8DC0CB4F8CF
:105B90006A0600B300201AE000204146BDF8142038
:105BA0000244B154401C80B20528F7D3A4F86A1609
:105BB00009B0BDE8F08FBDF8141029440144314408
:105BC0008978BDF814200244B154401C80B2B4F866
:105BD0006A168142EFD8B4F86A0600287EF4C9A894
:105BE000E6E794F8A6074FF47A7730B101287CD025
:105BF00002287BD003287AD11CE294F8E206C0F395
:105C0000C3000E2873D2DFE800F0F90713F81F2B4A
:105C10002B374D799DA9F7E6F8A1F94806F0E6FB88
:105C2000002864D094F8E20620F078001030DCE020
:105C3000F4A1F34806F0DAFB0028F2D094F8E2066B
:105C400020F078001830D0E0EFA1ED4806F0CEFB50
:105C50000028E6D094F8E20620F078002830C4E06E
:105C6000E9A1E74806F0C2FB0028DAD094F8E20682
:105C700020F078003830B8E0E3A1E14806F0B6FB48
:105C80000028CED09AF80100182805D994F8E20629
:105C900020F078005030A8E094F8E20620F0780078
:105CA0004030A2E0D9A1D64806F0A0FB0028B8D029
:105CB00052464146531903F5805383F82B176D1C48
:105CC000ADB2142DF6D30021431833441D79531877
:105CD00003F5805383F83057491C89B20F29F3D359
:105CE00000210320F3F73AFD02E088E033E171E0A0
:105CF00094F8E20620F07800483004E2C5A1C048DC
:105D000006F074FB00288CD052464146531903F527
:105D1000805383F8E4166D1CADB2142DF6D3002128
:105D2000431833445D79531803F5805383F8E956DB
:105D3000491C89B20F29F3D394F8E20620F07800C9
:105D40005030E0E1B0A1AE4806F050FB00288CD006
:105D500094F8E20620F07800583046E094F8AA075C
:105D600050B194F8E20620F07800603084F8E20642
:105D7000C4F8808684F87EB6A8A1A14806F036FB58
:105D8000002827D0C4F8808684F87EB63044417954
:105D900000793039303841EA0010C117FBF720FF95
:105DA00084F8AA079FA1964806F020FB002811D08E
:105DB00031184A78302A06D34978305C3038303987
:105DC00041EA001001E0305C3038C117FBF708FFF2
:105DD00084F8AB07A8E18CA1894806F007FB0028EE
:105DE00009D094F8E20620F0780084F8E206C4F8BE
:105DF000808684F87EB697E188E131E12AE194F863
:105E0000E206C0F3C3000D284CD2DFE800F008170B
:105E1000232D3861078189F64B8F9A003CE77AA1E0
:105E2000774806F0E3FAE8B3C4F8808684F87EB6D3
:105E300094F8E20620F07800083064E17AA197E057
:105E4000C4F8808684F87EB694F8E20620F07800E4
:105E5000103058E16CA16A4806F0C8FA10B3C4F8D3
:105E6000808684F87EB6B0E070A1654806F0BEFA80
:105E7000C0B194F8E20620F078002030B5E765A1C3
:105E80005F4806F0B3FA68B153464246591901F526
:105E9000805181F8E4266D1CADB2142DF6D300219B
:105EA000451800E03BE035446D795F1807F58057F1
:105EB00087F8E956491C89B20F29F1D3C4F8802626
:105EC00084F87EB694F8E20620F0780028301AE1D3
:105ED00052A14B4806F08AFA08B394F8AA1731B1D8
:105EE00094F8E21621F07801303184F8E216C4F813
:105EF000808684F87EB63044417900793039303874
:105F000041EA0010C117FBF76BFE84F8AA070BE10A
:105F10003DA13B4806F06AFA00287FF47FAF03E119
:105F200094F8E20620F0780048305EE736A1344865
:105F300006F05CFA10B394F8E20620F078006030C6
:105F400053E731A12E4806F051FAB8B194F8E206B1
:105F500020F07800D7E094F8E206C0F3C3000528EB
:105F60000CD2DFE800F003040CD338005CE726A174
:105F7000234806F03BFA00287FF462AFD4E0C4F86F
:105F8000808684F87EB6B07971793038303940EA4D
:105F90000110C117FBF724FE84F8AA0721A11848B5
:105FA00006F024FA88B131184A78302A06D34978A5
:105FB000305C3038303941EA001001E0305C303874
:105FC000C117FBF70DFE84F8AB0794F8E20620F04A
:105FD0007800183097E094F8E20620F0800084F80A
:105FE000E20694F8E20620F0780084F8E2060699CA
:105FF00081F87684C1F8788496E08DE06100000035
:10600000347400206F6B00004F4B0000494D454930
:106010003A00000049434349443A00004353513A8F
:10602000000000002C000000220000005245414406
:106030005900000094F8E206C0F3C300092873D2A7
:10604000DFE800F00807060E051142526400FBE588
:10605000EEE5E1E594F8E20620F078000830C4E6C9
:10606000AFF25C0101E735A1364806F0BFF950B345
:10607000C4F8808684F87EB65746411931440A79BF
:10608000791901F5805181F8AC276D1CADB2142D42
:10609000F3D32BA12C4806F0A9F958B100214246B0
:1060A0000B183B4403F5805383F8AB27491C89B296
:1060B0000229F5D394F8E20620F07800303084F815
:1060C000E20687F807B02FE0AFF2C4011D4806F0E2
:1060D0008DF948B3C4F8808684F87EB694F8E20659
:1060E00020F0780038300EE0AFF2E401154806F0F9
:1060F0007DF9C8B1C4F8808684F87EB694F8E206CB
:1061000020F07800403084F8E2060DE0AFF208118C
:106110000C4806F06BF938B194F8E20640F08000C4
:1061200084F8E206C4F884764146A4F86A86002022
:106130003154401C80B26428FAD339E544484350B6
:106140002C00000034740020502A00202DE9F74F65
:1061500086B00020019081460090FE4D0021295418
:10616000401C80B26428F8D3FB4890F87614A0F560
:10617000405431B394F8A51719B3002180F8761470
:1061800094F8E20620F0800084F8E20694F8A6076E
:1061900028B101280ED0022806D0032811D194F886
:1061A000E20620F078000AE094F8E20620F0780099
:1061B000203004E094F8E20620F07800583084F8AB
:1061C000E20694F8E206E54E00067CD594F8A606B1
:1061D000012879D194F8A407012875D10020DFF8AF
:1061E0008083824600EB400101EB0A1108EB0110AD
:1061F000039000F58050002702906AE0039800EBBE
:10620000071505F5805595F8860D00065FD595F8BC
:10621000860D40F0040085F8860D95F8860D000780
:1062200055D595F8860D20F0080085F8860D0020DC
:10623000C1F839000AEB0A1101EB0A2108EBC10091
:1062400007EB071100EBC10BC54842F23D21594451
:106250001022293005F68455F1F7F7FF0BF50850A9
:10626000414650F8352F41F81D2F40684860297885
:1062700088F81C1042F2502050F80B10C8F8251076
:10628000B84940468A6E40F83D2FB1F86C108180C5
:106290006968C8F84310D8F8580081B20220F2F7B4
:1062A00053FC00210620F3F759FAD8F85810B8F833
:1062B0001A00814204D2D8F85810491CC8F8581066
:1062C0000021052001E0FCE326E0F3F747FA7F1CFC
:1062D000BFB20298414690F85B0DB8428ED8514645
:1062E0000220F3F73BFA0AF1010080B2824604284B
:1062F000FFF478AF94F8A607032803D094F8A60714
:10630000012803D198490020C1F88802002084F8B0
:10631000A4070B2084F8A8078E4F00203A3F38705E
:1063200000980DE001F066FDC4F8F003D4F8F00326
:10633000C0F300400190D4F8F003C0F34200009095
:106340000028EFD094F8A607022811D194F8A507E9
:1063500070B1804855214FF007090170FD2141704F
:10636000AA2181700021C170017161224271817185
:106370007849F52201F809200020D4F8F013C0F183
:106380000302D200D140734A09EB00031A44D170D2
:10639000401C80B20428F0D394F8A50720B17248BD
:1063A000D0F80802B0B906E06A4908984944C871B3
:1063B00009F1080532E06A48007858B194F8A60758
:1063C000032807D094F8A607012803D0012084F8F9
:1063D000A606FDE3624A5F490020131803F58053C7
:1063E00093F82B5709EB00030B44DD71401C80B27E
:1063F0001428F2D30020131803F5805393F8EC57B8
:1064000009EB00030B44DD76401C80B20A28F2D36E
:106410004944089881F8250009F12605002DD8D0B7
:10642000089884F8670608981021FF2212287DD06A
:1064300009DCA0F10B0007281BD2DFE800F01A1AD4
:10644000FD0DFC1BFB00A22813DA4FF059021428A3
:1064500001D015280DD1D4E384F8A817434A3D494B
:1064600000202F18135CCB55401C80B20A28F8D3AB
:106470000A35CBE394F8DC01C0077DD0012080F31E
:106480001388BFF34F8F3A4801683A4A01F4E0613C
:1064900011430160BFF34F8FFEE700EB400101EBBA
:1064A0000B102F4901EB0010039000F5805080463F
:1064B00090F85A0D032816D098F85A0D012812D0DA
:1064C00098F85A0D02280ED098F85A0D04280AD0D0
:1064D00098F85A0D8A4605287ED098F85A0D0A4633
:1064E00006287AD067E11B4A01205055ED1CA8B25E
:1064F000022304901354401C80B21D231354401CEB
:1065000085B20020B5E0039800EB0A1202F5805234
:1065100092F8840D0F4948556D1C92F8863DA8B23B
:106520000B54401C85B292F8860D00E057E24007FC
:1065300007D492F8860D000703D492F8860D8007E1
:106540007BD50020D2F8883DC0F10307FF00FB4057
:10655000471912E052020020A4520020BC640240FD
:10656000A41200202426002000004042FCC40108A0
:106570000CED00E00400FA0520E1CB55401C80B290
:106580000428DFD32D1DABB20BEB0B1505EB0B2253
:106590000CEBC2050AEB0A1205EBC20202920020C4
:1065A00002F50052D2F83552C0F10307FF00FD405A
:1065B000C718CD55401C80B20428F3D31B1D9BB2D5
:1065C0000020D2F83952C0F10307FF00FD40C71880
:1065D000CD55401C80B201E05DE091E00428F0D38D
:1065E0001B1D9BB20020D2F85052C0F10207FF00E1
:1065F000FD40C718CD55401C80B20328F3D3DB1CE7
:106600009FB20025029901F50050D0F83D0201F536
:106610000051D1F84112C5F10502D200F1F703FE95
:10662000FE49EA1988546D1CADB2062DEAD3BF1D90
:10663000BFB203E078E110E256E117E000250299CD
:1066400001F50050D0F8450201F50051D1F849128A
:10665000C5F10502D200F1F7E6FDF049EA198854C8
:106660006D1CADB2062DEAD3BF1DBDB20AF101000B
:1066700080B2DFF8ACC398F85B1D824651453FF607
:1066800042AF0498E549049A281A1144030A01F814
:10669000023D48708FE0E14B02205855ED1CADB231
:1066A000A846002120E0481C074658550AEB010285
:1066B00002F580526D1C92F88525A8B21A54401C30
:1066C00082B200200AEB01110D1805F5805595F8EE
:1066D000915500EB020C03F80C50401C80B21028BE
:1066E000F2D3103295B2B9B294F884058842DAD860
:1066F00003EB0800002100F8021DA5EB080159E09A
:10670000C64F03207855ED1CA8B2022182463954A9
:10671000401C80B20E213954401C85B2002196469F
:106720003DE0039800EB0110A0F51F7000F500504C
:1067300002787A556D1CAAB28578BD54521C8078B7
:1067400095B2400729D50BEB0B1C0CEB0B220EEB83
:10675000C20201EB0113002002EBC302131803F580
:10676000005393F85B3200EB050C07F80C30401C2B
:1067700080B20A28F2D30A35ABB20020151805F50D
:10678000005595F8745200EB030C07F80C50401CB0
:1067900080B20228F2D39B1C9DB2491C89B298F8A2
:1067A0005B0D8842BDD807EB0A00002100F8021DEE
:1067B000A5EB0A0141700BF1010080B294F8241B93
:1067C000834659453FF669AE94F8C80B00287DD042
:1067D000AD1CADB2AB46002277E0914B02EB42001C
:1067E00003EB001101F5805191F8D20B04280FD171
:1067F0008A4F78556D1CA8B201253D54401C9D1848
:1068000005F5805580B295F8315D3D54401C85B248
:1068100091F8D20B9A4602280CD002EB420000EB12
:10682000021003EB001000F5805090F85A0D052877
:1068300037D048E0794F022078556D1C94F88415C4
:10684000A8B23954401C80B212213954401C85B280
:10685000002121E0481C804678550AEB010303F52E
:1068600080536D1C93F88535A8B23B54401C83B20D
:1068700000200AEB0115291801F5805191F89115B6
:1068800000EB030C07F80C10401C80B21028F2D368
:1068900010339DB21FFA88F194F884058842D9D844
:1068A00011E05E49052048556D1CA8B201250D5424
:1068B0000AEB020303F58053401C93F8313D80B28C
:1068C0000B54401C85B2521C92B200E09EE194F839
:1068D000C80B904281D851480021584400F8021D4D
:1068E000A5EB0B01417091E17878401C78707878C5
:1068F000052803D294F8DC01C00706D084F8A81755
:1069000094F8DC01C00704D005E00D2084F8A80746
:1069100001E084F8E0217888010A404841557988EF
:1069200028444170AD1C71E184F8A81794F8E10186
:10693000DFF8E88008F805000022DFF8E4C06D1CED
:106940003EE094F8E10102EB021700EB001101EBCD
:1069500000200CEBC00000EBC70000F5805090F861
:106960000C0A01282AD194F8E10100EB400101EB67
:1069700000100CEB001000EB021000F5805090F8B6
:10698000540C08F805006D1CABB2002094F8E1111E
:1069900001EB011505EB01210CEBC10101EBC70176
:1069A000014401F5805191F80D1A1D1808F80510E1
:1069B000401C80B20A28E9D30A339DB2521C92B21D
:1069C00094F8E10100EB400101EB00100CEB00102A
:1069D00000F5805090F82B0C9042B2D816E17878F0
:1069E000401C7870787805280ED294F8E10100EB0D
:1069F000400303EB00130A4800EB031000F580503E
:106A000090F83C0CC00716D084F8A81794F8E10160
:106A100000EB400101EB0011014803E052020020AD
:106A2000A412002000EB011000F5805090F83C0CFF
:106A3000C00704D005E0122084F8A80701E084F81C
:106A4000E02194F8E111FE48415579882844090A6B
:106A5000417079888170ED1CD8E0FA480121C1713C
:106A6000816D0A22B1FBF2F2F5494A55806D6D1C29
:106A70000A2801D90A2001E0F248806D0022029222
:106A80008346485522206D1C485517466D1CB0E0C2
:106A9000DFF8B083D8F8580038B1D8F85800C01BD8
:106AA000401E81B20220F1F7E3FF98F81C00DFF8E6
:106AB00090C30CF805006D1CA9B20020D8F81D2069
:106AC00000E0EEE0C0F10303DB00DA4043180CF80D
:106AD0000320401C80B20428F0D3091D89B2002095
:106AE000D8F82120C0F10303DB00DA4043180CF88A
:106AF0000320401C80B20428F2D3091D89B2002073
:106B00004346D3F82520C0F10205ED00EA404518C0
:106B10000CF80520401C80B20328F2D3C91C1FFAD0
:106B200081F800259A46514651F8290F4968C5F168
:106B30000502D200F1F777FBC14905EB0802885442
:106B40006D1CADB2062DEED308F106001FFA80F8D9
:106B500000258A46BB4951F8310F4968C5F1050245
:106B6000D200F1F760FB05EB08020AF802006D1C89
:106B7000ADB2062DEED3B34908F1060080B291F80C
:106B8000423052460AF80030401C91F8413080B241
:106B90000AF80030401C91F8403080B20AF800300A
:106BA000401C91F83F3080B20AF80030401C91F848
:106BB0003E3080B21354401C91F83D3080B21354E3
:106BC000401C83B20020D1F84350C0F1030C00E018
:106BD000F6E04FEACC0C25FA0CF500EB030C02F8BA
:106BE0000C50401C80B20428EDD31B1D7F1C9DB2AD
:106BF000BFB202990020B7EB0B028841FFF648AF05
:106C000004E084F8A8178E4842556D1C8C49A5EB0A
:106C1000090701EB09003A0A824642708770002397
:106C20008B460CE009EB030159448846C879DDE93D
:106C30000021F2F70FFD88F807005B1C9BB29F4212
:106C4000F0DC94F8E70328B1B9B2504600230422DF
:106C5000F3F7DCF9B9B25F465046F2F7E9FA010AF8
:106C600079556D1CA9B27854491C94F8A6078DB2C9
:106C700002280DD194F8A50750B1681F010AF970D8
:106C8000387181B2781D01F0FCF978556D1CADB2F8
:106C9000356001216C48F2F721FB09B02846BDE8B8
:106CA000F08F94F8A607DFF8A4C1694AACF1850912
:106CB00009F17A074FF47A7B42F21078A9F1020EBB
:106CC000A7F16701924630B1012877D0022876D02B
:106CD000032875D146E394F8E206C0F3C3000E28FA
:106CE0006ED2DFE800F0071523313E4D5C6E7D8CDF
:106CF0009BE4F5F30027E04604E018F80700E855A8
:106D00007F1CBFB25148F1F7BEFAB842F5D844E350
:106D1000002404E019F804002855641CA4B24B4870
:106D20008538F1F7B0FAA042F4D8D0E300247746D2
:106D300003E0385D2855641CA4B244488738F1F755
:106D4000A2FAA042F5D8C2E3002403E0385D28553A
:106D5000641CA4B23D480B38F1F795FAA042F5D86F
:106D6000B5E33A4F00241C3F03E0385D2855641C0E
:106D7000A4B236481C38F1F786FAA042F5D8A6E34B
:106D8000324F00242D3F03E0385D2855641CA4B227
:106D90002E482D38F1F777FAA042F5D897E3284F1F
:106DA0000024323F03E0385D2855641CA4B2244817
:106DB0003238F1F768FAA042F5D888E3AAE0E8E1B2
:106DC00058E2224F00243C3F03E0385D2855641C04
:106DD000A4B21E483C38F1F756FAA042F5D876E343
:106DE0001A4F0024163703E0385D2855641CA4B2FE
:106DF00016481630F1F747FAA042F5D867E3134F6B
:106E000000240A3703E0385D2855641CA4B20F48FB
:106E10000A30F1F738FAA042F5D858E394F8A507FC
:106E20000A4C643C02281CD00020215C2954401CE0
:106E300080B20D28F9D35046F1F725FA002309E076
:106E400052020020A4120020B86402404FCC010876
:106E50009D2900201A4650EA02011ED00021FE4C56
:106E600016E0002703E0E05DE8557F1CBFB2FB4859
:106E7000F1F709FAB842F6D817E1671807F5805715
:106E800097F8F97605EB010C8CF80D70491C89B266
:106E90000F1A73EB0207F0DB2CE1F148F1F7F3F97D
:106EA00087B202E10121EF48F2F718FA20E3EB4F35
:106EB0000024853703E0385D2855641CA4B2E748F8
:106EC0008530F1F7E0F9A042F5D800E312E0FFE7E2
:106ED000DFF888930027A9F1150904E019F80710D5
:106EE000E9557F1CBFB2DD481538F1F7CCF9B8423F
:106EF000F4D813E2A94600270D4604E0E95D09F83D
:106F000007107F1CBFB2D5480E38F1F7BCF9B84264
:106F1000F4D803E294F8E206C0F3C3000D28C5D20A
:106F2000DFE800F007212E3D4C5B6A798897F0FF7F
:106F3000ED00DFF828830027A8F1070804E018F81F
:106F40000700E8557F1CBFB2C448C01FF1F79BF98A
:106F5000B842F4D837600121C248F2F7BFF9584669
:106F6000C4F88406C4E20024BF4F03E0385D28550E
:106F7000641CA4B2BC48F1F786F9A042F6D8A6E298
:106F8000B94F0024AF3703E0385D2855641CA4B224
:106F9000B548AF30F1F777F9A042F5D897E2B24F94
:106FA00000240A3703E0385D2855641CA4B2AE48BB
:106FB0000A30F1F768F9A042F5D888E2AA4F002418
:106FC000153703E0385D2855641CA4B2A648153077
:106FD000F1F759F9A042F5D879E2A34F0024203700
:106FE00003E0385D2855641CA4B29F482030F1F7B7
:106FF0004AF9A042F5D86AE29B4F0024293703E002
:10700000385D2855641CA4B297482930F1F73BF944
:10701000A042F5D85BE2944F0024383703E0385D96
:107020002855641CA4B290483830F1F72CF9A042DE
:10703000F5D84CE28C4F0024563703E0385D2855D4
:10704000641CA4B288485630F1F71DF9A042F5D867
:107050003DE294F8A507844C6334022819D000203F
:10706000215C2954401C80B21428F9D31046F1F752
:107070000AF9044600277DA1504605F0B7F90146FC
:1070800054EA07003FF409AF0020A1F1010C724B54
:1070900018E0002703E0E05DE8557F1CBFB27248AE
:1070A0006330F1F7F0F8B842F5D83760FAE61A180D
:1070B00002F5805292F8F92605EB000888F81420B2
:1070C000401C80B26045F2DB22206A18D074641C38
:1070D00047F100020AE0581800F5805090F8F806D1
:1070E00005EB010C8CF81400491C89B2081B77EBE6
:1070F0000200F0DB5EA15A48F1F7B9F8CDE62FE0C7
:107100000FE0FFE7584F0024933703E0385D285520
:10711000641CA4B254489330F1F7B5F8A042F5D8F6
:10712000D5E1D4F8841640F2E930814207D194F8D1
:10713000E20620F07800603084F8E20601E0C4F84E
:107140008406464F0024193F03E0385D2855641C2F
:10715000A4B242481938F1F796F8A042F5D8B6E142
:10716000DFF80481002708F1A40804E018F80700FC
:10717000E8557F1CBFB23C48A430F1F784F8B84210
:10718000F4D8376001213748F2F7A8F843F6982081
:10719000E6E694F8E206C0F3C30005286AD2DFE809
:1071A00000F00313708DCF00002084F8A707044679
:1071B00003E0385D2855641CA4B228485930F1F723
:1071C00062F8A042F5D882E1002184F8A7170846AA
:1071D0002954401C80B26428FAD384F8A7172249A6
:1071E00000205B390A5C2A54401C80B20828F9D37D
:1071F000DFF8649041F26771002709EB010A09E0AA
:1072000009EB070000F5805090F86717E819017244
:107210007F1CBFB25046F1F736F8B842F0D82C21A7
:10722000EA19AA461172093741F28F72BFB20025DE
:1072300009EB020B0AE009EB050000F5805090F81D
:107240008F177A190AF802106D1CADB25846F1F783
:107250001AF8A842EFD80EE0A4120020EBCB0108E8
:1072600052020020B864024026CD01082C00000024
:107270000D0A0000FAE0AFF208019F48F0F7F7FFAF
:107280005AE00027DFF8748204E018F80700E85598
:107290007F1CBFB29948F0F7F6FFB842F5D83760C7
:1072A00001219748F2F71AF894F8E20620F07800E6
:1072B000183084F8E2064FF4FA6051E694F8A50716
:1072C0008E49293902284FF0000017D000222A5495
:1072D000401C80B26428FAD384F8A72700200A5CF7
:1072E0002A54401C80B20E28F9D35046F0F7CBFF49
:1072F0000104090C20D00020824A1AE084F8A70774
:107300000027894604E019F80710E9557F1CBFB231
:107310007A482938F0F7B7FFB842F4D83760E1E08F
:10732000131803F5805393F8F9362F18BB73401CDC
:1073300080B28842F4D38EE76F48F0F7A4FFD0E024
:10734000DFF8B891002709F10C0904E019F80710DB
:10735000E9557F1CBFB269480C30F0F794FFB84282
:10736000F4D8DBE794F8E206C0F3C30009287DD225
:10737000DFE800F005202D3B4857669FAF0000274F
:10738000E04604E018F80700E8557F1CBFB25B48F0
:10739000C238F0F778FFB842F4D837600121584876
:1073A000F1F79CFF94F8E20620F07800083084F8AA
:1073B000E206D4E5002404E019F804002855641C12
:1073C000A4B25148F0F75FFFA042F5D87FE0002457
:1073D000774603E0385D2855641CA4B24A48801EF5
:1073E000F0F751FFA042F5D871E0002403E0385DCA
:1073F0002855641CA4B244487A30F0F744FFA042F8
:10740000F5D864E03D4F00246D3F03E0385D28551A
:10741000641CA4B239486D38F0F735FFA042F5D8A6
:1074200055E0364F00245E3F03E0385D2855641C6C
:10743000A4B232485E38F0F726FFA042F5D846E005
:1074400094F8A5072D4F973F022810D00020395CF3
:107450002954401C80B20F28F9D35046F0F713FF8F
:107460000104090C20D00020264A16E040E0002448
:1074700003E0385D2855641CA4B220489738F0F723
:1074800002FFA042F5D822E0131803F5805393F8C9
:10749000F9362C18E373401C80B28842F4D3AFF263
:1074A00030211548F0F7E3FE1348F0F7ECFE84B204
:1074B0000DE0124F0024543F03E0385D2855641C52
:1074C000A4B20E485438F0F7DEFEA042F5D834607E
:1074D000E8E400200A5C2A54401C80B20728F9D353
:1074E000401E306001210648F1F7F8FEC4F884869A
:1074F00009B00020BDE8F08F5202002011CD010834
:10750000B8640240A4120020CACB010870B5164C22
:1075100040F224452946204603F03BF9002821D0BB
:107520002946204603F0D2F8104D00212846F1F7F5
:10753000D5FE61102846F1F7BBFE0D49012081F808
:10754000A7072088A088281D0268C2F5FA62A1F862
:107550006A264FF4FA6101602846BDE870400121B7
:10756000F1F7BCBE70BD000000100140886402400D
:10757000A422002010B5074C05492046F1F798FEDB
:1075800000212046F1F7AAFE03490120087010BD32
:1075900000800028B8640240180200202DE9F04362
:1075A00001218FB0880500F07BFBDFF894904846FE
:1075B000F1F79EFE4020050103900024CDE905452A
:1075C000C60207940894CDE909464FF000681E48AA
:1075D0000B940C940D941B4FCDF800800E94CDE9C4
:1075E000017069464846F1F72BFF012210214846F9
:1075F000F1F710FFDFF84890A9F130094846F1F79C
:1076000077FE4FF4FA60CDE90340CDE905450794D4
:107610000894CDE909460D480B940C940D94CDF8CF
:1076200000800E94CDE9017069464846F1F708FFE5
:1076300001214846F1F752FE0FB0BDE8F08300008B
:10764000B86402400410014052020020347400204B
:107650007CB50121032000F023FB164E07220621F2
:107660003046F2F797FC072211463046F2F792FCBB
:1076700002218DF8051000258DF806500124C02048
:107680008DF8074000908DF8041069463046F2F7F7
:1076900045FC202000908DF804408DF80650032012
:1076A0008DF805008DF8074069463046F2F736FC44
:1076B0007CBD000000040240F0B589B00025FFF752
:1076C000C7FFFFF76BFF4FF4E13000F00FF900F058
:1076D000EFF80121402000F0FBFA012000F07CFBD4
:1076E0004FF47A77384604F0E1FC5E4C0B2084F8C6
:1076F0002C01002684F828612676A6766676E67642
:10770000276284F82860012384F82A3084F829301D
:1077100084F82B30F80020632670A3706370E37048
:10772000A7602673A3736373E373001160614E490E
:107730000E708E704B70CB704EF660278F604B4A88
:1077400042F6F82CA1F27441A4F27C6405EB4500EA
:1077500002EB8000A0F5156000F500500670867001
:107760004370C670C0F808C06D1C042DEED394F8A9
:10777000A307000706D094F8A30700F00F00401EEF
:1077800084F8A50794F8A307000906D094F8A30786
:10779000FF2303EB101084F8A60784F8AA6794F877
:1077A000A60768B1324B01280DD0022808D0032863
:1077B00011D147F23050C1F87C04C3F888620AE066
:1077C000C1F87C7407E0C1F87C74C3F8886243F6A2
:1077D0009820C4F88406274827490068086025488F
:1077E000001D006848602348083000688860002059
:1077F000131803F5805383F82B67401C1428F7D324
:10780000087A04AFCD7A8B7A4A7A87E82D00087916
:10781000CD798B794A798DE82D0012488B780A78DA
:1078200016A1AF3003F054F800210320F1F796FFC2
:1078300010B11D48C0F8886294F8A5171B480029AC
:107840004FF0200104D009B0BDE8F040F2F7B9BB19
:10785000F2F7B9FB94F8E20640F0800084F8E20603
:1078600009B0F0BD2029002018570020A4120020E4
:1078700000004042107AFF1F047C0020253032783F
:1078800025303278253032782530327825303278FC
:1078900025303278253032782530327825303278EC
:1078A00025303278250000000000424200040240EA
:1078B00038B546208DF8000002208DF80100012423
:1078C0008DF802408DF803406846FBF7C3FE252083
:1078D0008DF800008DF8014000208DF802008DF831
:1078E00003406846FBF7B6FE38BD00001FB50446EE
:1078F0000121102000F010FA0020ADF804000094DF
:10790000ADF80600ADF80800ADF80C000C200D4CE9
:10791000ADF80A006946204602F072FF01212046B8
:1079200002F0D7FE012240F22441204602F050FF2F
:107930001021204602F0CAFE0122C021204602F09A
:10794000D2FE1FBD001001402DE9FC470121592046
:1079500000F0A6F943F6F8700024DFF8A0A000902C
:107960008DF8044002268DF8076069465046F2F70C
:10797000D5FAFC20DFF8889000908DF804400125AE
:107980008DF8075069464846F2F7C8FADFF8748068
:107990004FF440478DF8044000978DF80750694632
:1079A0004046F2F7BBFA8DF804408DF807600720D7
:1079B000154E009069463046F2F7B0FA072130467E
:1079C000F2F7FFFA39464046F2F7FDFA4FF47C51E0
:1079D0005046F2F7F8FAF8215046F2F7F2FAFC2195
:1079E0004846F2F7F0FA0948D0F828120848012969
:1079F00002D00470BDE8FC870570FBE70010024070
:107A000000180240000C0240000002400000424208
:107A1000A412002070B5FFF797FF642004F046FB26
:107A20002048D0F83C3201221F4920480024E3B10D
:107A300080F8A547D1F814021D4978B30C761D488B
:107A4000D0F81C22D0F81832120142EAC302D0F852
:107A5000143242EA8302D0F81032D0F80C0242EA23
:107A60004302024318324A7070BDD1F818328BB10C
:107A700080F8A527D1F80832D1F80C5243EA450323
:107A8000DB4380F8A63790F8A63703F0030380F8AD
:107A9000A637CFE7022380F8A537EBE7FFE70A76A2
:107AA000CDE700000080414200004342A4220020B4
:107AB000A4120020000042422DE9FC4101211120C6
:107AC00000F0EEF801248DF8044000254CF204008B
:107AD0008DF806500326184F00908DF805608DF83C
:107AE000074069463846F2F719FA04213846F2F79A
:107AF00068FA124890F8A617032903D090F8A60751
:107B0000012812D18DF804408DF8065004200C4D48
:107B100000908DF805608DF8074069462846F2F719
:107B2000FDF904212846F2F74CFA0648C0F8B8429D
:107B3000C0F8BC42BDE8FC8100100240A422002035
:107B40000000024000004242FFF7B6BF2DE9FE43AD
:107B500016200A9D16461F468DF800004B4800EB84
:107B60004114202109E09DF80000204480F85B1FAB
:107B70009DF80000401C8DF800009DF800002028B2
:107B8000F1D34FF0000840460BE09DF80000394665
:107B900082003046F0F747FB084308D09DF800000C
:107BA000401C8DF800009DF800001028EDD39DF8D2
:107BB0000000A84216D8FDB19DF8000020B99DF83C
:107BC000000028448DF800009DF80000401C8DF84E
:107BD00000009DF800103020C1F11E01214481F801
:107BE0005B0F00E045B101208DF80400C5F11E01D6
:107BF00021442E2081F85B0F404614E09DF80800D8
:107C0000394682003046F0F70EFB00F00F009DF879
:107C100008103030C1F11E01214481F85B0F9DF83E
:107C2000080000F101008DF808009DF80800A84246
:107C3000E4D39DF8040028441BE09DF808009DF85B
:107C40000410401A820030463946F0F7ECFA00F092
:107C50000F009DF8081030309DF80420A1EB0201C0
:107C6000C1F11E01214481F85A0F9DF8080000F16E
:107C700001008DF808009DF800009DF804100844EC
:107C80009DF808108842D8D8BDE8FE83A4120020D1
:107C90004FF400610148F2F78DB900000004024082
:107CA000044A0029116801D0014300E081431160BA
:107CB0007047000030380240044A0029116801D0A2
:107CC000014300E08143116070470000103802401A
:107CD000044A0029116801D0014300E0814311608A
:107CE0007047000034380240044A0029116801D06E
:107CF000014300E0814311607047000040380240BA
:107D0000044A0029116801D0014300E08143116059
:107D10007047000020380240044A0029116801D051
:107D2000014300E081431160704700004438024085
:107D3000044A0029116801D0014300E08143116029
:107D4000704700002438024070B5204B1968204C61
:107D500011F00C0104D06610042903D0082903D0C7
:107D600004601BE0066019E0184A121F1168C1F395
:107D70008055116801F03F0115B1B6FBF1F101E04A
:107D8000B4FBF1F114681268C4F388146143C2F3C0
:107D90000142521C5200B1FBF2F1016019680F223E
:107DA00002EA11110B4A545C0168E14041601C6811
:107DB000072505EA9424145D21FA04F484601B6805
:107DC00005EA5333D25CD140C16070BD083802402F
:107DD0000024F4000000002005490028086802D0B3
:107DE00040F0040001E020F004000860704700004B
:107DF0000008065001480068704700000808065057
:107E000070B5012080F310880C4D10212846F2F740
:107E1000D8F808212846F2F7D6F8D720F0F74CFF1B
:107E2000FF20F0F749FF044610212846F2F7CBF86F
:107E3000002181F31088204670BD00000000024040
:107E400070B5012080F31088194C0020A080FFF746
:107E5000D7FF000609D4012004F028F9A088401CAF
:107E600080B2A080C828F2D31EE0A088C8281BD208
:107E7000104D10212846F2F7A4F808212846F2F701
:107E8000A2F89F20F0F718FFFF20F0F715FFFF2062
:107E9000F0F712FF607010212846F2F794F80020E6
:107EA00080F31088607870BD002080F3108870BD6A
:107EB000220A00200000024070B5012188B088032A
:107EC000FFF712FF01210220FFF7EAFE00244FF422
:107ED00000602F4E8DF8044000908DF807406946F1
:107EE0003046F2F71BF801218DF8041002258DF8B9
:107EF000055008038DF806408DF80710009069467C
:107F00003046F2F70BF805220D213046F2F742F821
:107F100005220E213046F2F73DF805220F213046AA
:107F2000F2F738F84FF4604000908DF804500320C9
:107F30008DF805008DF806408DF8074069463046FB
:107F4000F1F7ECFF134D284600F04AF8ADF8104069
:107F50006815ADF812001820ADF814000720ADF830
:107F60001800ADF808404FF48270ADF80C40ADF841
:107F70000A00ADF80E40ADF8164002A9284600F000
:107F800064F80121284600F021F808B070BD000017
:107F9000000402400038004070B50B4C0546022139
:107FA000204600F047F80028F9D02946204600F086
:107FB0004AF80121204600F03DF80028F9D020467B
:107FC00000F03FF8C0B270BD0038004000290188C1
:107FD00002D041F0400101E021F0400101807047F2
:107FE000114910B588420AD1841401212046FFF7B7
:107FF0009FFE2046BDE810400021FFF799BE0B49C7
:10800000884202D10121041404E0094988420AD1BE
:108010000121C4132046FFF773FE2046BDE810403F
:108020000021FFF76DBE10BD003001400038004058
:10803000003C00400246002012890A4200D0012084
:108040007047808970478181704730B502884C88BD
:1080500002F441530A88CD8822438C882C43224362
:108060000C8922434C8922438C892243CC892243A8
:108070001A430280828B22F400628283098A018281
:1080800030BD0246002003E012F8013B1844C0B2A4
:10809000491E89B2F8D270472DE9F04101218D07C0
:1080A0000024284601F000FFF0B3F1F79FFF284EAF
:1080B000002006F580533DE006EB840101F5805178
:1080C000D1F8F8271278012AD1F8F82703D052788E
:1080D000012A08D02CE01070D1F8F8275070D1F8A0
:1080E000F827907030E0D1F8F827927802BBD1F8E9
:1080F000F82757687F1C5760D1F8F8275268D1F8E5
:10810000F877BF68BA4213D3D1F8F8770122BA7072
:10811000D1F8F827D278012A16D0D1F8F827507074
:10812000D1F8F827506000E008E0D1F8F817C870DF
:10813000641CE4B293F8F617A142BDD82846BDE806
:10814000F041012101F0FABDD1F8F8174860EFE7DE
:10815000A41200200CB50022254900920192086863
:1081600040F4803008604FF4A063086800F40030E9
:1081700001900098401C0090019810B90098984216
:10818000F3D10868800330D50120019018484030B1
:10819000026842F0805202601648026842F480424F
:1081A00002601348083002680260026802600268D8
:1081B0000260031F104A1A600A6842F080720A6067
:1081C0000A689201FCD50D4A40F205611160016810
:1081D00021F003010160016841F0020101600168C2
:1081E000C1F381010229FAD10CBD01920CBD00003E
:1081F000003802400070004008544007003C024034
:108200007CB500229FED170A00928DED010A6D46A4
:1082100001AC16E0835CA3F13006102E05D2009B62
:108220001B010093865C303E07E0413B062B0CD2DD
:10823000009B1B010093865C373E1E43521CD2B24A
:1082400000968A42E6D3002006E0BFEE000A7CBD1D
:108250002A5C2254401CC0B2B0EB510FF8D39DED04
:10826000010A7CBD0000000030B505460022104622
:1082700011E0AB5CA3F13004102C02D244EA0010F0
:1082800007E0A3F14104062C08D20401A3F1370052
:108290002043521CD2B28A42EBD330BD4FF0FF30A4
:1082A00030BD00002DE9FE43534C4FF03809A07853
:1082B00000263146F9F794FC012508270096CDE900
:1082C00001750246182000234946FBF713FC00F114
:1082D000040808EB48004006000E08232D224946FA
:1082E0000095FBF799FB607808F101080021F9F788
:1082F00077FC0246009608EB4800CDE90175400680
:10830000000E00234946FBF7F5FB804408EB4800CC
:108310004006000E08232D2249460095FBF77CFB02
:10832000207808F101080021F9F75AFC024600966E
:1083300008EB4800CDE901754006000E00234946D0
:10834000FBF7D8FB804408EB48004006000E0823EA
:10835000202249460095FBF75FFB607908F1010890
:108360000021F9F73DFC0246009608EB4800CDE9F4
:1083700001754006000E00234946FBF7BBFB804415
:1083800008EB48004006000E08232D2249460095C0
:10839000FBF742FB207908F101080021F9F720FCE6
:1083A0000246009608EB4800CDE901754006000E34
:1083B00000234946FBF79EFB804408EB480040063B
:1083C000000E08232D2249460095FBF725FBE07897
:1083D00008F101080021F9F703FC0246009608EBBA
:1083E0004800CDE901754006000E00234946FBF721
:1083F00081FBBDE8FE8300008C2600200249087145
:108400000120C87170470000A41200202DE9F04F30
:10841000002587B02F46F1F7D3FBF74EF0790028FF
:108420007ED0A94686F80790FBF750F930794FF0D7
:10843000080A4FF001084FF0100B06F58054102881
:1084400081F00E84DFE810F010008D00F9007F024B
:10845000FF0343044505FD06EB075608AB08670913
:10846000060A4B0AEB0AE50BF1F7B0FD01280AD02A
:10847000022808D0042806D0082804D10220FFF7DB
:10848000BDFF84F8E091CDE900B8002145461523F1
:10849000DAA20846FBF7FBFB94F8E10128B3CDE92B
:1084A00000A557460523DAA214210020FBF7EFFBB5
:1084B000CDF80090CDE9017594F8E1210023142155
:1084C0001E20FBF717FBCDE9007594F8E1010A23A4
:1084D00000EB400101EB001006EB001141F63240C9
:1084E0000A1814212820FBF7D2FB94F8E001FF289A
:1084F00029D094F8E001CDE900050A2364221E2169
:108500001846FBF707FACDF80090CDE901A594F8DD
:10851000E0214E4600232D213220FBF7EBFA00E04C
:10852000F5E300EB4000322101EB4000C0B208232C
:1085300025222D210095FBF76FFA94F8E0016428BD
:1085400009D001F08DBBCDE900A515232D21B2A2E4
:10855000142001F061BA84F8E0610220FFF74EFFB9
:10856000EFE7F1F733FD01280BD0022809D00428EA
:1085700002D0082805D101E0092000E00420FFF71F
:108580003DFF94F8A40738B194F8A50738B1012845
:1085900008D0022811D108E01523A3A207E0152373
:1085A000A4A204E01523A7A201E01523A8A2CDE907
:1085B00000A800210846FBF76AFBF078012802D0EA
:1085C00002280CD101E0A64901E0A5491231CDE90C
:1085D000001809231A460A210020FBF70BFBA048CC
:1085E00018234838CDE9000844461A46002168207F
:1085F000FBF700FBCDE900A45546152399A21A21EB
:108600000020FBF744FBCDE9005415239BA2242155
:108610000020FBF73CFBCDF80090CDE90154B26D92
:10862000002324215420FBF765FAB06D10B9022015
:10863000FFF7E4FEFFF736FE83E7F1F7C7FC0128FA
:1086400006D002280ED0042814D008281BD125E01B
:108650000320FFF7D3FE94F8DC0120F0800084F8BB
:10866000DC0110E094F8DC0120F0800084F8DC01EB
:10867000032006E094F8DC0120F0800084F8DC019F
:108680000920FFF7BBFE94F8A40778B194F8A5077A
:10869000A8B1012816D002281CD120E094F8DC01F2
:1086A00020F0800084F8DC010420EAE7CDE900A88E
:1086B0000021152375A20846FBF7E9FA15E01523FA
:1086C0005CA201E015235FA2CDE900A800210846C5
:1086D000FBF7DDFA94F867060F2803D005E01523B1
:1086E0005BA2F1E70120FFF789FEF078012802D0B4
:1086F000022811D106E05A49CDE9001809231A468B
:108700000A2106E0564809231230CDE900081A462E
:108710000A210020FBF76EFA94F8E00110B1002066
:10872000FFF76CFE94F8A50758B394F8A6674C4A77
:108730005C32A2F12A00A2F10E05A2F11C03A0F105
:108740000E01022E07D094F8A667012E3FD094F8B0
:10875000A667E6B315E04F4ED6F80062C6B394F8AC
:10876000AA17322947D394F8AA173C293ED2CDE95B
:10877000005808230E220021592000E05920FBF761
:1087800039FA374818234838CDE9000845461A46D3
:1087900000216820FBF72EFACDE900B55F461023D3
:1087A0003DA214212820FBF772FACDE900A5564618
:1087B00015233BA224211220FBF769FA94F8DC016F
:1087C00000060AD510232E213AA2002001E087E0FE
:1087D00080E0CDE90075FBF75AFAFFF763FD94F8E6
:1087E000E206000672D594F8A827A1E094F8AA172B
:1087F00046296CD392E07CE0A41200204669726D99
:1088000077617265446F776E6C6F61640000000081
:10881000506F72743A000000446F776E6C6F616441
:10882000204661696C2100004E6F205369676E61BC
:108830006C000000547970653A53746174696F6E0E
:1088400000000000547970653A436C6F7564000055
:10885000547970653A436C6F75642D546573740078
:1088600074EC01084F66666C696E65205265636F33
:1088700072642055706C6F61640000005265636F14
:108880007264206E756D6265723A00004F66666CA8
:10889000696E650000004042424C5545534B5900FB
:1088A000454E4552475920544543484E4F4C4F473B
:1088B000590000005570677261646520455252206E
:1088C000436865636B2047756E0000002CE01DE077
:1088D0000E2203E0CDE9001808230E2200214DE707
:1088E00094F8AA67202EBFF435AF94F8AA671A2E21
:1088F00003D9CDE900280823EAE794F8AA27172A24
:108900003FF635AF94F8AA27142A03D9CDE90038E9
:108910000823DDE794F8AA27122ADBD9CDE900085D
:1089200008230E22002129E794F8E206C0F3C302CF
:10893000F7A103A801F0CCFF022303AACDE900654B
:108940003821002005E6F1F741FB012806D0022876
:108950001CD0042835D008283ED138E03F210FE054
:10896000707918B17079401E707100E07171707982
:1089700000EB8002C2EB8010304490F86000F8B940
:1089800070796D1CADB2402D26D8E9E7494614E058
:108990006D1CADB2402D1FD870793F2803D270797D
:1089A000401C707100E07171707900EB8002C2EBC5
:1089B0008010304490F8600010B970794028E7D3F7
:1089C0000AE0707984F8DB0C84F8DC8C04E0022087
:1089D000FFF714FD86F805903079344603287DD1E1
:1089E00060790122010906910021CB4801F044F988
:1089F000CDF80090CDE901B8607945465F464E4616
:108A000000EB8001C1EB8010204490F8602000232F
:108A100019465820FBF76EF8CDE900751023BFA268
:108A200019460020FBF733F9607900EB8001C1EBB8
:108A300080102044D0F861000021F9F7D1F80699A0
:108A4000024601EB410000EB011004EB001101F5BF
:108A50008051884691F8700D002300F00300CDE9A5
:108A60000007102102951820FBF744F8CDE90075A6
:108A70001023AFA220210020FBF709F9607900EB59
:108A80008001C1EB80102044D0F865000021F9F787
:108A9000A7F8024698F8700D0023C0F38100CDE9D5
:108AA0000007202102951820FBF724F8607900EBDD
:108AB0008001C1EB8010204490F883000021F9F779
:108AC0008FF80096CDE901A50246574638211820B7
:108AD0000023FBF70FF800F1040800E092E208EB36
:108AE000480040063821000E08232D220095FAF791
:108AF00093FF607908F1010800EB8001C1EB801061
:108B0000204490F882000021F9F76AF802460096A6
:108B100008EB4800CDE9017540063821000E00231E
:108B2000FAF7E8FF804408EB480040063821000EC1
:108B300008232D220095FAF76FFF607908F10108EC
:108B400000EB8001C1EB8010204490F881000021EF
:108B5000F9F746F80246009608EB4800CDE90175A2
:108B600040063821000E0023FAF7C4FF804408EBCA
:108B7000480040063821000E082320220095FAF70D
:108B80004BFF607908F1010800EB8001C1EB801018
:108B9000204490F886000021F9F722F8024600965A
:108BA00008EB4800CDE9017540063821000E00238E
:108BB000FAF7A0FF804408EB480040063821000E79
:108BC00008232D220095FAF727FF607908F10108A4
:108BD00000EB8001C1EB8010204490F8850000215B
:108BE000F8F7FEFF0246009608EB4800CDE9017554
:108BF00040063821000E0023FAF77CFF804408EB82
:108C0000480040063821000E08232D220095FAF76F
:108C100003FF607908F1010800EB8001C1EB8010CF
:108C2000204490F884000021F8F7DAFF024600960D
:108C300008EB4800CDE9017540063821000E0023FD
:108C4000FAF758FF7DE4F1F7C1F9012806D00228B0
:108C500009D004280ED008281ED121E07079D8B19F
:108C60007079401E04E07079032815D27079401C99
:108C7000707111E0707930B1012806D0022806D059
:108C8000032809D105E0052004E0062002E00720C2
:108C900000E00820FFF7B2FB3079042805D050E44B
:108CA0000220FFF7ABFB4846E2E71B480422002105
:108CB000803800F0E1FFCDE900B9707916498039BC
:108CC00001EB001270790007010E1023FEE3F1F7AB
:108CD0007DF9082802D10420FFF790FB30790528A0
:108CE000B0D10D4804220021403800F0C5FF94F8AF
:108CF000A50720B1012825D002283DD158E0102336
:108D0000AFF2D042CDE900A81946002032E0F0E3EE
:108D100025303278000000005EED01084C3A20203A
:108D200020202020202020202020202000000000C3
:108D3000503A2020202020202020202020202020E9
:108D40000000000047461023AFF20852CDE900A80A
:108D500019460020FAF79BFFCDE900A71023FDA2DA
:108D600038210020FAF793FFCDE900A71123FB4A31
:108D700038211E20FAF78BFF94F8A50700288ED023
:108D800094F8A617F64841F23F72871841F22B7209
:108D900000EB020921B394F8A60701285AD094F8F1
:108DA000A607022871D094F8A60703287DD043E4D3
:108DB000CDE900A810235746EAA219460020FAF789
:108DC00066FFCDE900781023E2A238210020FAF7EF
:108DD0005EFFCDE9007811233821E64A1E20C9E75D
:108DE000701900F5805090F8E40618B96D1CADB20A
:108DF000152DF5D3CDE900A8444655461023DEA233
:108E00001A210020FAF743FFCDE9005410233A4617
:108E10001A212420FAF73BFF707818280AD9CDE9E7
:108E200000541023D6A224210020FAF730FF142387
:108E30004A460AE0CDE900541023D1A224210020A3
:108E4000FAF725FFC54A14232A322E21CDE9005412
:108E5000002077E5701900F5805090F8E40618B905
:108E60006D1CADB2152DF5D3CDE900A8444655468D
:108E70001023C1A21A210020FAF709FF10231A219A
:108E80003A46242020E000E00FE0CDE900A8444667
:108E900055461023BCA21A210020FAF7F8FEAF4A6B
:108EA000102361321A211E200EE0CDE900A84446AD
:108EB00055461023B6A21A210020FAF7E8FEA74A69
:108EC0001023A6321A211220CDE90054FAF7DFFE52
:108ED000A5E7F1F77BF8012804D0022807D008287D
:108EE0000FD10BE0707960B17079401E04E07079A9
:108EF000032806D27079401C707102E00420FFF74D
:108F00007DFA307906287DD104220021A14800F0A5
:108F1000B3FE4FF00009CDF80090CDE901B844460A
:108F20007279B346B046012349463E20521CFAF7F7
:108F3000E1FDCDE900A45646102397A20021482068
:108F4000FAF7A5FEDFF85CA2CDE900A408231A46D3
:108F500000217820FAF74EFECDE90064102392A29A
:108F600008214820FAF793FE0823CDE900A91A4604
:108F700019467820FAF73EFECDE9006410238DA251
:108F800019460020FAF783FE98F8050000EB40012F
:108F900001EB001108EB011000F5805090F8610D15
:108FA0004FF01003012844D084A2CDE900641021C1
:108FB0001E20FAF76CFECDE90064A046102381A2C2
:108FC00018210020FAF763FE9BF8050000EB400132
:108FD00001EB00100BEB001000F5805090F85A0DDB
:108FE000CDE9006805289BF8050000EB400101EB86
:108FF00000100BEB001000F580501CD090F85A0DBB
:10900000644900E00AE2403101EB00120C23182110
:109010003620FAF73CFE0120CDE90060B04610236F
:109020006BA220210020FAF732FE09264FF0200B18
:10903000F7E06AA2B9E790F8600D5649B031E3E76E
:1090400006EB46014FF07A09B9EB410F02D27F1CC3
:10905000BFB20026607900EB400101EB001004EB89
:10906000001000EB051000F5805090F8860D4FF0D1
:10907000000AC009CDF800A0CDE90180607900EBBD
:10908000400101EB001004EB001000EB051000F5AF
:10909000805090F8842D0BEBC700C1B206EB460060
:1090A0004006000E5346FAF725FD304486B206EB23
:1090B0004601B9EB410F02D27F1CBFB20026607996
:1090C00000EB400101EB001004EB001000EB051079
:1090D00000F5805090F8860D0823C00900900BEB36
:1090E000C700C1B206EB46004006000E2D22FAF77B
:1090F00093FC761CB6B206EB4601B9EB410F02D2E7
:109100007F1CBFB20026607900EB400101EB00102C
:1091100004EB001000EB051000F5805090F8860D70
:10912000CDF800A0C009CDE90180607900EB4001D5
:1091300001EB001004EB001000EB051000F580506F
:1091400090F8852D0BEBC700C1B206EB46005C46DC
:10915000400647E055524C3A00000000AA29002082
:10916000A4120020547970653A436C6F75642D54D5
:1091700061737400F8CB010841504E203A000000A2
:10918000494D45493A000000535349443A00000014
:1091900049503A009EED01084F6E4C696E65203AC9
:1091A0002000000024EC01084F66664C696E653AA9
:1091B00020000000547970653A00000052533438A2
:1091C0003500000050726F746F636F6C3A000000DE
:1091D00047756E2D416464723A0000004C4F524155
:1091E00000000000000E0023FAF784FC304486B231
:1091F00006EB4601B9EB410F02D27F1CBFB200263D
:109200000120009004EBC700C1B206EB4600400607
:10921000000E08233B22FAF7FFFB761C6D1CB6B24A
:10922000ADB2F74C607900EB400101EB001004EBAC
:10923000001000F5805090F85B0DA8423FF600AF9B
:10924000ECE0F0F7C3FE012804D0022807D008287C
:109250000FD10BE0707960B17079401E04E0707935
:10926000032806D27079401C707102E00420FFF7D9
:10927000C5F830790728E3D10124F47104220021D4
:10928000E04800F0F9FC0020CDE9000B029472796F
:10929000014601234020521CFAF72CFC0820CDE99E
:1092A00000041023D8A214210020FAF7F0FC0924AE
:1092B000A5E004EB44014FF07A09B9EB410F02D26B
:1092C0007F1CBFB200244FF0000A4FF001080821B4
:1092D000CDF800A0CDE90118707900EB400101EB59
:1092E000001006EB001000EB051000F5805090F820
:1092F000842D4FF0140B0BEBC700C1B204EB4400FC
:109300004006000E5346FAF7F5FB204484B204EB06
:1093100044017A20B0EB410F02D27F1CBFB200247F
:109320000BEBC700C1B204EB44004006C146000E7F
:1093300008232D22CDF80080FAF76EFB641CA4B23E
:1093400004EB44014FF07A08B8EB410F02D27F1CC6
:10935000BFB200240821CDF800A0CDE90119707931
:1093600000EB001101EB002006EBC00005EB05113E
:1093700000EBC10000F5005090F85802642110FB8A
:1093800001F0020A0BEBC700C1B204EB4400400637
:109390005E46000E0023FAF7ADFB204484B204EBD6
:1093A0004401B8EB410F02D27F1CBFB2002406EB90
:1093B000C700C1B204EB44004006000E082325227A
:1093C000CDF80090FAF728FB641CA4B204EB44012A
:1093D000B8EB410F02D27F1CBFB2002406EBC700DE
:1093E000C1B204EB44004006000E08233B22CDF836
:1093F0000090FAF711FB641C6D1CA4B2ADB2804E54
:10940000707900EB400101EB001006EB001000F555
:10941000805090F85B0DA8423FF64BAF19E2F0F791
:10942000D5FD082802D10420FEF7E8FF307908288E
:10943000F4D1744804220021403000F01DFCCDE935
:1094400000A847465446102372A214210020FAF7C0
:109450001EFCCDE9004710236F4A14211220FAF7B1
:1094600016FCCDE9004710236CA214215A20FAF70C
:109470000EFCCDF80090CDE901477278022314214B
:109480006C20FAF737FBB24605EB450000EB0511FF
:109490000AEB011841F66C5010F80800C00723D001
:1094A00005EB8501142000EB4106CDE90047F1B240
:1094B00005235BA20020FAF7EAFBCDF80090CDE986
:1094C000014701236A1CF1B21E2000E065E0FAF7B3
:1094D00011FB41F66251CDE9004708EB0102F1B200
:1094E0000A232A20FAF7D3FB6D1CADB2042DCBD38F
:1094F000B6E3B7E3F0F76AFD012806D002280BD0E7
:10950000042811D0082830D133E0707910B1707977
:10951000401E25E0052023E07079052802D27079ED
:10952000401C1DE048461BE0707906281DD2DFE88C
:1095300000F00305070911190A2014E00B2012E0BE
:109540000C2010E00D20FEF759FF94F8A30700F05F
:109550000F0005E00E20FEF751FF94F8A307000965
:10956000707102E00F20FEF749FF3079092804D01E
:1095700076E30220FEF742FFD4E77079214C042203
:10958000803404EB0010002100F076FBCDE900B937
:109590007079102304EB0012002100203CE2F0F768
:1095A00015FD012806D0022809D004280ED008286D
:1095B00064D167E0707910B37079401E04E070796F
:1095C00003285BD27079401C707157E0707900EB12
:1095D000400101EB001006EB001000F5805090F800
:1095E000610D012820D0707900EB400101EB0010E3
:1095F00006EB001000F5805090F8610D40B33DE09F
:10960000A41200207EEE010847756E2D5253534977
:109610003A00000053563A00FCC4010848563A008C
:10962000506F72742D00000070794C4600EB4001C1
:1096300001EB001006EB001000F5805080F8619DF2
:1096400071790220F0F78AF8FC48C0F8884215E0EA
:109650007079444600EB400101EB001006EB00106E
:1096600000F5805080F8618D7079F8F78BFFF34832
:10967000C0F8884271790220F0F770F830790A2832
:1096800005D0EDE20920FEF7B9FE48469CE704222A
:109690000021EB4800F0F0FACDE900A84446554619
:1096A0001523E8A214212820FAF7F1FACDF800904A
:1096B000CDE901547279012314214620521CFAF796
:1096C00019FA707900EB400101EB001006EB001075
:1096D00000F5805090F8610D01280CD0707900EBF6
:1096E000400101EB001006EB001000F5805090F8EF
:1096F000610D18B10AE01523D4A201E01523D6A20A
:10970000CDE900541E210020FAF7C1FA1523D5A295
:109710003221FFF79BBBF0F759FCD74C012806D04C
:1097200002280FD004281AD0082830D11CE0707904
:1097300068B394F88D0410B17079F8F723FF70794D
:10974000401E0AE07079032821D294F88D0410B1EC
:109750007079F8F717FF7079401C707117E084F882
:109760008D8484F8818412E00920FEF747FE484684
:1097700086F8059084F8808494F88D1439B1AF4947
:10978000C1F8880284F88D047079F8F7FBFE30790F
:109790000B2832D1AA4804220021403000F06CFA94
:1097A000CDE900A8454657461523A6A21221282038
:1097B000FAF76DFACDF80090CDE9017572790123C1
:1097C00012214620521CFAF795F9CDE900751523B0
:1097D000AAA21C210020FAF75AFACDE90075152338
:1097E000ACA226210020FAF752FACDE90075152324
:1097F000AEA230210020FAF74AFA94F88D0401282D
:1098000027D1454686F8078094F8820480B18B49B9
:10981000C1F8889284F8829470790121F8F7DCFF0E
:10982000CDE900A51523A6A238210020FAF72FFACA
:1098300094F88C0400280CD084F88C94CDE900A511
:109840001523A3A238210020FAF721FA7B48C0F89B
:10985000885205E2F0F7BAFB012813D0022811D094
:10986000042802D008280DD109E0EFF7A1FB142845
:1098700003D0484684F8E70304E04046FAE70920AD
:10988000FEF7BCFD30790C287ED16D480422002102
:10989000803000F0F1F9CDE900A845465646152381
:1098A0008FA21A210020FAF7F2F9CDE900651523FD
:1098B00090A224210020FAF7EAF9CDE900651523EA
:1098C00090A22E210020FAF7E2F994F8E7034FF076
:1098D000150310B191A2FFF731B896A2FBE7F0F79C
:1098E00075FB012806D002280BD0042812D00828C6
:1098F00057D165E0707910B17079401E08E00320FF
:1099000006E07079032802D27079401C00E04846D6
:10991000707146E0717994F8A30761F3030084F84D
:10992000A30700210320EFF719FF70B394F8A357A2
:10993000022004F5EE74FEF761FDEFF765FF84F891
:10994000C75500210320EFF709FF207820F0010020
:109950002070207840F006002070A4F802900021CA
:109960000120EFF7FBFE94F8060520F0800084F854
:10997000060594F8CA05A4F5EE74B0B1012819D013
:10998000022805D0032801E06AE10AE007D10CE0D3
:1099900094F8E20620F07800203084F8E206FDF723
:1099A0008BFE30790D280FD05AE194F8E20620F0B2
:1099B0007800F2E794F8E20620F078005830ECE7FF
:1099C0000920FEF71BFDA2E71D4804220021C0303C
:1099D00000F052F9CDE900B894F8A3075D46584F5E
:1099E00000F00F0007EB0012102319460020FAF7D1
:1099F0004EF994F8A307717900F00F00884202D065
:109A0000CDE9005901E0CDE9005870790C2307EB4E
:109A1000001220210020121DFAF739F920E1F0F799
:109A2000D5FA012806D0022805D0042804D0082839
:109A300003D1CBE086E08CE094E0CBE00000424232
:109A40008EEF0108504F52543A00000054595045CF
:109A50003A4C4F5241000000545950453A52533449
:109A6000383500005061737320456E746572204371
:109A700068616E6765000000A4520020313A4469B5
:109A800070207377697463682031616E6432204F8F
:109A90004E000000323A496E7365727420736C6137
:109AA0007665206D6F64756C65000000333A506117
:109AB000737320456E746572205374617274000074
:109AC00053746174653A53656E64696E6700000093
:109AD00053746174653A436F6D706C657465000012
:109AE000496E7365727420552D4469736B20466905
:109AF000727374005468616E205061737320456EF8
:109B000074657200466F726D61743A464154333227
:109B10003B4D41583A3332470000000046696E64BD
:109B200020552D4469736B2C4F7574707574696E74
:109B30006700000053746174653A49646C65000005
:109B4000CEF00108707910B17079401E08E0042051
:109B500006E07079042802D27079401C00E0484683
:109B6000707137E0717994F8A30761F3071084F8F6
:109B7000A30700210320EFF7F1FD58B30220FEF701
:109B80003DFC94F8E20620F0800084F8E20694F8A8
:109B9000A60780B1012813D0022802D0032807D1DC
:109BA00009E094F8E20620F07800203084F8E2061C
:109BB000FDF782FDD3E794F8E20620F07800F5E7A0
:109BC00094F8E20620F078005830EFE70920FEF71D
:109BD00015FCC4E730790E2842D104220021234825
:109BE00000F04AF8CDE900B894F8A3075D461F4F8E
:109BF00020F00F008037C219102319460020FAF711
